:10800000F0FE002021840000AB840000AB8400005F
:10801000AB840000AB840000AB84000000000000D3
:108020000000000000000000000000004F4A0100B6
:10803000AB84000000000000C54A0100AB840000D2
:10804000AB840000AB840000AB840000AB84000074
:10805000AB840000AB840000AB840000AB84000064
:10806000AB840000AB840000AB840000AB84000054
:10807000AB840000AB840000AB840000AB84000044
:10840000FFFFFFFFFFFFFFFFFFFFFFFFFEFFFFFF7D
:048410000000000068
:1084200013481449144A4FF0080333B140F8042BA1
:1084300041F8042BA3F10103F7E7EFF3088080F381
:108440000988EFF3148040F0020080F31488BFF332
:108450006F8FDFF82800016841F47001016008485F
:108460004FF00001016000F00DB880F308887047FC
:1084700080E100E080E200E0FFFFFFFF88ED00E028
:1084800034EF00E0C046C04600F002F800F00EF8FD
:108490004EF68851CEF20001086840F47000086082
:1084A0004FF00070E1EE100A7047FEE700F00BF8A5
:1084B000002801D000F00CF80020C046C04600F0B3
:1084C0001BF800F021F880B500F020F8012002BD73
:1084D00010B5074979441831064C7C44163404E041
:1084E0000A68081D511888470146A142F8D110BDFD
:1084F0005C2C0100BC2C010080B5024800F00CF897
:10850000002002BD0C6E010000F056B980B500F0ED
:10851000F6FC00F0D8FE01BDF0B583B00500686838
:108520000F3004092401DFF874020460DFF87002E0
:108530002060DFF8700220604FF4517200212000AB
:1085400001F03CF814F5D4702900302201F050F805
:10855000C4F8AC41D4F8B00100090001C4F8B0017E
:1085600000F0B4F801F069FA0500002D02D02800EF
:1085700000F0A2F8D4F8D001002804D0D4F8D061DB
:10858000D4F8B45117E0D4F8B401D82802D2D820D6
:10859000C4F8B401D4F8B40110F11005280001F0BA
:1085A00042FA0600002E02D1042000F085F80221D4
:1085B000300001F086FA2900300001F076FDA8199C
:1085C000401E00090001E063D825280001F02BFAC5
:1085D0000700002F02D1042000F06EF801213800BE
:1085E00001F06FFAE819401E0009000114F150066D
:1085F000B0F164017161306117F10F0000090001F1
:10860000B06170696849086001F011FE0500002D35
:1086100002D0280000F050F8012114F5EC7001F0B0
:108620006AFE012114F5A67001F065FE01F0FEFE60
:108630000500002D02D0280000F03EF8D4E9BF016B
:108640000A3051F10001C4E9BF010020019000206F
:10865000009001230022E069C16814F5367001F032
:1086600051FC0600002E02D1042000F025F8300055
:1086700001F025FDD4F8B85117E0287DC00713D5C7
:1086800000200190002000900023AA69E069C168E1
:10869000280001F037FC0600002E02D1042000F073
:1086A0000BF8300001F00BFD203528680028E4D1DC
:1086B0000CF0B6F90020FEBD80B501F0A1FF3748EF
:1086C0000068FEE7354909680881704710B53348EE
:1086D000046843F6F93020824FF4D5706082082098
:1086E0002060012060600220E0810F2060810F2067
:1086F000A081D4F8B801002802D10120FFF7DCFFE7
:108700000120C4F8F8020120C4F81C0101F068FD42
:1087100014F15000E061E18A6183E18A8184D4F838
:10872000A811090441F47F4151F0FF01C160032108
:108730008160002114F5A07001F0EAFF002114F51A
:10874000C07001F0E5FF0021D4F8B801002205E077
:10875000C368994200D2C168521C20300368002BC4
:1087600003D04FF6FF739A42F2D3C4F8181114F5F0
:1087700036700E4A0260E02282600D4A02610D4AA4
:108780004260491CC160002114F5907001F0C0FFE7
:108790000120C4F82C0110BD000000000004FF1FE0
:1087A000FC6D0100006E01009C9BFF1F0300008018
:1087B000E06D0100412B01000746384602F004F845
:1087C000FBE750F8041B61B150F8042BD30744BFFA
:1087D000A9F101039A18002342F8043B091FFAD1BA
:1087E000EFE77047DFF88C180978012921D1C0B272
:1087F000002808D1DFF880181E220A70DFF87C18E4
:108800000A220A7007E0DFF870181F220A70DFF8EA
:108810006C1880220A70C0B200280CD1DFF86409FD
:10882000007810F0BF0050F08000DFF85819087091
:1088300009E0012014E0DFF84C09007850F0C00096
:10884000DFF840190870DFF83C0900780006FAD418
:10885000DFF830090078800601D4002000E01B20FA
:10886000704780B501F0B6FFDFF81408FF210170F2
:10887000DFF81008FF210170DFF80C08FF210170FC
:10888000DFF80409007850F08000DFF8FC18087069
:10889000DFF8F808007850F08000DFF8F018087072
:1088A00001BDC0B2002828D1DFF8E408862101709C
:1088B000DFF8E00880210170DFF8DC081A21017080
:1088C000DFF8D8082D210170DFF8D40800210170ED
:1088D000DFF8D00800210170DFF8CC08002101701A
:1088E000DFF8C8084E210170DFF8C4080078C0B274
:1088F00010F00C000C28F7D1FFE77047C0B2002839
:1089000002D0012826D03EE0DFF8840886210170DD
:10891000DFF8800880210170DFF87C089A2101705F
:10892000DFF878082D210170DFF87C080021017044
:10893000DFF878084E210170DFF874080078C0B2C3
:1089400010F00C000828F7D1DFF864080078400622
:10895000FAD518E0DFF8380806210170DFF834088E
:1089600000210170DFF830089A210170DFF82C082F
:108970002D210170DFF838080078C0B210F00C002B
:108980000828F7D1FFE77047C0B2002802D00128BD
:1089900043D085E0DFF81C08007810F0FE00DFF817
:1089A00014180870DFF8F4072D210170DFF8E007D4
:1089B00086210170DFF8DC0780210170DFF8D8071D
:1089C0009A210170DFF8F007007810F01F00DFF83F
:1089D000E8170870DFF8D00700210170DFF8CC0736
:1089E0000E210170DFF8B80700210170DFF8B4072D
:1089F00000210170DFF8B80700788007FAD5DFF8AA
:108A0000B0070078C006FAD4DFF8A4070078C0B237
:108A100010F00C000828F7D142E0DFF89807007842
:108A200010F0FE00DFF88C170870DFF870072D21BA
:108A30000170DFF85C0706210170DFF8580700219C
:108A40000170DFF854079A210170DFF86C07007895
:108A500010F01F00DFF860170870DFF84C070021E6
:108A60000170DFF8480700210170DFF834070021AA
:108A70000170DFF8300700210170DFF8340700785B
:108A80008007FAD5DFF828070078C006FAD4DFF8A7
:108A900020070078C0B210F00C000828F7D1FFE7DB
:108AA0007047C0B201281AD1DFF8EC0646210170E8
:108AB000DFF8E8062F210170DFF8D40606210170E7
:108AC000DFF8D00600210170DFF8E4060078C00668
:108AD000FAD5DFF8DC060078C007FAD5FFE7704763
:108AE000C0B2002802D001283ED07BE0DFF8A80603
:108AF00046210170DFF8A4062D210170DFF8B806C9
:108B0000007810F01F00DFF8B0160870DFF880065C
:108B100086210170DFF87C0680210170DFF8940661
:108B2000007810F0FE00DFF88C160870DFF8780689
:108B300000210170DFF874060E210170DFF8600675
:108B400000210170DFF85C0600210170DFF860068B
:108B50000078C006FAD5DFF858060078C0B210F0E9
:108B60000C000428F7D13DE0DFF82C064621017007
:108B7000DFF828062D210170DFF83C06007810F0A0
:108B80001F00DFF834160870DFF8040606210170B4
:108B9000DFF8000600210170DFF81806007810F0F9
:108BA000FE00DFF810160870DFF8FC0500210170E8
:108BB000DFF8F80500210170DFF8E40500210170FD
:108BC000DFF8E00500210170DFF8E4050078C00659
:108BD000FAD5DFF8DC050078C0B210F00C000428EC
:108BE000F7D1FFE7704770B504000025E4B2002C10
:108BF00002D0012C02D003E0042501E00125FFE7AB
:108C000000F031F80600EDB2F6B20520DFF8AC1541
:108C100000FB06102E5CF6B2002E06D0022E0ED0FF
:108C200008D3042E15D00FD318E02000C0B2FFF7F0
:108C300057FF13E02000C0B2FFF733FF0EE0200023
:108C4000C0B2FFF7A1FE09E02000C0B2FFF756FE58
:108C500004E02000C0B2FFF724FEFFE7EDB2F6B259
:108C6000B542D0D170BDDFF830050078C0B210F049
:108C7000C000002804D0402804D080280BD013E086
:108C8000042012E0DFF814050078800701D40020EA
:108C90000BE0012009E0DFF814050078400601D45C
:108CA000022002E0032000E00020704710B504001D
:108CB000E4B2032C01D302201CE1E4B2002C04D066
:108CC000022C00F0C0805FD30DE1DFF8A80300782C
:108CD000022841D1DFF8D404007810F0DF00DFF87B
:108CE000CC140870DFF8D804DFF8D8140160DFF87E
:108CF000AC040078C0070AD4DFF88804007810F0CC
:108D0000F30050F00200DFF87C14087019E0DFF87F
:108D10008C04007810F0FE00DFF880140870DFF893
:108D20006404007810F0F30050F00200DFF85414EF
:108D30000870DFF86804007850F00100DFF85C1478
:108D400008700020FFF74FFFDFF86004007850F054
:108D50002000DFF858140870DFF86404DFF86814A6
:108D60000160DFF86804006830F4003050F48030AF
:108D7000DFF858140860DFF85804006850F4002049
:108D8000DFF84C140860AEE0DFF8E8020078022853
:108D900041D1DFF81804007810F0DF00DFF80C1480
:108DA0000870DFF81C04DFF81C140160DFF8EC0326
:108DB0000078C0070AD4DFF8CC03007810F0F30085
:108DC00050F00200DFF8BC13087019E0DFF8CC03A4
:108DD000007810F0FE00DFF8C4130870DFF8A40379
:108DE000007810F0F30050F00200DFF898130870DC
:108DF000DFF8A803007850F00100DFF8A013087036
:108E00000020FFF7F0FEDFF8A403007850F0200008
:108E1000DFF898130870DFF8A803DFF8B8130160D3
:108E2000DFF8A803006830F4003050F48030DFF839
:108E30009C130860DFF89803006850F40020DFF806
:108E4000901308604FE0DFF86403007810F0DF0053
:108E5000DFF858130870DFF86803DFF86813016063
:108E6000DFF838030078C0070AD4DFF81803007869
:108E700010F0F30050F00200DFF80813087019E05A
:108E8000DFF81803007810F0FE00DFF81013087008
:108E9000DFF8F002007810F0F30050F00200DFF885
:108EA000E4120870DFF8F402007850F00100DFF8F7
:108EB000EC1208700120FFF796FEDFF804035FF460
:108EC00040310160DFF80403006850F44030DFF8FF
:108ED000FC120860DFF8F802006830F40020DFF8C8
:108EE000F0120860FFE72000C0B201F076FC614894
:108EF0000470002010BD5F48007870470000B6483D
:108F0000006850F00050B4490860B4480068C005DB
:108F100011D4B248006830F47050B0490860AF48CE
:108F2000006850F48070AD490860AC48006830F4C7
:108F30000070AA490860AA484CF220510180A84854
:108F40004DF628110180A7484FF4E9710180A64829
:108F5000006850F4F050A449086040F2FF300078F7
:108F6000C0B2FF2810D0A14840F2FF31097801704B
:108F70009148007810F0E00040F2FE31097811F0DD
:108F80001F0108438C4908708D488F4901608F4844
:108F9000006830F4003050F480308C4908608C4810
:108FA000006850F400208A4908609148006850F039
:108FB00020008F4908608F4800688F4908408D491C
:108FC00008608E4800688C4908408C4908607948E0
:108FD000007810F0FE007749087070482D2101706C
:108FE0006B48862101706B48802101706A489A2184
:108FF00001707148007810F01F006F4908706A48CE
:109000000021017069480E2101706548002101703E
:10901000644800210170664800788007FBD56448E9
:109020000078C006FBD462480078C0B210F00C0093
:109030000828F8D15D484E2101705D480078C0B223
:1090400010F00C000828F8D1594800784006FBD5EC
:1090500051481A21017056480078C0B210F00C0037
:109060000C28F8D15148007850F020004F49087082
:1090700070470000B49BFF1F0A4006400B400640AB
:1090800005C0074006C0074007C0074010B50022D2
:109090005B49252001F0DCFA04004C48006830F4FC
:1090A0000A6050F04000494908605648006830F0B6
:1090B000807050F4E060534908605348007810F025
:1090C000E000514908705148007810F0F8004F490D
:1090D00008704F48007810F0F6004D4908704D4870
:1090E000007810F0DC0050F050004A4908704A48FF
:1090F000007810F0DC0050F0400047490870474805
:10910000006850F0805045490860454800210170D2
:109110004448002101704448002101704348002167
:1091200001704348007810F0410050F001004049C0
:1091300008701548802101701448802101703D4855
:10914000002101703C48282101703C480021017039
:109150003B48002101703B48002101703A48002142
:1091600001703A48002101703948002101703948E6
:109170000068800880003749086001F02FFB10BDAF
:10918000000000000840064008C0074009C0074032
:109190000050064000500E4000400640014006408E
:1091A000104006401140064004400640054006407D
:1091B000064006400C40064003400640344D010086
:1091C000448004400000771300002501048004401F
:1091D00000700440000099993C80044010D0034086
:1091E0000E20054000200540388004400240064023
:1091F0002880044048900440FFF8FFFE4C90044053
:10920000638800001090044005F0074004F0074018
:1092100002D0074000D0074001D00740348004400E
:1092200000C0074001C0074002C0074003C007401C
:1092300004C007400AC0074000E007402DE400E0FA
:109240002EE400E02CE400E03EE400E014E400E062
:1092500015E400E0108004400FB403980499C9039A
:1092600051EA0040059950EA0120069950EA811020
:10927000089950EA4110099950EA0110079950EAFB
:1092800081000A9908430299019A42F821000C983A
:10929000002805D10120029988400099886004E0E7
:1092A0000120029988400099486000984069012196
:1092B000029A914088430B99029A91400843009981
:1092C000486104B0704710B58AB0DFF8C402006886
:1092D00050F4FC40DFF8B812086000240DE03420A0
:1092E000DFF8B01200FB041184B06846342200F0AD
:1092F0007FF90FBCFFF7B0FF641C622CEFD3DFF8DF
:1093000098021F210160DFF894024FF44071016060
:1093100000200AB010BDDFF88822C0B200280AD0B1
:10932000022853D02DD3042800F0948073D305284D
:1093300000F0B580D8E0DFF86C02CB0705D54FF41C
:10934000107343604FF4107383608B0703D50023C1
:10935000436000238360480707D541F234008058FA
:1093600050F4806041F234039850080707D541F269
:109370003400805830F4806041F23401885000207D
:109380007047DFF82402CB0705D54FF45073C36054
:109390004FF4507303618B0703D50023C360002390
:1093A0000361480707D541F23400805850F400604B
:1093B00041F234039850080707D541F23400805831
:1093C00030F4006041F234018850D8E7DFF8DC0166
:1093D000CB0705D54FF4507383604FF45073C360CF
:1093E0008B0703D5002383600023C360480707D59C
:1093F00041F23400805850F4805041F234039850C8
:10940000080707D541F23400805830F4805041F20B
:1094100034018850B3E7DFF89001CB0705D54FF44E
:10942000507303644FF450734364480707D541F207
:109430003400805850F4005041F23403985008072B
:1094400007D541F23400805830F4005041F2340125
:10945000885094E7DFF85001CB0705D54FF45073DF
:1094600083634FF45073C3638B0703D50023836377
:109470000023C363480707D541F22800805850F401
:10948000806041F228039850080707D541F2280070
:10949000805830F4806041F2280188506FE7DFF88F
:1094A0001001CB0705D54FF4507303624FF450738E
:1094B00043628B0703D500230362002343624807FE
:1094C00007D541F22800805850F4006041F228038B
:1094D0009850080707D541F22800805830F4006002
:1094E00041F2280188504AE75FF0FF3048E780B535
:1094F000DFF8C00001F06FF9012802D15FF0FF3002
:1095000008E0DFF8B400006850F00050DFF8A81061
:109510000860002002BDDFF88810002802D0012872
:1095200012D021E0DFF884004FF4087202624FF499
:109530000872426241F23400405850F0400041F25B
:10954000340250500020704717484FF4087282626E
:109550004FF40872C26241F23400405850F080006B
:1095600041F234025050EDE75FF0FF30EBE70328A3
:1095700002D0042805D009E00B484FF44071816403
:1095800004E00B484FF44071C166FFE700207047CC
:10959000388004406C4E0100C8C00440C0C0044084
:1095A000007004400090044000B0044000C004403B
:1095B00000D0044000D003403C80044010B5044675
:1095C00010460A460146204601F0E6F9204610BD45
:1095D00062B38B0708D0521E11F8013B00F8013B23
:1095E00000F024808B07F6D1830740F0208000BF75
:1095F000103A07D330B4B1E83810103AA0E8381068
:10960000F9D230BC530724BFB1E80810A0E8081015
:1096100044BF51F8043B40F8043BD20724BF31F863
:10962000022B20F8022B44BF0B7803707047083AD6
:1096300007D3B1E80810083A40F8043B40F804CBDF
:10964000F7D25307E4E700002DE9F84304000D00CA
:1096500091461E005FF00008D9F80800DFF890146A
:10966000884204D0382000F0E6FB002020E00C34D3
:10967000102C00D2102414F10F000409240100F072
:10968000BFFFD9F8147001E0B846BF68002F09D0B9
:10969000C9F8187000F0C3FF00F0B2FFD9F81870D5
:1096A000002F07D100F0BBFF042000F0C4FB002016
:1096B000BDE8F283D9F81400874200D1B846386873
:1096C000A042E1D3011B102908D3E0190160C0F8C2
:1096D0000490B9688160B8603C6001E00400B8683B
:1096E000D9F814108F4202D1C9F8140001E0C8F86B
:1096F0000800D9F81400C9F81800D9F81400C9F8FE
:109700001C00D9F81400C9F82000D9F80C00C9F8D9
:109710002400D9F80C00C9F82800E8683881002036
:109720007881C7F80490D9F82C00B84201D2C9F862
:109730002C7000F074FF002E06D0B4F10C02002152
:1097400017F10C00FFF73AFF17F10C00B0E7F8B57E
:1097500004000D0016001F000021B868DFF89023F8
:10976000904204D0382000F066FB00201DE00C344D
:10977000102C00D2102414F10F000409240100F071
:109780003FFF786901E001008068002807D0B861D8
:1097900000F045FF00F034FFB869002806D100F062
:1097A0003EFF042000F047FB0020F2BD79698842AB
:1097B00000D101000268B5F10C0110F110039942CB
:1097C000E1D3111863190C3B9942DCD3B5F10C01BC
:1097D000B1EB000C121BB2EB0C03C0F800C0102B55
:1097E00006D362181360576083689360826001E05B
:1097F0001C1982680C608A607A69BA617A69FA61B8
:109800007A693A62FA687A62FA68BA62F2680A8138
:1098100000224A814F60F96A814200D2F86200F06A
:10982000FEFE0698002805D0B4F10C0200212800A5
:10983000FFF7C4FE2800B8E780B5DFF8B812096862
:109840000023D1F81823C969FFF7FEFE02BD80B5D9
:10985000DFF8A022126800230093D2F81833D269EF
:10986000FFF775FF02BDDFF88C020068D0F818031F
:10987000704780B5DFF87C1209680123D1F81823FE
:10988000C969FFF7E1FE02BD38B50400DFF86402E4
:109890000568501800090001206111F10F0000094E
:1098A0000001E060E0622169091A01600021816025
:1098B00044606061A061E061206200F0A1FED5F823
:1098C0000C03002804D1002115F5437000F020FF9F
:1098D000210015F5437000F021FF00F0A0FEDFF835
:1098E0001002A060200032BD38B50C000F30050911
:1098F0002D01302200212800FFF760FE15F1300015
:10990000B4F1300201002800FFF7BEFF280032BD8D
:1099100070B5DFF8E0110968002804D1012000F0DB
:109920008AFA01207EE0B0F10C046568A868DFF8CF
:10993000C021904204D0382000F07DFA382071E038
:109940002089C969C96889B2884209D020894FF63F
:10995000FF71884204D0032000F06DFA032061E01B
:1099600000F04EFE6E6906E0B668EE6100F057FE4C
:1099700000F046FEEE696869002802D068698442FA
:1099800014D26E6920680019B0420BD1206831688A
:1099900008182060B068A0600C2200213000FFF79A
:1099A0000DFE00E0A6606C61002006E0B068844215
:1099B00002D3B0680028D7D10120002825D0206824
:1099C0000019B16888420DD12068B168096808188B
:1099D0002060B0688068A0600C220021B068FFF7AA
:1099E000EDFD01E0B068A06030688019A0420BD1A5
:1099F0003068216808183060A068B0600C2200212F
:109A00002000FFF7DBFD00E0B4606869A8616869C9
:109A1000E86168692862E8686862E868A86200F03E
:109A2000FEFD002070BD80B5324909680023D1F8E1
:109A300018235031FFF708FE02BD80B52D4802689B
:109A400012F551710800C2F818033031D2F8B02174
:109A5000521AFFF719FF002002BDF8B504000D00EF
:109A600024480668002D03D1D6F81873FD6803E07A
:109A70000C3D6F682868451900F0C2FD786901E067
:109A800029684D1939698D4211D22989E26892B24B
:109A90009142F5D100E08068002801D0A842FAD3B5
:109AA000A842EDD000F0BBFD15F10C0008E03F68C6
:109AB000FD68D6F818038742E0D100F0B0FD002021
:109AC000F2BD002803D00C384181012000E00020C5
:109AD00070470C38C9680181704780B5054909682D
:109AE0000123D1F818235031FFF7AEFD02BD00006D
:109AF00070656D6C0004FF1F70B582B00C00110022
:109B00000025DFF8FC231268002C04D5152000F096
:109B100092F9002018E080B2002816D1D2F8A801EE
:109B2000009300230022200000F09DF90400002C87
:109B300009D0E56800F064FD200000F0C0FA00F0F4
:109B40006EFD0AF071FF280076BD80B2FF2804DDAB
:109B5000132000F070F90020F6E780B2D2F8A821B7
:109B60009042DDD0132000F066F90020ECE780B5CC
:109B7000002380B2FFF7C0FF02BD2DE9F843DFF8F4
:109B800080130C68002808D0010CD4F8A82189B2F1
:109B900092B2914201D01220F6E000F023F90500C4
:109BA000002D03D014F15000854201D11220EBE0CA
:109BB00014F5A67000F0DEFB00F022FDA86809286D
:109BC00007D100F02CFD14F5A67000F09AFB0020E0
:109BD000DAE0A868022807D1E069854228D06868E1
:109BE00029680160486023E0A868C00514D5A8680A
:109BF000C0051DD56868296801604860B4F888010F
:109C0000401EA4F88801A86830F48070A860A86895
:109C100050F00300A8600BE0A868800508D56868CC
:109C2000296801604860A86B0089401EA96B088103
:109C3000A868400508D5286CE96B01604860A86BEE
:109C40000089401EA96B08810920A860A06CA84269
:109C500001D10020A06400F0E2FC00260CE014EB2F
:109C60008600D0F83402002805D0280014EB8601C5
:109C7000D1F834128847761C102EF0D3EF68E669CD
:109C800095F8280080061ED400212800FFF7E5FE85
:109C9000804615E041462800FFF7DFFE8146AE42D0
:109CA00004D014F150014046FFF713FFA84506D039
:109CB000D5F88C00804502D04046FFF729FEC84603
:109CC000B8F1000FE6D15FF00040E860B4F8280179
:109CD000012806D10120C4F82C010020C4F830016D
:109CE0000BE0BFB2D4F82C01874206D2BFB2C4F851
:109CF0002C71286F6C38C4F83001286FE96E016050
:109D00004860B4F82801401EA4F8280114F5A67094
:109D100000F0F7FAB54224D100F072FC68682968B7
:109D200001604860280000F06AFE95F8280080066F
:109D300015D4D5F88C00002809D014F15001D5F8BD
:109D40008C00FFF7C6FED5F88C00FFF7E1FD14F19B
:109D500050012800FFF7BDFE2800FFF7D9FD0AF0EB
:109D600061FE280000F04BFE95F8280080060AD41A
:109D7000D5F88C00002803D0D5F88C00FFF7C8FD7B
:109D80002800FFF7C5FD0020BDE8F28380B5002163
:109D9000FFF7F3FE02BD10B559480068C46900F032
:109DA0002FFCA06A50F48050A06200F038FC10BD77
:109DB00010B553480068C46900F022FCA06A30F472
:109DC0008050A0620AF030FE00F029FC10BD4C4823
:109DD0000068018B002902D0406BC06801E0C069B7
:109DE000C06D704770B5040045480568002C01D16E
:109DF000E8691FE0E86D844202D115F1500019E0D6
:109E000000F0FEFBD5F82001B0F16C06B5F8280192
:109E100002E0F16EB1F16C060100481E002906D087
:109E2000F168A142F5D100F0FAFB300002E000F049
:109E3000F6FB002070BD32490A68118B002902D060
:109E4000516BC96801E0D169C96D002801D00029B2
:109E500007D1138B002B02D0526BD06001E0D26986
:109E6000D065080070472DE9F04383B00F0014005F
:109E70001D0023490E68002811D05FF00008B94684
:109E8000D6F8B87100E020373968002902D0396867
:109E90008142F8D13868002805D1002703E0D7F8BF
:109EA00018905FF00108002F04D11020FFF7C3FFC6
:109EB000002012E016F5A67000F05CFA01950094FF
:109EC00043464A46F069C168380000F01BF80400B8
:109ED00016F5A67000F015FA2000BDE8FE8300001C
:109EE00080B507480068C069D0F88410002902D006
:109EF000D0F8840080470020FFF748FF01BD000034
:109F00000004FF1F2DE9F24F84B0804691461C00EB
:109F1000AD480668D6F81801D8F80C10884208D267
:109F200016F53670804504D00E20FFF784FF002020
:109F3000B8E00E9D002D18D0DDF83CA0BAF5CA7F20
:109F400004D80220FFF777FF0020ABE000232A00AF
:109F500002A9504600F0D0F807000298BAEB000AB8
:109F6000002C1BD0BAF1200A18E0D8F808A0BAF1EA
:109F7000D90F01D25FF0D80A1AF10F005FEA101A68
:109F80005FEA0A1A002C02D01AF1200000E05046C5
:109F90000023002202A900F0AFF80700002F04D12F
:109FA0000A20FFF748FF00207CE00320B860D7F8C4
:109FB0008C00002802D0D7F88CB002E0029810EB99
:109FC000070B002C0ED05C461BF1200B20004146F5
:109FD0002022FFF70DFBA046D8F8000050F000400B
:109FE000C8F800005146584600F05FF8D8F80C0059
:109FF0007FF00F01326A01FB0020F861386281892D
:10A00000B984D8F81410B962002D03D0B96A51F0A0
:10A010002001B962CDF804908089009043465246F1
:10A020005946380000F0ECFC002801D1002039E04E
:10A03000C7F86880D8F800007866D8F81C000028B7
:10A0400009D0D7E92923D8F81C000021101859415C
:10A05000C7E9290107E017F1A40016F53F711CC9F3
:10A060001CC00C390C38D6F8F802022803D1B86AA3
:10A0700050F00400B862D6F89C027867D6F8A002C7
:10A08000B867D6F8A402F86704983866002D08D19E
:10A0900039003800FFF71DFD3900D7F88C00FFF7B5
:10A0A00018FD380005B0BDE8F08F8908491C02E0B2
:10A0B000464A0260001D491E0029F9D1704710B4BC
:10A0C00041490968C26953684C6A944200D24A62A5
:10A0D00002218160436019680160186050600021AE
:10A0E000C0F8B0100021C0F8B4100021C0F8B810BA
:10A0F00010BC70474069704770B506001400BC2062
:10A10000314A1568B5F828214FF6FE739A4201DBF3
:10A11000002058E00860002C05D00200002120003B
:10A12000FFF74CFA1FE0FFF7A4FB0400002C04D05B
:10A130003000FFF781FBC4F88C00002C01D1200017
:10A1400041E0D4F88C00002804D12000FFF7E0FBA8
:10A15000002038E024212000FFF7B3FC2521D4F8AB
:10A160008C00FFF7AEFCD5F82C61D5F83011D5F88E
:10A17000A801B6B256EA0040E060002902D115F508
:10A18000907100E06C3114F16C0215F5907000F0E4
:10A19000FBFA20000100C86EB0F16C021000761CC2
:10A1A000B6B2002E00D1012615F590739A4204D064
:10A1B000D26892B2B6B2B242ECD0C5F83011B6B2A3
:10A1C000C5F82C61200070BD0004FF1F6B61747323
:10A1D000C26D002901D0002A00D1C165100070476E
:10A1E0002C48006810F5D4714A69082A03D3072265
:10A1F00007234B6104E0002A02D1012201234B61B5
:10A20000510111F0E001C182002003E02249C02287
:10A210004254401C6A28F9D32049002004E05FF032
:10A22000FF3241F82020401C0428F8D3704770B555
:10A230001848046800202062D4F81801861C3001F8
:10A24000FFF717FB0500002D01D1042021E00521B7
:10A250002800FFF736FC05E0C020A881206AA8602E
:10A26000256210353000461E00280FD02D606D602D
:10A27000EE81D4F8BC0180190728EDD2D4F8BC01D6
:10A280008019400110F0E000A881E7E7206A6062D1
:10A29000002070BD0004FF1F00E400E080E100E04A
:10A2A00070B504001500DFF83C010668A1610021CB
:10A2B00014F1080000F02CFA00F0A2F9002D13D1DF
:10A2C000D6F8400100E0006816F5A071884206D07B
:10A2D000A042F8D100F0A3F94FF482600AE0210017
:10A2E00016F5A07000F01AFADFF8FC00606100F0CB
:10A2F00096F9002070BD80B500230022FFF7D0FF43
:10A3000002BD38B505003748046868693649884297
:10A3100001D01F202DE000F073F9A869002822D495
:10A32000288A00281FD015F1080000F016FA3C38E2
:10A330008168C90510D5416802680A605160B4F8A7
:10A340008811491EA4F88811816831F480718160F8
:10A35000816851F00301816000218163FFF7AFFE46
:10A360000AF062FB02E0A869401CA86100F057F9FE
:10A37000002032BD38B504001A480568288B002833
:10A3800001D00D202CE060691749884201D01F20C0
:10A3900026E000F035F9A069012813DAE86940F2F7
:10A3A0002B41816014F108018163416802680A60F1
:10A3B000516010F13C0114F1080000F0AFF90AF00F
:10A3C00041FB02E0A069401EA06160690649884225
:10A3D00003D000F024F91F2002E000F020F9002053
:10A3E00032BD00000004FF1F6D73776CB0FBF1F00D
:10A3F000401E62490860704780B500F052FB0021A2
:10A40000C0B200F052FBC821FFF7F0FF5C48072103
:10A4100001605C48006850F080505A4908605A4812
:10A42000006850F080405849086001BD10B542F204
:10A430006300FEF747F95FF000510020FFF707FACD
:10A44000FA21002000F037FB002878D14F4800F0B7
:10A450003DFB0F2000F0D9FD00220FF2E5010F2097
:10A4600000F0F6F8002801D1262068E04848494964
:10A4700088420AD247484649474A5118884204D27E
:10A48000FFF7F1F94549086009E0414842490818D9
:10A490004349411A4248FFF727FA4049086000F053
:10A4A00085FEFFF7A9FF012000F038FE002801D04B
:10A4B000262044E000F062FE002801D026203EE085
:10A4C000002000F02BFE002801D0262037E0354880
:10A4D00004683548C4F89801C82000F091FDD4F80C
:10A4E000980100F09EFD00210FF25D0000F092FD4A
:10A4F00000F060FE00F068FE002820D1FEF7F7FFB4
:10A50000002805D1042000F07AFE012000F0F6FFBB
:10A5100026482749016027482549016001F012F8C3
:10A5200001F018F8244802682349244801F058F83B
:10A530002349244801F02EFB01F05EFF002010BDEE
:10A5400080B500F070FC01BD00220C4800680002DC
:10A55000000A401C1C4909680902090A1B4B1B68B8
:10A560005B0104D5184909680902090A020000299B
:10A5700000D10100401A10187047000014E000E0FC
:10A5800010E000E01CED00E020ED00E00000FF1F07
:10A590000000FF1FC09BFF1F00000200F897FF1F75
:10A5A0000000FF1F0004FF1FC0270900202808E04B
:10A5B00000A00FAA202008E0686201005C4E0100A4
:10A5C00054620100644E010018E000E004ED00E078
:10A5D00038B504004B480068C56900F011F8A86858
:10A5E0000B280AD00B20A860AC6341212800FFF79C
:10A5F000EFFD686829680160486000F010F831BD1F
:10A6000040480068C169496D002902D1C18A81F3BF
:10A610001188C169496D491CC06941657047394855
:10A620000068C169496D002911D0C169496D491E91
:10A63000C269516500290AD1018B002904D0406B01
:10A64000806880F3118802E0408B80F311887047A6
:10A65000F8B50C0015002B4909688A6B002A04D153
:10A660001820FFF7E8FB002018E0CA6A904202D3E6
:10A670000A6B824204D21420FFF7DDFB00200DE0BC
:10A68000CA6A801A0C22896B02FB0016FFF7B8FF1A
:10A6900037683460B560FFF7C2FF3800F2BD2DE9BE
:10A6A000F04104000D00A54201D20C2026E015481F
:10A6B00006681548C6F80C011448B062281B10F152
:10A6C00001080C2000FB08F0FFF707FA0700002F35
:10A6D00001D1042012E003213800FFF7F2F9B7633B
:10A6E000F462356304E009483860BC60641C0C37D0
:10A6F0004046B0F101080028F5D10020BDE8F08106
:10A70000000000000004FF1F934B0100D1A50000D2
:10A7100000604060002202814181704738B504002A
:10A720000D00FFF76DFF6089002807D0208961893F
:10A73000884203D3FFF773FF00200DE060680068D4
:10A74000286061680D606168696045602089401C0F
:10A750002081FFF764FF012032BD38B50400FFF708
:10A760004FFF2089002803D1FFF759FF00200AE09E
:10A77000256868682968016048602089401E20813A
:10A78000FFF74DFF280032BD70B504000D00160024
:10A79000002D00D12500FFF733FF6089002807D086
:10A7A00020896189884203D3FFF739FF00200AE03E
:10A7B000286830602E60756046602089401C2081CA
:10A7C000FFF72DFF012070BD01491820ABBEFBE74C
:10A7D0002600020070470020704770474548006817
:10A7E00050F48060434908604348007810F0F3005B
:10A7F00041490870414841210170414800210170E0
:10A800004048002101704048002101703F48032169
:10A8100001703F48002101703E48C02101703E4850
:10A82000002101703D48002101703D482021017048
:10A830003C48202101703C48032101703B48C02165
:10A8400001703B48007850F0880039490870394859
:10A850000021017038480121017038480A21017037
:10A860003748002101703748F72101703648002130
:10A8700001703648002101703548002101703548CB
:10A88000002101703448002101703448002101701A
:10A890003348002101703348002101703248002103
:10A8A00001703248002101703148002101703148A7
:10A8B000002101703048007810F00F002E49087018
:10A8C0002E48DF2101702E480F2101702D4800789D
:10A8D00010F080002B4908702B4800782B4909782C
:10A8E0002B4A002313702B4A00231370024A0C23B7
:10A8F000137070473480044003A0064001A0064056
:10A9000000A0064008A0064009A006400AA0064094
:10A9100002A0064005A006400DA006400EA006407D
:10A9200013A0064015A0064012A0064011A0064044
:10A9300010A006401CA006401DA006401BA006401B
:10A940001EA006401AA0064019A0064018A0064006
:10A9500022A0064023A0064024A0064025A00640D1
:10A9600026A0064027A006402AA006402FA00640A9
:10A9700030A0064031A0064021A006402BA0064092
:10A980002CA0064029A0064004A0064007A00640CF
:10A990000BA0064006A0064062F30F2262F31F429E
:10A9A000401810F0030308D0C91A1FD3DB0748BFB3
:10A9B00000F8012D28BF20F8022D130030B41446F2
:10A9C0001546103928BF20E93C00FAD8490728BFAE
:10A9D00020E90C0048BF40F8042D890028BF20F86A
:10A9E000022D48BF00F8012D30BC7047C91818BFB0
:10A9F00000F8012DCB0728BF00F8012D70477047E4
:10AA0000F8B504001D0001265018401E0009000181
:10AA1000B0F16407206111F10F0000090001A0618D
:10AA20006761642200213800FEF7C8FD0E483864D3
:10AA30000798F862696851F0010179645FF08071EC
:10AA4000B964B86500203860069878607FF002002D
:10AA5000B86294F82800800703D5200000F006F8BB
:10AA600006003000F2BD0000E19E000038B5040091
:10AA70009420FEF7FEFE0500002D05D104212000E4
:10AA8000FFF7A6FB00200BE022212800FFF719F8B2
:10AA900021002800FFF71DF8E068286165630120A8
:10AAA00032BD80B500F052FB02BD80B5C9B2C0B264
:10AAB00000F050FB02BD10B5FFF7F1FD0400002CC3
:10AAC00001D101F0B3FC200010BD0000024909686B
:10AAD000014A10600800704708ED00E038B5DFF863
:10AAE00020160C68002813D0E56915F1440101F027
:10AAF000B3FCFFF785FD15F1440214F5B47115F1AF
:10AB0000440001F0E9FC280000F01EF8FFF787FD83
:10AB100031BD70B50400DFF8E8050568002C03D1ED
:10AB20000C20FFF788F90EE0EE69FFF769FD16F1DA
:10AB3000440215F5B471200001F0CEFC300000F0A5
:10AB400003F8FFF76CFD70BDF8B50400DFF8B00541
:10AB5000006810F5C071B0F88821002A27D0D0F81D
:10AB60008051B0F8882112F1010C01E029002D6814
:10AB7000BCF1010CBCF1000F19D0D4E91167D5E983
:10AB800011239F4204D801D3964201D201220CE046
:10AB9000D5E91167D4E911239F4205D801D3964224
:10ABA00002D25FF0FF3200E00022002ADED46268A9
:10ABB000236813605A60220010F5C070FFF7E4FDAF
:10ABC000A06850F48070A06009F03CFFF1BD70B542
:10ABD0000400DFF82C050668002C0FD0F569FFF79C
:10ABE0000FFDD6E95A232000002110185941C5E96C
:10ABF00011012800FFF7A8FFFFF711FD70BD38B560
:10AC0000DFF8FC140968002803D10C20FFF713F9C2
:10AC10000DE0CC6914F144012CC82CC10C380C395E
:10AC2000FFF7EEFC2000FFF78FFFFFF7F8FC31BDC8
:10AC300070B504000D00002C01D0002D01D10020C2
:10AC4000C0E0A089B0F57A7F0FDB6089A1894FF45D
:10AC50007A7291FBF2F108186081A0894FF47A7141
:10AC600090FBF1F201FB1200A08160893C280DDB12
:10AC7000208961893C2291FBF2F1081820816089CA
:10AC80003C2190FBF1F201FB1200608120893C28FD
:10AC90000DDBE08821893C2291FBF2F10818E0806D
:10ACA00020893C2190FBF1F201FB12002081E08819
:10ACB00018280DDBA088E188182291FBF2F1081812
:10ACC000A080E088182190FBF1F201FB1200E080E7
:10ACD000A088002801D1002074E060880D280DDBD9
:10ACE000208861880C2291FBF2F10818208060888E
:10ACF0000C2190FBF1F201FB12006080208840F2F1
:10AD0000B271884221DA40F2B27020801DE0A18841
:10AD100062880D23DFF8EC6303FB0060105C081A07
:10AD2000A0806088401C608060880D280DDB208832
:10AD300061880C2291FBF2F10818208060880C21B8
:10AD400090FBF1F201FB12006080208800F037F9DF
:10AD500061880D22DFF8AC3302FB0032895CA288E7
:10AD600089B29142D3D32188B1F50C6F01DB002069
:10AD700028E0DFF894132288DFF8903313EB820287
:10AD8000895862883423DFF8886303FB006010EB86
:10AD9000820050F8040C4118A088401EDFF874238C
:10ADA00002FB0011E0884FF4616202FB0011208970
:10ADB0003C2202FB0011608911FA80F12960A08910
:10ADC0006860012070BD10B584B0040000A800F0D8
:10ADD00005F8210000A801F0A3FB1FBD38B5040051
:10ADE000002C1FD0DFF818030568FFF709FC15F5E4
:10ADF000B4700EC80EC40C380C3CD5F8A001002865
:10AE000005D0D5F8A401D5F8A0118847A06022008C
:10AE100015F5BA71200001F05FFBFFF700FC200080
:10AE200001F0CCFB31BD2DE9F843DFF8D402046812
:10AE3000D4E95A01401C51F10001C4E95A01FFF75D
:10AE4000DFFBD4F8A001002806D0D4F8A401D4F880
:10AE5000A0118847C4F8700114F5B47001F0AEFB7E
:10AE6000B4F88851002D41D0D4F880016D1C1FE04A
:10AE7000B4F88811491EA4F88811416802680A6074
:10AE80005160816831F480718160816849050CD519
:10AE9000816831F480618160016CC26B0A6051602D
:10AEA000816B0989491E826B1181FFF708F9300017
:10AEB0006D1E002D1AD00668D0E91123D4E95A89F5
:10AEC0004B4504D801D3424501D201210CE0D4E91D
:10AED0005A23D0E911894B4505D801D3424502D206
:10AEE0005FF0FF3100E000210029C1D5E06990F852
:10AEF0002810490729D5D0E92C23521C53F100030F
:10AF0000C0E92C23816AC9041FD4D0E92923D0E9E0
:10AF10002C67BB4204D801D3B24201D201210CE01C
:10AF2000D0E92C23D0E92967BB4205D801D3B2422E
:10AF300002D25FF0FF3100E00021002905D4416812
:10AF400002680A605160FFF7BAF8FFF768FBD4F8AF
:10AF50000803002802D0D4F808038047D4F840033F
:10AF6000002802D0D4F840038047BDE8F18310B533
:10AF700084B0DFF88C110C684168B1F57A7F0FD38B
:10AF8000016842684FF47A73B2FBF3F25118016022
:10AF900041684FF47A72B1FBF2F302FB1311416086
:10AFA00000A901F025FBFFF72BFB14F5BA7214F58D
:10AFB000B47100A801F030FBFFF731FB1FBD80B278
:10AFC000642190FBF1F201FB120100290CD180B247
:10AFD0004FF4C87190FBF1F201FB1200002801D17F
:10AFE00001200CE000200AE080B2042190FBF1F285
:10AFF00002FB1102002A01D1012000E0002070476D
:10B000003F490968C1F8940170473D490968C1F892
:10B010008C0170473A4A1268C2F8A001C2F8A41124
:10B02000704737490968C1F89C01704770B5040042
:10B030000D00002C01D0002D01D100205EE0206821
:10B040003549884203D26068B0F57A7F01D3002089
:10B0500054E00020288002E02888401C28802068D6
:10B0600029882A4A12EB810149688842F4D2206873
:10B070002988264A52F82110461A288800F2B27010
:10B0800028802888FFF79BFF0121698002E06988FA
:10B09000491C6980698834221D4B02FB003252F83A
:10B0A00021108E42F3D269883422194B02FB003002
:10B0B00010EB810050F8040C361A1648B6FBF0F07D
:10B0C000A880A888134901FB1066A888401CA880A6
:10B0D0004FF46160B6FBF0F0E880E8884FF46161FE
:10B0E00001FB10663C20B6FBF0F0288128893C214A
:10B0F00001FB10666E816068A881012070BD0000B0
:10B100000004FF1FBCAE010038E1FFFF40AF0100AB
:10B11000D8AE010080510100015786F438B5040013
:10B1200000252000C0B2FDF7C1FD0500ADB2002D25
:10B1300002D0280080B208E000212000C0B2FFF752
:10B14000B4FCC821FFF752F9002032BD80B5FDF7ED
:10B15000D2FE02BDC0B203280BD2C9B21E2908D24A
:10B16000C9B2C0B22822044B02FB003050F82100C3
:10B1700000E00020704700003C6E010010B5002484
:10B180000020FDF72FFB0400A4B2002C02D0200009
:10B1900080B20AE00120FDF725FB0400A4B2002CD8
:10B1A00002D0200080B200E0002010BD80B5FDF785
:10B1B0006DFF01BD03480068400840000149086078
:10B1C0000020704700D0004010B5064804680021F8
:10B1D00014F52470FFF79CFA012114F51D70FFF798
:10B1E0008AF810BD0004FF1F4FF47A71484378219C
:10B1F000484301E000BF401E0028FBD1704770B5F6
:10B2000004000025DFF8B462E00720D5FFF7F8F965
:10B21000306950F001003061DFF8A40200210160C4
:10B22000DFF8A00200210160DFF89C02002101602C
:10B23000DFF8980200210160306940084000306169
:10B240005FF0FF30B06001203060FFF7E8F9A00741
:10B2500015D5FFF7D5F9306950F00100306130693C
:10B2600040084000306101203060DFF85C020021BE
:10B270000160DFF8580200210160FFF7D0F9600794
:10B2800029D53069C00703D53069400840003061D6
:10B2900032000FF249015220FFF7DAF9002802D1FB
:10B2A000FEF795FD0500002D15D17069C00602D589
:10B2B0003069C0050AD4306950F4807030617D2057
:10B2C000FFF792FF706950F01000706101220421B5
:10B2D000522001F0C1F9280070BD000038B5DFF838
:10B2E000DC410120616911F0030F1CD0626932F06A
:10B2F000100262615FF0FF32A26001222260626987
:10B3000052F010026261CA0701D5082200E0002253
:10B310008B0701D5042300E000236C4D2D681A43F0
:10B320002A436A4B1A6049072AD5A5686449096807
:10B330008D420CD16548006850F0010063490860F7
:10B34000614800684008400000F093F800205D4923
:10B3500009688D420CD15D48006850F002005B49DD
:10B3600008605948006830F0020000F082F80020C0
:10B37000012805D1544800688008800000F079F861
:10B3800053480068002809D0504800684E490968B1
:10B39000084203D020004E490968884731BD00218A
:10B3A00080B2042290FBF2F303FB1203002B13D1B3
:10B3B000012180B2642290FBF2F302FB1302002A07
:10B3C00000D1002180B24FF4C87290FBF2F302FB6F
:10B3D0001300002800D101210800704770B5040057
:10B3E00000252088A0F2B27040F26D11484305009C
:10B3F00040F2B27605E0300080B2FFF7D0FF451989
:10B40000761C20888642F6D301260DE0314810EBE9
:10B41000460030F8020C15FA80F5022E03D1208880
:10B42000FFF7BDFF4519761C60888642EED3A088E1
:10B43000401E45192848E1884FF46162514300FBE2
:10B44000051021893C2202FB0100618910FA81F07C
:10B4500070BD1A494A6932F010024A6100680860FA
:10B46000486950F01000486170471449096801604C
:10B470007047124910F00302002A03D15FF0FF3039
:10B48000886019E0032A0FD10A680E480068801A04
:10B490000B4B1B689A1A904202D30948006801E0DE
:10B4A00008480068886007E0C00702D504480068C3
:10B4B00001E00448006888607047000000D0034045
:10B4C000FC97FF1F0098FF1F0498FF1F0898FF1F9D
:10B4D0000C98FF1FB06201008051010000B583B0DD
:10B4E000006800900020019000A8FFF79FFD07BDB5
:10B4F00010B50C00FFF772FF206010BD00B587B0DB
:10B5000001280ED100A8FFF7B0FF03A900A8FFF79C
:10B51000E5FF01A903A8FFF78BFB01A8FFF727FDB3
:10B520000DE001A8FFF74FFC03A901A8FFF77EFD7E
:10B5300000A903A8FFF7DCFF00A8FFF78AFF00209F
:10B5400007B000BD074808490160064800680028A8
:10B55000FBD470470548044901600448006800288E
:10B56000FBD47047002808E003000085002008E0B5
:10B5700010B400230024002917D0002A15D013018D
:10B58000B1FBF3F3002B0BD01C0104FB1211540888
:10B5900014EB4101B1FBF2F4202C01D35B1C00241D
:10B5A000B3F5005F01D316200EE0190A11F01F0158
:10B5B00001704370817A11F0E0018172817A14F098
:10B5C0001F0211438172002010BC7047C17851F0F6
:10B5D0000C01C1707047C17811F0F301C170704760
:10B5E00070B586B004000D0016006868C0B201F0A6
:10B5F00087F8FFF7F0F8002802D05FF0FF3013E083
:10B60000049603950FF2C91002900FF26D1001908D
:10B610000FF2511000900FF239130FF205120FF2D2
:10B620000D01200001F092F806B070BD2DE9F04147
:10B6300006000F0075682800C0B201F061F8040030
:10B64000002C01D12B2068E05820FEF746FA8046F6
:10B65000B8F1000F01D104205FE0C7F80080C8F8FE
:10B660002040404631002022FDF7C2FF0120C8F8EB
:10B670003000D8F8087015263100C9B22800C0B2D1
:10B68000FDF749FE04212800C0B2FDF744FED8F8BA
:10B690000C2039002000FFF76BFF0020A070E0783D
:10B6A00010F0FD00E070A07A10F03F00A0720020C2
:10B6B0002072002060720020A071207CC0F3021074
:10B6C000C0B2002802D10020E07407E00120217CF4
:10B6D000C1F30211491C8840401EE07401206075CE
:10B6E000E07810F0F300E070207C50F088002074C7
:10B6F000607C50F0C0006074F00603D52000FFF7B6
:10B7000065FF02E02000FFF766FF300704D508213F
:10B710002800C0B2FDF7FFFD0020BDE8F081000069
:10B7200070B504000D00042604216068C0B2FDF766
:10B73000F2FD286A0021C170300704D50821606835
:10B74000C0B2FDF7E8FD2800FEF7E2F8002070BD6A
:10B75000016A0A799206FCD5826B521C8263C87911
:10B7600070470000026A13791B06FCD5D171C16BCA
:10B77000491CC16370470000016A0A79130702D5AA
:10B78000C36C5B1CC364D30702D5436C5B1C43646E
:10B79000530702D5436D5B1C4365930702D5836C49
:10B7A0005B1C83640A2002420BD0C8798A7CD207D2
:10B7B00007D5487C50F040004874887C50F0010068
:10B7C0008874887C400601D4012000E00020704786
:10B7D00070B506001400356AC91E00F0628140F69B
:10B7E000FF40091A00F02981491E6CD0491E6DD016
:10B7F000491E76D0491E00F08D80891F2CD0491E2D
:10B8000018D0491E00F05E81491E00F05181491E8A
:10B8100000F0AB80491E00F09C80091F00F08B8077
:10B82000491E00F08F80491E00F02781491E00F05C
:10B83000318181E10820A978C9060AD596F830102F
:10B84000C90706D5A978890702D5A97A890600D53E
:10B85000401C2060002070BD2068082804D02068AB
:10B86000092801D00C20F6E72068082814D196F8A2
:10B870003000C0070AD5A87A10F0DF00A872A878B7
:10B88000800704D5A87850F01000A870E2E7A878E7
:10B8900010F0EF00A870F9E796F83000C00710D557
:10B8A000A87850F01000A870A878800704D5A87A6E
:10B8B00050F02000A872E9E7A87A10F0DF00A87223
:10B8C000E4E71620C7E7F0682060C3E7B0682268A5
:10B8D00001002800FFF74CFE0028BCD12068F06072
:10B8E000B8E7706B2060241DB06B2060241DF06BE6
:10B8F0002060241D306C2060241D706C2060241D8D
:10B90000B06C2060241DF06C2060241D306D206020
:10B91000241D9FE7002070630020B0630020F063C7
:10B9200000203064002070640020B0640020F064C7
:10B93000002030658EE72879C0F3C01010F00100B8
:10B94000206087E72879C0F3401010F001002060E4
:10B9500080E70120A978890705D5A878C00701D517
:10B96000022000E00320206074E72068012804D052
:10B9700061D3032838D014D35DE0A87880070FD5B1
:10B98000A87810F0FC00A870A87A800604D5A87AE0
:10B9900010F0DF00A87203E0A87810F0EF00A870A4
:10B9A00058E796F83000C00701D4162053E7A8786E
:10B9B000800704D5A87850F00100A87013E0A8789B
:10B9C00050F00300A870A878C00604D5A87A50F0FB
:10B9D0002000A87207E0A87A10F0DF00A872A8780B
:10B9E00050F01000A870DBE796F83000C00701D4D3
:10B9F000162030E7A878800704D5A87810F0FE005C
:10BA0000A87017E0A87850F00200A870A87810F08D
:10BA1000FE00A870A878C00604D5A87A50F02000CF
:10BA2000A87207E0A87A10F0DF00A872A87850F09A
:10BA30001000A870B4E70C200DE7207880060BD525
:10BA40007068FDF794FD687B10F0F6006873687B02
:10BA500050F0020068730FE02078000708D5687B7B
:10BA600010F0FD006873687B50F00900687303E014
:10BA7000687B10F0F4006873ECE62068012804D1BC
:10BA8000E87810F0FB00E87003E0E87850F004007C
:10BA9000E870DFE62879002801D1012000E00020CD
:10BAA000D8E6A87C0006FCD528794006FCD5D1E66E
:10BAB00096F83000C00702D50120206001E0032085
:10BAC0002060C7E62068012814D196F83000C0072E
:10BAD0000FD4A87A10F0DF00A872A87810F0EF0059
:10BAE000A870A87910F0BF00A871306B50F0010069
:10BAF0003063AFE6206803281CD196F83000C007F9
:10BB0000F7D5A878C00602D4A878800701D51620FA
:10BB1000A1E6A87A10F0DF00A872A87850F0100013
:10BB2000A870A87950F04000A871306B4008400020
:10BB30003063DEE70C208EE640F609208BE600003D
:10BB4000F0B4002600225FF0FF35002317E0DFF895
:10BB5000907457F82370DFF88CC45CF824C00CFB99
:10BB600007F74F433F1A002F00D57F42AF4202D262
:10BB70003D001E002200641C402CE8D35B1C032BFC
:10BB800001D20024F8E7B001C0B212F03F0108432F
:10BB9000F0BC70473EB504000D00287801F06AF84B
:10BBA000FEF719FE002802D04FF420600FE0029546
:10BBB0000FF2191001900FF2BD4000900FF22D43CB
:10BBC0000FF2D1020FF20901200001F063F83EBD2F
:10BBD000F8B504000F00207801F04CF80500002DA6
:10BBE00002D14AF6021054E05C20FDF776FF060011
:10BBF000002E01D104204CE040F20B413000FDF753
:10BC000060FF2078FDF787FC3E60300021001422A1
:10BC1000FDF7EEFC75610020B0610020F0610020AE
:10BC20003062607886F82400002086F82500002025
:10BC300086F82600002086F827000020B062002049
:10BC4000F06200203063002070630020B0630020A9
:10BC5000F06300203064002070640020B064002095
:10BC6000F06400203065002070650020B065002081
:10BC7000A8700020E870A078400028706168DFF8A4
:10BC80006803FFF75DFF6870A87850F08000A87027
:10BC90000020F2BD10B50400002901D0002C02D113
:10BCA0004AF6031010E04869C178890602D54AF6C1
:10BCB000011009E000218170FF21C170A069FDF72A
:10BCC00027FE0020A061002010BD000070B588B0E4
:10BCD0000300160000245D69C91E36D040F2FE3014
:10BCE000091A00F0F880491E00F00681491E00F094
:10BCF000D380491E00F0DB80491E00F0E380491E1E
:10BD000000F02381491E00F02981491E00F00B81BB
:10BD1000491E00F01181491E00F0AC80491E4BD035
:10BD2000491E66D0491E00F02281491E00F028817C
:10BD3000491E00F03681491E00F0A480491E00F023
:10BD4000A680491E00F03A8146E100208DF80000EF
:10BD500004E09DF80000401C8DF800009DF80000F4
:10BD6000FF28F6D1E8788DF80000A878C00609D53C
:10BD70009DF8000010F0A0002028E6D0D86B196CC8
:10BD80008842E2D1186CD86393F8270080070BD55E
:10BD90009DF80000800607D4002083F827000020CB
:10BDA0009862072083F82500002E04D09DF800003B
:10BDB00010F0010030600FE14AF60114A878800607
:10BDC00016D593F82500022803D1D86B196C884248
:10BDD0000AD093F82500032802D1986A002803D0DE
:10BDE00093F82500072803D1012083F825000024BB
:10BDF000F2E0A87810F0E700A870E87850F01200A0
:10BE0000E87000209862002083F82700002083F863
:10BE10002500186B5863A878800603D428798DF81C
:10BE2000000003E0A87810F0DF00A87000208DF873
:10BE3000000004E09DF80000401C8DF800009DF813
:10BE40000000FF28F6D1E8788DF800000DE09DF89D
:10BE50000000800706D5E87850F00200E8702879E5
:10BE60008DF80000E8788DF800009DF8000080064D
:10BE7000EDD4B1E0002E02D14AF6031401E030689F
:10BE80009862A9E0A87810F07F00A870A4E0A878D4
:10BE900050F08000A8709FE093F82500002802D0A1
:10BEA0004AF6011402E0002083F8240094E093F89D
:10BEB0002500002802D04AF6011402E0012083F890
:10BEC000240089E0002E02D14AF6031402E093F820
:10BED0002400306080E0002E02D14AF603140AE00C
:10BEE000E878800602D54AF6011404E031683E483D
:10BEF000FFF726FE68706FE0002E02D14AF60314A9
:10BF000010E068788009364951F82010687810F000
:10BF10003F00344A52F82000334A00FB01F0B2FBE4
:10BF2000F0F0306058E0002E02D14AF6031402E02F
:10BF3000306883F826004FE0002E02D14AF6031441
:10BF400002E093F82600306046E0002E02D14AF667
:10BF5000031402E03068400028703DE0002E02D15A
:10BF60004AF6031402E028784008306034E0002EDE
:10BF700002D14AF6031402E093F8250030602BE06A
:10BF8000002E02D14AF603140AE001A813F144017D
:10BF90001822FDF72DFB300001A91822FDF728FB20
:10BFA0001AE000205864002098640020D864002023
:10BFB000186500205865002098650DE0002E02D11C
:10BFC0004AF6031407E0E878800602D501203060C5
:10BFD00001E000203060FFE7200008B070BD0000E5
:10BFE000504D01005C4D01000087930338B5846912
:10BFF000606994F8273053F0010384F8273094F8EF
:10C000002530DBB2002B02D0DBB2012B2CD1032573
:10C0100084F8255094F82450002D25D1857855F0CA
:10C0200010058570C57855F00205C570DBB2012B8F
:10C0300004D1837853F00403837003E0837853F0D2
:10C040002003837094F8273053F0020384F82730DC
:10C0500094F826305B0053F001030371E36C5B1C22
:10C06000E364C3789B07FCD513000A00210000F0AD
:10C0700043F832BD38B58469606994F8273013F00D
:10C08000FE0384F8273094F82530DBB2002B02D071
:10C09000DBB2012B2AD1022584F8255094F82450D4
:10C0A000002D23D1857855F010058570C57855F0A1
:10C0B0000205C570DBB2012B04D1837853F0040371
:10C0C000837003E0837853F02003837094F8273063
:10C0D00053F0020384F8273094F826305B00037194
:10C0E000E36C5B1CE364C3789B07FCD513000A0078
:10C0F000210000F001F832BD78B40400002001E016
:10C100000300401C8342C0F07481E578A678B6062F
:10C1100011D4984200F06E8191F82760B6070AD5D5
:10C12000AE0608D4002281F8272000228A62072266
:10C1300081F825205EE1AE07E7D591F8276056F03B
:10C14000020681F82760A678B60640F19480A678AA
:10C15000F60651D5ED070BD5E37853F00203E370F3
:10C16000072381F825308B6D5B1C8B650300C8E7C6
:10C1700091F82550022D12D191F82750ED070CD4DB
:10C180009842BED2E57855F00205E5701578257124
:10C19000521CCD6C6D1CCD64B3E70300B1E791F880
:10C1A0002550032D26D191F82750ED0720D5A578ED
:10C1B00015F0EF05A5708D6A012D04D1A57855F015
:10C1C0000805A57003E0A57815F0F705A570E578DA
:10C1D00055F00205E5708D6A002D04D1072381F822
:10C1E000253003008DE725798DF80050401E88E743
:10C1F000030086E7030084E791F82550032D38D12A
:10C2000091F82750ED0732D58D6A002D2FD0984236
:10C21000BFF477AFE57855F00205E5708D6A6D1EC5
:10C220008D628D6A012D04D1A57855F00805A570A1
:10C2300003E0A57815F0F705A5708D6A002D03D1F0
:10C24000A57855F01005A57025791570521C8D6ADA
:10C25000002D08D1A37813F0EF03A370072381F812
:10C260002530431C18008D6C6D1C8D6449E703005C
:10C2700047E7030045E7EE060AD5E37853F01003DD
:10C28000E370062381F825300B6D5B1C0B65030002
:10C290006E064AD591F82460002E02D14E6D761CB0
:10C2A0004E656D071AD5052581F8255091F8275060
:10C2B000ED0711D49842BFF424AFA57855F01005CE
:10C2C000A570E57855F00205E57015782571521CCA
:10C2D000CD6C6D1CCD6414E7030012E7042581F8D2
:10C2E000255091F82750ED071DD500281BD18D6AE8
:10C2F000002D18D0A57815F0EF05A570E57855F05C
:10C300000205E5708D6A012D04D1A57855F0080568
:10C31000A57003E0A57815F0F705A57025798DF8CF
:10C320000050401EEDE60300EBE6EE063FF5E8AEFA
:10C33000A678F60629D5ED070BD5E37853F002036E
:10C34000E370072381F825308B6D5B1C8B65030040
:10C35000D7E691F82550022D03D091F82550052DF0
:10C3600011D191F82750ED070DD49842BFF4C9AE12
:10C37000E57855F00205E57015782571521CCD6CF5
:10C380006D1CCD64BDE60300BBE691F82550032D7E
:10C3900003D091F82550042D29D191F82750ED07AD
:10C3A00025D58D6A002D22D09842BFF4AAAEE5783B
:10C3B00055F00205E5708D6A6D1E8D628D6A012D46
:10C3C00004D1A57855F00805A57003E0A57815F00F
:10C3D000F705A5708D6A002D02D1072581F825503B
:10C3E00025791570521C8D6C6D1C8D6489E60300D7
:10C3F00087E6180072BC704710B50B480468D4F883
:10C40000C80100280FD0D4F8CC11D4F8C80100F02E
:10C41000F5FCC4F89C02D4F89C02C4F8A002D4F83D
:10C420009C02C4F8A40210BD0004FF1F0748006866
:10C43000C06B80F308880649102003E0054A41F8E4
:10C440002020401CFF28F9D9704700BF0004FF1FBF
:10C450000000FF1F934B010010B50C000021A160EC
:10C460001A490968012907D119490968B0FBF1F097
:10C470000021C4E9000110BD16490968134A126879
:10C48000022A0BD1D1F89411A1FB00014FF47A726A
:10C49000002300F025FDC4E90001ECE74FF47A72B7
:10C4A000D1F89431B2FBF3F2094B1A60084A1268D2
:10C4B000D1F894315A43B2F57A7F03D1034901226E
:10C4C0000A60D1E7014A02231360DBE7A49BFF1F48
:10C4D000A09BFF1F0004FF1FF0B4D0E90045D1E985
:10C4E0000067A4197D41C2E90045806889680B4B4B
:10C4F0001B68D3F89C315C1AA0420AD3D2E90045EC
:10C50000641C55F10005C2E900450818C01A906086
:10C5100001E008189060F0BC704700BF0004FF1FE6
:10C520002DE9F04307000D0023480668D6F8944132
:10C53000D7E900012200002300F0D2FC01290AD330
:10C5400001D8002807D35FF0FF30286040F2E730C1
:10C55000686000202EE0D7E900234FF47A700021B4
:10C56000A0FB028900FB039901FB0299B8684FF414
:10C570007A714843D6F89C11B0FBF1F0002118EB1A
:10C58000000659EB0107300039002200002300F0BB
:10C59000A7FC06000F00300039004FF47A72002328
:10C5A00000F09EFC286028684FF47A7101FB10604F
:10C5B00068600120BDE8F0830004FF1F30B40B4920
:10C5C0000968D1F89C1182688A420DD38268B2FB57
:10C5D000F1F2D0E900450023A4185D41C0E900450F
:10C5E000836801FB1231816030BC70470004FF1F7B
:10C5F00030B589B004000D0004A9206800F0E8FC03
:10C6000000A9606800F0F2FC2A0000A904A8FFF766
:10C6100063FF09B030BD0000F0B4D0E90045D1E9B6
:10C620000067A41BBD41C2E9004580688968884253
:10C630000BD2084B1B68D3F89C311818D2E900457F
:10C64000641E75F10005C2E90045401A9060F0BC17
:10C65000704700000004FF1FF8B5284DB0F110032B
:10C66000082901D30C2025E0FB2822D29C0815EBD9
:10C6700084049E0815EB8605D5F80053FF2613F0B9
:10C680000307FFB2FF00BE40B543490111F0E001CE
:10C6900013F00303DBB2DB0099402943C4F8001315
:10C6A000002A02D000F007F801E000F014F80020A2
:10C6B00000E00C20F2BD11491038FB2809D24209D4
:10C6C000012310F01F0013FA00F041F822000020AF
:10C6D00000E00C20704709491038FB280BD24209B2
:10C6E00011EB8201012210F01F0012FA00F0C1F8D4
:10C6F0008000002000E00C207047000000E100E016
:10C70000C0B2002808D002280AD007D304280BD0D2
:10C7100008D305280AD00BE006480AE0064808E0DE
:10C72000064806E0064804E0064802E0064800E045
:10C730000020704700A0064000B0064000C0064040
:10C7400000D0064000A00E4000B00E402DE9F041A0
:10C7500084B004000E00170098463020FDF7BDF9A4
:10C760000500002D01D1042022E040F2F93128001B
:10C77000FDF7A7F92E606F60C5F808800A98E86099
:10C780000B9828610C9868610D98A8610E98286232
:10C7900002950FF2614001900FF2453000900FF2C8
:10C7A0000D130FF2D9020FF21101200000F05CFC12
:10C7B00004B0BDE8F08100002DE9F04182B0050031
:10C7C0008846170000242868466A706A002806D048
:10C7D000706A401C7062B06AA86020004CE0306A49
:10C7E0001030FDF720F9F062F06A002801D1042032
:10C7F00042E04FF47F71F06AFDF763F9F06A316A45
:10C800000160F06A00214160F06A00218160F06AF5
:10C810000021C160B762AF60424616F11C01B069E9
:10C82000336898470400002C1CD17069002806D09A
:10C83000009700AA40F60251F069736998473800E2
:10C84000C0060FD517F00700002801D00C2409E01E
:10C850007069002806D000AA40F61551F069736986
:10C8600098470400002C04D0F06AFDF751F820002E
:10C8700002E0012070622000BDE8F68138B5002595
:10C880000068446A606A401E606200280CD16068DB
:10C89000002804D0E169A069626890470500E06A59
:10C8A000FDF736F80020E062280032BD2DE9F047A0
:10C8B0000E00140027000068D0F82480D8F82890D3
:10C8C000D8F81CA01BE0EDB2082D0CD15FEA49702E
:10C8D00009D508215046D8F80C2090472021504611
:10C8E000D8F80C2090475FEA497005D52900C9B2F5
:10C8F0005046D8F80C2090473570761C7F1E002FCC
:10C9000000F0EA805FEAC97026D498E0D8F82C00DD
:10C910004068D8F82C10096888421DD2D8F82C003D
:10C92000C068D8F82C10421CCA60D8F82C104018E7
:10C930000574D8F82C00C068D8F82C100968884213
:10C9400003D1D8F82C000021C160D8F82C00406831
:10C95000401CD8F82C104860D8F82C004068D8F853
:10C960002C100968884278D25046D8F810108847B1
:10C97000002872D05046D8F8081088470500EDB25C
:10C98000132DC3D1EDB2112DE6D05046D8F80810C2
:10C9900088470500EDB2112DF4D0D8F82C0040687E
:10C9A000D8F82C1009688842ECD2D8F82C00C0685E
:10C9B000D8F82C10421CCA60D8F82C104018057406
:10C9C000D8F82C00C068D8F82C100968884203D128
:10C9D000D8F82C000021C160D8F82C004068401C19
:10C9E000D8F82C104860CDE75046D8F80810884792
:10C9F0000500D8F82C004068D8F82C100968884247
:10CA00001DD2D8F82C00C068D8F82C10421CCA607F
:10CA1000D8F82C1040180574D8F82C00C068D8F845
:10CA20002C100968884203D1D8F82C000021C1607D
:10CA3000D8F82C004068401CD8F82C104860D8F872
:10CA40002C004068D8F82C100968884205D250465E
:10CA5000D8F8101088470028C6D1D8F82C004068B4
:10CA6000002834D0D8F82C00406800281DD0D8F811
:10CA70002C004068401ED8F82C104860D8F82C00D4
:10CA80008068D8F82C10421C8A60D8F82C10401806
:10CA9000057CD8F82C008068D8F82C1009688842EA
:10CAA00003D1D8F82C00002181605FEA89707FF5FE
:10CAB0001AAFEDB20D2D7FF406AF5FEA497004D5D1
:10CAC0000D215046D8F80C2090470A250BE75FEA65
:10CAD000C9607FF514AFE41B2000BDE8F0870000BB
:10CAE0002DE9F8430C0015006E1C0068476AD7F862
:10CAF0002880D7F81C9004E02178F869FA689047FC
:10CB0000641C761E002E1ED05FEAC8703AD45FEA1D
:10CB1000887006D520780A2803D10D214846FA6886
:10CB200090475FEAC860E7D578690028E4D000AA9A
:10CB300040F61551F8697B6998470028DCD10098C8
:10CB40000028D9D1AD1B2800BDE8F283F96A4968F5
:10CB5000FA6A1268914215D2F96AC968FA6A4B1CDE
:10CB6000D360FA6A89180874F86AC068F96A0968B3
:10CB7000884202D1F86A0021C160F86A4068401C0E
:10CB8000F96A4860F86A4068F96A09688842BED262
:10CB90004846396988470028B9D04846B968884767
:10CBA000C0B21328D2D104E0F96A4968491CFA6A74
:10CBB0005160C0B21128E5D04846B9688847C0B274
:10CBC0001128F6D0F96A4968FA6A12689142F0D2DF
:10CBD000F96AC968FA6A4B1CD360FA6A8918087442
:10CBE000F96AC968FA6A12689142DDD1F96A0022CD
:10CBF000CA60D9E770B5150000240268536A0A00BC
:10CC0000921F09D0D21E012A22D940F6F846921B63
:10CC10000ED0521E0FD023E0D86A4068002802D000
:10CC20000120286003E0D8691969884728601FE05F
:10CC3000986A28601CE02A689A622A6882605869AB
:10CC4000002804D02A00D8695B69984704000FE0E7
:10CC50000F202860002068604C20A860002407E0B6
:10CC60005869002804D02A00D8695B6998470400F5
:10CC7000200070BDC0B2002802D0012802D003E01D
:10CC8000024802E0024800E00020704700600640D1
:10CC9000007006402DE9FF4104000D0016001F0042
:10CCA0002420FCF71AFF8046B8F1000F01D10420C0
:10CCB00027E04FF481614046FCF703FFC8F80050BD
:10CCC000C8F80460C8F808700A98C8F80C000B98F7
:10CCD000C8F810000C98C8F81400CDF80C800FF2BA
:10CCE000290002900FF2E90001900FF2D9000090A4
:10CCF0000FF2C5030FF291020FF23D01200000F088
:10CD0000C1F904B0BDE8F08138B50400656AE8698E
:10CD100000280DD16868002803D0A96968696A688D
:10CD200090472800FCF7F4FD00206062002001E03D
:10CD300040F60A2032BD00002DE9F04105000E004A
:10CD400017005FF000082868446AFDF759FCE069A5
:10CD5000002803D0FDF763FC2C2012E00120E061E5
:10CD6000FDF75DFC2762AF60320014F118016069C5
:10CD7000236898478046B8F1000F01D00020E06199
:10CD80004046BDE8F081000038B500250068446ADF
:10CD9000FDF736FCE069401EE061002807D16068BD
:10CDA000002804D0A1692000626890470500FDF7C3
:10CDB00036FC280032BD000080B50068406A8368F8
:10CDC000984702BD80B50068406AC368984702BDB5
:10CDD00010B5030000201B685B6A092907D11720E2
:10CDE0001060002050604C209060002005E01C691D
:10CDF000002C02D098691B69984710BDF8B5040053
:10CE00000D002548076817F51D70FDF7B3FAD7F830
:10CE1000906200E0366817F52470864211D0B06841
:10CE2000210001E0491C401C0A78002A06D0027843
:10CE3000002A03D00A7803789A42F3D000780028B9
:10CE4000E8D117F51D70FDF75CFA17F524708642DE
:10CE500001D100201EE02020FCF73FFE0700002F3C
:10CE600001D1002016E010213800FCF72AFE3E60B8
:10CE7000F06800280DD02A0021003800F368984798
:10CE8000002806D0FCF7D7FF3800FCF741FD002052
:10CE900000E03800F2BD00BF0004FF1F13F0004C9B
:10CEA00003D55B42524263F100039CEA210C00F07F
:10CEB000178010B5644603D34942404261F1000136
:10CEC00000F00EF8640004D34942404261F10001D1
:10CED000244203D55B42524263F1000310BD0000BF
:10CEE0001B4213D1094236D12AB18446B0FBF2F07D
:10CEF00002FB10C2704700F03BB9FCD300220023B4
:10CF000070470B000200002100207047904271EB37
:10CF1000030CF6D370B5B1FA81F4B3FA83F52C1B88
:10CF2000A340C4F1200532FA05F63343A2405FF076
:10CF30000046E64002E05B085FEA3202841A71EBC9
:10CF4000030524BF204629467641F4D302000B0096
:10CF50003000002170BD012ACFD970B5140C20D04B
:10CF6000B1FA81F4B2FA82F5C4F120046419B4F183
:10CF70002006D6D3B2405FF00044F440002502E022
:10CF800052085FEA3303C61A71EB020E24BF304623
:10CF9000714664416D41F3D302000B00200029006B
:10CFA00070BD0C46B1FBF2F102FB11452D0445EAC0
:10CFB0001045B5FBF2F402FB145580B240EA05457A
:10CFC000B5FBF2F002FB105240EA044070BD0000D5
:10CFD000054A126800238B60D2F89421A2FB00233B
:10CFE000C1E90023704700BF0004FF1F2DE9F04393
:10CFF0000C001C490D68D5F89411A1FB00673000A6
:10D0000039004FF47A720023FFF76AFFC4E9000188
:10D010004FF47A785FF000093000390042464B4601
:10D02000FFF75EFFA8FB002308FB013309FB003379
:10D03000B61A9F41D5F89C010021A0FB062300FBF6
:10D04000073301FB063312F5FA7053F100014FF478
:10D050007A720023FFF744FF06000F00A660BDE8C8
:10D06000F08300BF0004FF1F1FB5089C0394002439
:10D070000294079C0194069C009400F003F804B00D
:10D0800010BD00002DE9F84304000D0016001F003C
:10D0900000213648D0F800802800002802D0300057
:10D0A000002801D10C205EE0002001E0491C401C5A
:10D0B000B0F5806F05D2025D3A2AF7D0025D002AF2
:10D0C000F5D1012901D1012801D10C204BE018F53F
:10D0D0001D70FDF74FF9D8F8909201E0D9F8009053
:10D0E00018F5247081450FD04FF48062D9F80810EC
:10D0F000200000F03EF80028F0D118F51D70FDF773
:10D1000000F94FF420602EE02C20FCF7E6FC81466D
:10D11000B9F1000F05D118F51D70FDF7F2F80420E4
:10D1200021E00F214846FCF7CCFCC9F80840C9F8BB
:10D130000C50C9F81060C9F814700898C9F81800A4
:10D140000998C9F81C000A98C9F820000B98C9F87A
:10D150002400494618F52470FDF7E0FA18F51D7013
:10D16000FDF7CFF80020BDE8F28300BF0004FF1FE9
:10D17000704701E0491C521E72B10B7890F800C054
:10D180009C4505D002D24FF0FF3070470120704718
:10D1900010F8013B002BEDD100207047000000008B
:10D1A00000B502B401464FF00300ABBE02BC00BDA7
:10D1B00000B502B401464FF00400ABBE02BC00BD96
:10D1C00000B54FF000014FF00700ABBE00BD0000FE
:10D1D000401E00BF00BF00BF0028F9DC00BF00BF39
:10D1E00000BF00BF7047000038B505462DED028B2B
:10D1F0006868C0F30A5040F2FF7143EC182B884274
:10D2000006D0012806DA284600F0EEF8012801DBF6
:10D21000002406E06A6840F2FE3161F31E526A6043
:10D22000441AD5E9000153EC182B00F0FFF8C5E9CA
:10D230000001BDEC028B21B22846BDE8344000F06D
:10D24000C7B90000F8B52DED028B140003B482B00D
:10D250001F4600F09280DDE902230020002100F04B
:10D2600041FA00F08A809FED488B002C42D5644241
:10D270000FF22C1508260CE0E00707D5D5E90001D0
:10D2800053EC182B00F0D2F841EC180B6408083569
:10D29000761E002C18BF002EEED102A900A800F0C7
:10D2A00031FADDE9020153EC182B00F057FACDE911
:10D2B0000201BDF9001002A800F08AF905004FD55F
:10D2C000002C4FD0002C4BD002A900A800F01AFA75
:10D2D000DDE902012E4A2F4B00F0A8F8CDE902014A
:10D2E000BDF9001002A800F073F9050048BF641EE4
:10D2F000E8D435E0012C33DB0FF2A4050826E00763
:10D3000007D5D5E9000153EC182B00F08FF841EC5C
:10D31000180B64100835761E012C01DB002EEED1AF
:10D3200053EC182B02A8FFF75FFF050018D5012C5E
:10D3300018DB00E0641E012C12DB02A900A800F03B
:10D34000E1F9DDE90201144A144B00F06FF8CDE970
:10D350000201BDF9001002A800F03AF90500E9D475
:10D360002DB20DB1012D08D100F01CFB222101606E
:10D370001FB1386840F001003860DDE9020104B0F7
:10D38000BDEC028BF4BD0000000000000000F03F87
:10D39000436FAC642806C80A3CBF737FDD4F157528
:10D3A0000000000000002440000000000000594080
:10D3B000000000000088C3400000000084D79741AF
:10D3C0000080E03779C34143176E05B5B5B8934681
:10D3D000F5F93FE9034F384D321D30F94877825A4D
:10D3E0003CBF737FDD4F157530B4436803F00042D6
:10D3F00001211B031B0B436004BF0368002B08D1F2
:10D400000DE00368DD0F45EA440444605B000360FF
:10D41000491E4468E302F4D523031B0B43604368B1
:10D420001A434260084630BC70470000B0B581EA3C
:10D43000030C0CF0004C40F2FF7515EA11541DBFAF
:10D4400015EA1357AC42AF4239E0E41923EA4553D9
:10D4500043F48013C90241F0004141EA505EC70223
:10D460001100A7FB020200284FF00000EEFB012094
:10D470004FF00001E3FB072118BF42F00102401802
:10D4800000214941E3FB0E01A4F580640F0302D2A1
:10D4900052004041494154F101046CDD470872F1EA
:10D4A000004250F1000051EB0451A1F580115CBF26
:10D4B00041EA0C01B0BD4CEA05510020B0BD05EABF
:10D4C0001357AC4214BFAF4241E050EA410E1CBFBB
:10D4D00052EA430E02E061460020B0BD24423C44C3
:10D4E0001BD15FEA070EF6D0090302BF01460020F8
:10D4F000AEF1140EB1FA81F7AEEB070401FA07FEA4
:10D500000C37C7F1200100FA07F7C8404EEA000EB9
:10D5100023EA455343F48013A2E733F00043B3FA00
:10D5200083F704BFB2FA82FE77440B3FE41BB7F1E6
:10D53000200E2FBF02FA0EF3BB40C7F1200E22FAD5
:10D540000EFE38BF43EA0E03BA40641C82E750EA7D
:10D55000410E14BF52EA430E6FF000014FF4001762
:10D5600017EB430F8ABF194617EB410FB5E74CEA9B
:10D5700005510020B0BDD4F10104B4F120070FDA49
:10D58000C4F12007520828BF42F0010210FA07F543
:10D5900001FA07F7E1BF2A43E0403843E1400FE0DA
:10D5A000352C98DCC7F1200452EA400220FA07F239
:10D5B00018BF42F0010231FA07F0A1400A430021EE
:10D5C00072F1004250F1000051EB0C01B0BD0000BF
:10D5D00070B504460D466068C0F30A5040F2FF7112
:10D5E000884207D16068000304BF2068002817D074
:10D5F000022070BD20B92046FFF7F6FE012867DA49
:10D60000012D0FDB40F2FF71091A8D420AD36068C9
:10D6100000284CBF9FED2F0B9FED300B84ED000BCE
:10D62000012070BD4142A942616806DA6FF31E51C4
:10D63000401941EA0050606041E0401E63680122E9
:10D64000451962F31F5305F1350001F00041636095
:10D65000352803D361600020206070BD002215F1E1
:10D660001F0F04DA226823600020203560606842C2
:10D6700013D0521E25689241C0F12003D2439D4031
:10D6800045EAD27225686668C54006FA03F32B4363
:10D690002360636823FA00F060606068084360609C
:10D6A000B2F1004F03D80DD12078C0070AD5206809
:10D6B000401C2060206828B96068401C60604FF002
:10D6C000FF3070BD6068884204BF20680028F6D132
:10D6D000002070BD000000000000F0FF000000000E
:10D6E0000000F07F90420CD141EA030C50EA4C0C50
:10D6F00007D0994205D14FF4001C1CEB410F38BFF5
:10D700008942704738B50C4605466068C0F30A5038
:10D7100040F2FF7188420BD100202880606800032E
:10D7200004BF2068002801D0022032BD012032BD94
:10D73000012804DA2046FFF757FE01280ADA62685A
:10D7400040F2FE3161F31E526260401A28804FF0B1
:10D75000FF3032BD0020288032BD0000F0B540F21D
:10D76000FF7581EA030C0CF0004C15EA11541DBF43
:10D7700015EA1357AC42AF42E5E0BC41C1F31301D7
:10D78000C3F31303801A994143F4801304D2641E37
:10D790004000494180185941C90241EA5051B1FB4A
:10D7A000F3F603FB1611A2FB0675D7EBC020A941C7
:10D7B00002D2761E80185941C90241EA5051B1FB8C
:10D7C000F3FE03FB1E11A2FB0E75D7EBC020A9418F
:10D7D00003D2AEF1010E80185941890241EA9051FD
:10D7E000760546EA8E2EB1FBF3F603FB1611A2FB7B
:10D7F0000675D7EB8020A94102D2761E80185941C8
:10D80000C90241EA50514EEA060EB1FBF3F603FBA2
:10D810001611A2FB0675D7EBC020A94102D2761ED5
:10D8200080185941C90241EA5051B1FBF3F703FB9B
:10D830001711A2FB0735D3EBC020A94167F1000700
:10D840000CBF004247F0010766F3D5274FEA1E31AF
:10D85000B80814F5806412DDBD0775F1004250EB85
:10D860000E5051EB045111F5801F5CBF41EA0C01D1
:10D87000F0BD4CF07F6141F0E0410020F0BDBD07FC
:10D880006D0840EA0E5041F48011D4F10104B4F166
:10D8900020060ADAC4F120060200E04001FA06F38D
:10D8A000E1401843B24015430EE0342C13DCC6F1BE
:10D8B000200445EA40056D0820FA06F2154321FAD6
:10D8C00006F0A1400D43002175F1004250F1000027
:10D8D00051EB0C01F0BD00205FEA0C01F0BDCFB9A7
:10D8E00092185B41B3FA83F704BFB2FA82F6BF190C
:10D8F0000B3FB7F120062FBF02FA06F3BB40C7F17A
:10D90000200622FA06F638BF3343BA401CB1E419A8
:10D91000641E33E77F4231F00041B1FA81F404BF65
:10D92000B0FA80F6A4190B3CB4F120062FBF00FA20
:10D9300006F1A140C4F1200620FA06F638BF3143B3
:10D94000A0403C1B1AE7AC421ABF05EA1357AF428E
:10D9500012E050EA41061CBF52EA4306BFE750EA14
:10D960004107304661461CBF41EA0551F0BD52EA0D
:10D97000430C08BFC143F0BD00204FF4001616EB66
:10D98000410F98BF16EB430F08BF16EB410F24BFA2
:10D99000C14305E016EB430F0CBF61464CEA05514D
:10D9A000F0BD0000014800F003B800000005FF1FB3
:10D9B0007047000080B50121022000F0DBFADFF89B
:10D9C0002C05006830F0C000DFF820150860DFF893
:10D9D000200500210160DFF81C0500210160DFF84F
:10D9E000180500210160DFF8140500210160DFF84F
:10D9F000FC04006850F08000DFF8F0140860DFF8E5
:10DA00000005DFF8001509680180DFF8F404DFF88D
:10DA1000F81409684180DFF8E804DFF8F0140968B9
:10DA20008180DFF8DC04DFF8E8140968C180DFF8E2
:10DA3000D004DFF8E01409680181DFF8C404DFF8DE
:10DA4000D81409684181DFF8B804DFF8D0140968F8
:10DA50008181DFF8AC04DFF8C8140968C181DFF800
:10DA6000A0040088DFF898140969B0EB2130DFF8D2
:10DA70009014C861DFF888040069DFF88414C9696C
:10DA80000818DFF87C140861DFF874048088DFF878
:10DA900070144969B0EB2130DFF864140862DFF8D4
:10DAA00060044069DFF85814096A0818DFF8501458
:10DAB0004861DFF84C040089DFF844148969B0EB51
:10DAC0002130DFF83C144862DFF834048069DFF865
:10DAD0003014496A0818DFF828148861DFF8200438
:10DAE000806CDFF81C14D1F89410DFF8142412EBCA
:10DAF0004101098D401ADFF808148864DFF800043A
:10DB0000D0F89400DFF8F81311EB4000DFF8F013C1
:10DB100049880185DFF8E803806CDFF8E413D1F869
:10DB20009410DFF8DC2312EB4101098D10FA81F02B
:10DB3000DFF8CC138864DFF8C803D0F89400401CE9
:10DB4000DFF8BC13C1F89400DFF8B403D0F89400F8
:10DB5000102804D3DFF8A8030021C0F89410DFF8E0
:10DB6000A003806C102190FBF1F0DFF89413C1F852
:10DB70009800DFF8B0030068B0F5C86F80F08880C7
:10DB8000DFF8A0030068DFF8A013DFF87423D26980
:10DB900021F81020DFF88C030068DFF88C1311EBFC
:10DBA0004000DFF85C13096AA0F8801CDFF87403FA
:10DBB0000068DFF8741311EB400010F5C850DFF86F
:10DBC0004013496A0180DFF85C030068DFF85813EE
:10DBD00011EB400010F51650DFF82413D1F898101F
:10DBE0000180DFF840030068DFF83C1311EB4000D0
:10DBF00010F54850DFF80813B1F906100180DFF87E
:10DC000024030068DFF8201311EB400010F57A5070
:10DC1000DFF8EC12B1F90C100180DFF8080300689E
:10DC2000DFF8041311EB400010F59640DFF8D01236
:10DC3000B1F90E100180DFF8EC020068DFF8E8129D
:10DC400011EB400010F5AF40DFF8B412B1F9081045
:10DC50000180DFF8D0020068401CDFF8C8120860BD
:10DC6000DFF8C0020068B0F5487F03D1802000F0E3
:10DC7000FDFD0DE0DFF8AC020068B0F5C86F07D11C
:10DC80004FF4807000F0F2FDDFF89802002101608F
:10DC90000021022000F06EF901BDDFF8900200685B
:10DCA00050F08050DFF884120860DFF880020068CE
:10DCB00050F00060DFF874120860DFF8740200684A
:10DCC00050F08050DFF868120860DFF864020068E6
:10DCD00050F00060DFF858120860704744218160FE
:10DCE0000021C16000210162002141620021016523
:10DCF00020214160102101607047202101606521D1
:10DD000081600021C16000210162C7214162416A36
:10DD10000906FCD4C16C826C5118426C5118026C1B
:10DD20005118C26B5118826B5118490889B251F4CD
:10DD30000041C162C16E826E5118426E5118026E6E
:10DD40005118C26D5118826D5118490889B251F4A9
:10DD500000410163406A400601D5FF2000E0002039
:10DD6000704713F0010312F0010211F01F0111EBD3
:10DD7000421140F823107047016A51F040010162DE
:10DD8000704780B5DFF8A801006850F48000DFF824
:10DD9000A0110860DFF89C0100210160DFF8980104
:10DDA00040F203210160DFF8940140F20321016099
:10DDB000DFF88C0140F203210160DFF8880140F2B6
:10DDC00003210160DFF880018A210160DFF87C0116
:10DDD0008A210160DFF878018A210160DFF874018F
:10DDE0008A210160DFF870014FF48A71016000221E
:10DDF000DFF868115820FCF72BFC01220321582082
:10DE0000FEF72AFC394840F6A101016001BD80B54A
:10DE1000FFF743FF5248FFF770FF5249086052482E
:10DE2000FFF76BFF4F4948605048FFF766FF4D49C9
:10DE300088604F48FFF761FF4A49C8604848FFF7CC
:10DE40004DFF4948FFF74AFF4848FFF747FF48485A
:10DE5000FFF744FF0023002210214148FFF781FF14
:10DE60000123002211213E48FFF77BFF00230022FF
:10DE700010213D48FFF775FF012300221A213A487F
:10DE8000FFF76FFF0023002210213848FFF769FFDA
:10DE9000012300220C213548FFF763FF00230022F5
:10DEA00007213348FFF75DFF012300220521304899
:10DEB000FFF757FF2A48FFF75FFF2B48FFF75CFF8C
:10DEC0002A48FFF759FF2A48FFF756FFFFF759FF87
:10DED00001BD002107E04FF44862134B02FB013201
:10DEE00040F82120491C0B29F5DB704700600340F6
:10DEF000146003403C600340646003408C60034056
:10DF00009005FF1F10B0034014B0034010B00B4049
:10DF100014B00B4010C0034014C0034010C00B40AD
:10DF200014C00B40AC8FFF1F2C06FF1F3080044035
:10DF30003C80044018800440106003403860034077
:10DF400060600340886003401C60034044600340FD
:10DF50006C600340946003400C600340B5D900003E
:10DF600000B003408005FF1F00B00B4000C003401D
:10DF700000C00B40012804D026D3032819D00CD3AD
:10DF800022E0C80704D582485FF08071016003E099
:10DF900080485FF08071016016E0C80704D57C48B6
:10DFA0005FF00071016003E07A485FF0007101608A
:10DFB0000AE0C80704D576485FF08061016003E09D
:10DFC00074485FF0806101607047002803D1724897
:10DFD0008021016002E071488021016070470128C2
:10DFE00004D16B484FF40051016003E069484FF4DD
:10DFF000005101607047002804D169484FF4005176
:10E00000016003E067484FF4005101607047002849
:10E0100004D165484FF40061016003E063484FF4A8
:10E02000006101607047002804D15F484FF48051BF
:10E03000016003E05D484FF48051016070470028A3
:10E0400004D159484FF40051016003E057484FF4A0
:10E05000005101607047002804D153484FF48041BB
:10E06000016003E051484FF480410160704700288F
:10E0700004D14D484FF40041016003E04B484FF498
:10E080000041016070474A480068C00401D5002083
:10E0900000E00120704780B546480068C00110D5F7
:10E0A0004448006850F08070424908604048006869
:10E0B000C00403D5012000F0D9FB02E0022000F0EB
:10E0C000D5FB01BD80B53C480068C00110D53A4879
:10E0D000006850F0807038490860384800680007D0
:10E0E00003D5042000F0C2FB02E0082000F0BEFBD4
:10E0F00001BD80B52F48006850F430202D490860DC
:10E100002C48006850F010002A4908602C48002173
:10E1100001602C48012101602B481E210160284824
:10E12000006850F480502649086000222749672083
:10E13000FCF78EFA012203216720FEF78DFA01BD5C
:10E1400080B51D48006850F430201B4908601A480B
:10E15000006850F01000184908601D480021016057
:10E160001C48002101601C480C210160184800680F
:10E1700050F0080016490860002218496820FCF792
:10E1800067FA012203216820FEF766FA01BD00004C
:10E1900008F00F4004F00F4008F10F4004F10F4069
:10E1A00088F00F4084F00F40C8F00F40C4F00F40DB
:10E1B00010F00F40309004400CA0044050F00F408D
:10E1C000C0900440C4900440C890044097E0000010
:10E1D000C0A00440C4A00440C8A00440C5E00000A2
:10E1E00081FB0001C00F40EA4100C917704700B52C
:10E1F00040F6A66181FB0001B0F1404071F5EA7183
:10E200005FF000420023FEF749FE002905DC01DB38
:10E210005A2802D20020002108E0002906DB02DC97
:10E22000B0F5D46F02D340F25370002100BD00005E
:10E2300030B585B0040000A901A800F0BFFDDFF8EB
:10E240007C0AC068322880F0AB80DFF8700A406832
:10E25000002852D1DFF8642AD2E9040100F0CAFD97
:10E2600000EE100ADFF8540AD0ED160A20EE200A5C
:10E27000DFED8C0A80EE200AF7EE000AB4EE600AA9
:10E28000F1EE10FA32D5DFF8342AD2E9040100F0B9
:10E29000B1FD00EE100ADFF8240AD0ED160A20EED8
:10E2A000200ADFED800A80EE200AFFEE000AB4EEBD
:10E2B000600AF1EE10FA14DBDFF8002AD2E904015B
:10E2C00000F098FD00EE100ADFF8F009D0ED160A14
:10E2D00020EE200ADFED730A80EE200ABEEEE00A8F
:10E2E00003E09FED710ABDEEC00A03E09FED6E0AE8
:10E2F000BDEEC00A10EE105AA8E0DFF8C029D2E93E
:10E30000040100F077FD00EE100ADFF8B009D0ED4F
:10E31000160A20EE200ADFED630A80EE200AF7EEEF
:10E32000000AB4EE600AF1EE10FA32D5DFF88C295B
:10E33000D2E9040100F05EFD00EE100ADFF87C096E
:10E34000D0ED160A20EE200ADFED560A80EE200AF4
:10E35000FFEE000AB4EE600AF1EE10FA14DBDFF80B
:10E360005C29D2E9040100F045FD00EE100ADFF857
:10E370004C09D0ED160A20EE200ADFED4A0A80EEA5
:10E38000200ABEEEE00A03E09FED470ABDEEC00A98
:10E3900003E09FED450ABDEEC00A10EE105A55E0AD
:10E3A000DFF818094068002828D1DFF8100990ED3F
:10E3B000160AF7EE000AB4EE600AF1EE10FA16D56E
:10E3C000DFF8F80890ED160AFFEE000AB4EE600AD6
:10E3D000F1EE10FA06DBDFF8E40890ED160ABEEE67
:10E3E000E00A03E09FED300ABDEEC00A03E09FEDB6
:10E3F0002E0ABDEEC00A10EE105A27E0DFF8BC0866
:10E4000090ED160AF7EE000AB4EE600AF1EE10FA8B
:10E4100016D5DFF8A80890ED160AFFEE000AB4EE54
:10E42000600AF1EE10FA06DBDFF8900890ED160AAC
:10E43000BEEEE00A03E09FED1C0ABDEEC00A03E059
:10E440009FED190ABDEEC00A10EE105A019928007E
:10E45000FFF7C6FE019000992800FFF7C1FE00906B
:10E4600000A902A800F0E9FC05000298FFF7BFFE32
:10E470002060DFF848084068002808D10398FFF7BB
:10E48000B6FE60600498FFF7B2FEA06007E0049853
:10E49000FFF7ADFE60600398FFF7A9FEA06005B02E
:10E4A00030BD0000000048520000004F80B5DFF88A
:10E4B0000C08DFF80C188162DFF80008DFF8041898
:10E4C0000163DFF8F807DFF8F817C162DFF8EC073F
:10E4D000DFF8F4170164DFF8E407DFF8EC17816474
:10E4E000DFF8D807DFF8D8174164DFF8D00732210A
:10E4F0004163DFF8C8070A218163DFF8C0070A21FA
:10E50000C163DFF8B8073221C164DFF8B0070A2120
:10E510000165DFF8A8070A214165DFF8A0270FF29F
:10E52000C1514E20FCF794F8012203214E20FEF742
:10E5300093F8DFF89807006850F08070DFF88C17C8
:10E540000860DFF88C07DFF88C1709680160DFF8D6
:10E55000840720210160DFF87807DFF87C1709685D
:10E560000160DFF86C07DFF8741709680160DFF8F5
:10E570006007DFF86C1709680160DFF85407DFF8FF
:10E58000641709680160DFF84807DFF85C1709685D
:10E590000160DFF83C07DFF8541709680160DFF815
:10E5A000380700210160DFF8340700210160DFF83F
:10E5B000300700210160DFF82C0700210160DFF83F
:10E5C000280700210160DFF8240700210160DFF83F
:10E5D000200700210160DFF81C0700210160DFF83F
:10E5E0001807006850F00400DFF80C170860DFF827
:10E5F0000807006850F00100DFF8FC160860DFF83B
:10E60000FC0640F253710160DFF8F406002101605E
:10E61000DFF8F0062A210160DFF8EC060021016036
:10E62000DFF8E80600210160DFF8E406DFF8E41611
:10E630000160DFF8E40600210160DFF89C060C2190
:10E640000160DFF898060C210160DFF894060C21C8
:10E650000160DFF890060C210160DFF88C060C21C8
:10E660000160DFF888060C210160DFF884060021D4
:10E670000160DFF8800600210160DFF8A0060021BC
:10E680000160DFF89C0600210160DFF89806002198
:10E690000160DFF8940600210160DFF89006002198
:10E6A0000160DFF88C0600210160DFF88806002198
:10E6B0000160DFF8840600210160DFF88006002198
:10E6C0000160DFF8740600210160DFF874060221A2
:10E6D0000160DFF8700640210160DFF81C060721A9
:10E6E0000160DFF864064FF420710160DFF85C061A
:10E6F00000210160DFF8580600210160DFF85406B0
:10E7000040210160DFF85006C0210160DFF84C06AF
:10E710004AF6FF210160DFF8BC052821016001BD38
:10E72000E0B5DFF89825D160DFF890154860002843
:10E7300006D1DFF88805DFF88415896A816505E070
:10E74000DFF87805DFF87415096C8165DFF86C0572
:10E75000C068002101000020DFF86025C2E9040143
:10E76000DFF85805C06800F01AFB00A8FFF760FD4D
:10E77000DFF8A80500990160DFF8A40500990160A1
:10E780000198DFF8A01508600198DFF89C15086073
:10E790000298DFF8981508600298DFF89415086071
:10E7A000FBF72EFFDFF8A005006850F48070DFF85B
:10E7B00098150860DFF88805006850F08000DFF8E1
:10E7C00080150860DFF8400500210160DFF878055A
:10E7D000006830F48070DFF870150860DFF87C05A1
:10E7E00000210160DFF8EC04006830F08000DFF801
:10E7F000E4140860DFF8DC04006850F04000DFF843
:10E80000D4140860FBF70BFF07BDDFF8C8040068ED
:10E8100030F04000DFF8BC140860DFF840054AF62D
:10E82000FF2101607047DFF8AC040068400601D5A5
:10E83000012000E00020704738B5040010000B00F4
:10E8400000220100DFF8180500F0C5FC0500002DCE
:10E8500008D100F0E4FB20602168DFF8040500F037
:10E86000C8FB01E000202060280032BD80B5010017
:10E87000DFF8EC0400F0D9FB02BD80B50021DFF821
:10E88000E00400F0B1FB01BD70B504000D001600FE
:10E89000FFF7C9FF00280DD1FFF7F5FB002809D0CD
:10E8A0000521E4B22000FFF73BFF320029000120E0
:10E8B00000F04AF870BD10B50400FFF7B4FF00285F
:10E8C00004D022000021022000F03EF810BD80B5E7
:10E8D000FFF79BFFFBF794FEDFF8E0030021C16028
:10E8E000DFF8D80300220023C0E90423DFF8CC03BB
:10E8F00000218160DFF8C40300220023C0E9062361
:10E90000DFF8B80300210160FBF789FE01F0FFF892
:10E9100001BD10B50400FBF773FE6822DFF89C13FD
:10E92000200001F0DFF9FBF77AFE10BD10B50400FE
:10E93000FBF766FE68222100DFF8800301F0D2F9C0
:10E94000FBF76DFE10BD0000F0B59BB004000D009C
:10E95000170000A8FFF7DDFF012C02D10120009075
:10E9600003E0022C01D102200090039EB54200F08A
:10E97000B380002F41D0019800280DD1022C0BD17B
:10E9800001F0AFF8F2EE020AB4EE600AF1EE10FA0E
:10E9900001D5052500E00F250198012802D1022CA0
:10E9A00000D1062F380001F0ADF90022DFF8B433B2
:10E9B000FEF7D4FE01F0B4F900EE100ADFED580ABC
:10E9C00020EE200AFCEEC00ACDED020A00EE905ABD
:10E9D000F8EE600A01EE106AB8EE411A70EEC10A54
:10E9E0009FED501A60EE810A80EE800A10EE100A48
:10E9F00001F0DEF9CDE906010DE001200290A81B2F
:10EA0000002100220123A2FB006702FB017703FB28
:10EA10000077CDE90667019800282DD1012C14D18B
:10EA20009DED0C0ADDED160A30EE600A10EE100ABC
:10EA300001F0FAF90022CC4BFEF790FE01F070F9DC
:10EA400017904FF4FA50189043E0022C41D19DEDFD
:10EA50000B0ADDED160A30EE600A10EE100A01F026
:10EA6000E3F90022C04BFEF779FE01F059F9179047
:10EA70004FF4FA5018902CE0012C14D19DED120A9D
:10EA8000DDED160A30EE600A10EE100A01F0CCF946
:10EA90000022B54BFEF762FE01F042F917904FF4E9
:10EAA000FA50189015E0022C13D19DED110ADDEDFE
:10EAB000160A30EE600A10EE100A01F0B5F90022D5
:10EAC000A94BFEF74BFE01F02BF917904FF4FA50CB
:10EAD000189000A8FFF72AFF01F019F81BB0F0BD4D
:10EAE00080B501210320FFF745FA7A480068000647
:10EAF00005D57848006830F0800076490860914874
:10EB0000006830F080008F49086000219748006855
:10EB100001F025FA00210320FFF72CFA01BD0000C7
:10EB200000007A460000804F3EB5002001F0A4F9B5
:10EB30008E4908608D480068002802D10020F9F74E
:10EB4000BBFD8A48006801F0D4F901210320FFF7DA
:10EB500011FA00A8FFF76CFB70480099016070483B
:10EB60000099016001986F49086001986E4908603A
:10EB700002986E49086002986D4908607048006804
:10EB800050F080006E49086079480068B0F5C86FA1
:10EB90001AD277480068774911EB400010F5C84059
:10EBA0000099018072480068724911EB400010F52D
:10EBB000E140019901806E4800686E4911EB400008
:10EBC00010F5FA40029901803C488068002853D033
:10EBD0003A48D0E904233948D0E90645101953EBE7
:10EBE0000501364AC2E904013448D0E9042312F190
:10EBF000004053F100013148C1603048C06800F066
:10EC0000D7F82E488068401E2C4988602B488068C1
:10EC1000002831D129484068002824D127480068BD
:10EC2000012820D100F05DFFF2EE020AB4EE600A86
:10EC3000F1EE10FA15D52148806D01F0F5F80200CB
:10EC40000B0000204C4901F0C1F90022464BFEF7B1
:10EC500085FD01F065F81949C86518484FF4FA5167
:10EC6000016600F054FF15480068022801D1FFF743
:10EC70002EFE1248032101601048006E00280FD0BC
:10EC80000E4890ED160A0D48D0ED170A30EE200A16
:10EC90000A4880ED160A0948006E401E07490866BA
:10ECA0000648C068052801D2FFF711FE00210320A5
:10ECB000FFF760F945E70148704700001805FF1F9E
:10ECC0009A99193F6666263F9A99993E3C8004407E
:10ECD000709BFF1F008003400C80034014800340A2
:10ECE0001C800340248003402C8003403480034078
:10ECF0003C8003404480034054800340088003402C
:10ED00004C8003405C8003400480034068800340E3
:10ED10006480034072727200908003401080034050
:10ED20001880034020800340288003403080034047
:10ED300038800340788003407C8003408880034013
:10ED4000588003406C8003408C80034080800340E7
:10ED500074800340848003406080034094800340BB
:10ED6000749BFF1F000024400040BF40989BFF1F82
:10ED7000AC8FFF1F2C06FF1F0000E03F30B50200E4
:10ED8000002300240125A4FB020104FB031105FB61
:10ED900002114FF47A520023FEF7A2F830BD80B57D
:10EDA000104900220A60FFF7E9FF0F49086001BD22
:10EDB00080B5FFF7E3FF0C49086001BD094A1268FE
:10EDC000520D0A4B53F822300360094850F82200D4
:10EDD0000860044800680449096808180149086087
:10EDE00070470000A89BFF1FAC9BFF1FB46E010083
:10EDF000B48E010050EA010200F00E80094200BF0B
:10EE00000BD1B0FA80F18840C1F19D01C90502061D
:10EE100072F1004241EB10207047B1FA81F241409B
:10EE20009040C2F1200261FA02F181EA000018BFAD
:10EE300040F0010002F19D01E8E7F0B40A6846F6EF
:10EE4000DA63121413FB02F24C685200A31055103F
:10EE5000EE182146B6F1804FA8BF6FF0404205DAA8
:10EE6000324612F1804FB8BF4FF0404252005D1B56
:10EE700015F1804FB8BF4FF0404305DB2B46B3F18F
:10EE8000804FA8BF6FF040435B006FF04047002AFF
:10EE900036D54FEA610C002B0ED58CFA87F4002191
:10EEA000002CA8BF2146416083FAA4F1016082FAD8
:10EEB000A1F18160052059E0012C10DB8CFAA6F34A
:10EEC00083FA87F40023002CA8BF2346036082FA4C
:10EED000A4F2826081FA82F14160032046E085FA63
:10EEE000ACF282FA87F40022002CA8BF224602600E
:10EEF00083FA84F2426081FAA2F18160042035E055
:10EF0000002B23D5012C0FDB86FAA7F40022002C5E
:10EF1000A8BF2246826081FA84F141606A0082FAC9
:10EF2000A1F10160012021E04B1086FAA3F383FADE
:10EF300087F40023002CA8BF2346436081FAA4F184
:10EF4000816082FA81F1016006200FE085FA86F186
:10EF500081FAA7F40021002CA8BF2146816082FA23
:10EF600084F1016083FA81F141600220F0BC7047B6
:10EF700070B504000E00DFF8A4020568002114F14A
:10EF80000800FBF7C5FB0020A061E661F00703D590
:10EF90005FF0FF30206201E000202062FBF730FBD1
:10EFA000D5F81C03002804D1002115F54770FBF7A4
:10EFB000AFFBDFF86C026061D5F81C0300E000686D
:10EFC00015F54771884206D0A042F8D1FBF727FB20
:10EFD0004FF4826007E0210015F54770FBF79EFBB8
:10EFE000FBF71DFB002070BD80B50022FFF7C0FFBE
:10EFF00002BD70B504000D0088480668FBF700FBF1
:10F0000060698749884203D0FBF709FB392005E096
:10F01000A069A843A061FBF702FB002070BD7F48F8
:10F020000068C069D0F8A00070472DE9F0410400E5
:10F030000E007A480568FBF7E3FA60697849884270
:10F0400003D0FBF7ECFA392052E0A0690643208A8E
:10F05000002847D0A06841E007003C3FD0F800807E
:10F0600097F82810090606D5D7F8A0103140D7F830
:10F07000A020914207D097F8281009062DD4D7F880
:10F08000A010314229D04168006808604160208AA0
:10F09000401E2082B868C00510D5786839680160C4
:10F0A0004860B5F88801401EA5F88801B86830F4BA
:10F0B0008070B860B86850F00300B8600020B86392
:10F0C0003800FAF7FCFFD7F8A0003040C7F8A000DE
:10F0D000206AD7F8A01008408643404614F1080182
:10F0E0008842B9D1A661FBF79AFA05F09DFC002091
:10F0F000BDE8F0812DE9F84304000D0016001F0063
:10F1000046480068018B002901D00D2061E05FF0C6
:10F110000008D0F81C90FBF773FA606940498842F8
:10F1200003D0FBF77CFA392053E0002E03D0A0690E
:10F130002840A84204D0002E0FD1A06928420CD04C
:10F14000A0692840C9F8A000A069216A2940884325
:10F15000A061FBF764FA40463BE0C9F8A050002EDE
:10F1600006D0D9F8280050F08000C9F8280005E042
:10F17000D9F8280030F08000C9F8280019F13C01C6
:10F1800014F10800FBF7CAFA40F22D40C9F8080054
:10F1900014F10800C9F83800002F10D00898002892
:10F1A00003D03800FBF72BFD02E03800FBF7B1FC81
:10F1B000D9F83800002804D04FF4447801E005F075
:10F1C00044FC6069002801D15FF03908FBF727FA99
:10F1D0004046BDE8F283F0B585B0002B15D001ACF8
:10F1E000104DB5E8C010A4E8C0100C3D0C3CDDE9A2
:10F1F00001671C00002534197D41CDE9014500233C
:10F20000009301ABFFF776FF04E000230093002397
:10F21000FFF770FF05B0F0BD000000000004FF1F05
:10F220006E76656CF06D010000B585B000A800F049
:10F230008DFF00A9DFF84C0A00F0CEFF05B000BD3D
:10F2400038B501210120FEF795FE00210220FEF7CE
:10F2500091FE00210320FEF78DFEFFF70EFBFFF766
:10F26000E3FF01F02BF9DFF8201ADFF8200A01F0A4
:10F2700074FAFEF7CCFD002203210020FAF777FC98
:10F28000002204210020FAF772FC00220521002050
:10F29000FAF76DFC4FF47A70FBF720FC0120FEF7C3
:10F2A000AAFE6420FBF71AFC00210120FEF762FE93
:10F2B000FFF7FCF8FEF71DFFFEF742FF0120FEF707
:10F2C0008EFE002201210020FAF751FCDFF8BC2954
:10F2D00007210020FAF74BFCDFF8B02906210020B7
:10F2E000FAF745FCFFF7E7FC040004E029000120E1
:10F2F000FEF740FE6D1C7922022100A8FFF79CFA60
:10F300000028F3D1009800070DD5FFF7E0FA01209F
:10F310002062606A401C606241F28830FBF7DEFBCD
:10F3200000202062E7E70098C00702D5FFF7CFFA78
:10F33000E1E7009840060AD56068012803D1606DB6
:10F34000FFF7B9FAD7E7E06BFFF7B5FAD3E7009814
:10F35000C00605D5226DE16C0120FFF795FACAE7DA
:10F3600000988006C7D5A26B616B0020FFF78CFA6E
:10F37000C1E70000F8B52DED028B00EE100A9FEDFD
:10F38000A98AF6EE068AB8EEC00A10EE100A00F05E
:10F390004BFD5FF06632DFF8F838FEF747F80400FF
:10F3A0000D0018EE100A00F03FFD0022DFF8E438EF
:10F3B000FEF73CF806000F0018EE900A00F034FD4E
:10F3C00032003B00FEF732F802000B00200029005B
:10F3D000FEF7C4F900F0A4FC00EE100ABDEC028BAD
:10F3E000F1BD0000F8B52DED028B9FED8E8AF6EE93
:10F3F000068A10EE100A00F017FD5FF06632DFF8A3
:10F400009038FEF713F804000D0018EE100A00F013
:10F410000BFD0022DFF87C38FEF708F806000F002D
:10F4200018EE900A00F000FD32003B00FDF7FEFFF1
:10F4300002000B0020002900FEF790F900F070FC9C
:10F4400000EE100ABDEC028BF1BD000038B52DEDC9
:10F45000028B00EE100A9FEDB28ADFEDB28AB8EEA1
:10F46000C00A10EE100A00F0DFFC5FF06632DFF831
:10F470002038FDF7DBFF04000D0038EE280A10EEFF
:10F48000100A00F0D1FC22002B00FDF7CFFFDFF8BF
:10F490000828DFF80838FDF7C9FF04000D0018EE52
:10F4A000100A00F0C1FC0022DFF8E837FDF7BEFFCC
:10F4B00002000B0020002900FEF750F900F030FC9C
:10F4C00000EE100ABDEC028B31BD000038B52DED09
:10F4D000028B9FED938ADFED938A10EE100A00F005
:10F4E000A3FC5FF06632DFF8A837FDF79FFF04004A
:10F4F0000D0038EE280A10EE100A00F095FC2200EC
:10F500002B00FDF793FFDFF89027DFF89037FDF72A
:10F510008DFF04000D0018EE100A00F085FC00229B
:10F52000DFF87037FDF782FF02000B002000290092
:10F53000FEF714F900F0F4FB00EE100ABDEC028BAC
:10F5400031BD000038B52DED028B00EE100A9FEDA5
:10F55000748ADFED738AB8EEC00A10EE100A00F06C
:10F5600063FC5FF06632DFF82837FDF75FFF0400C9
:10F570000D0038EE280A10EE100A00F055FC2200AB
:10F580002B00FDF753FF04000D0018EE100A00F0E9
:10F590004BFC0022DFF8FC36FDF748FF02000B00B1
:10F5A00020002900FEF7DAF800F0BAFB00EE100A9E
:10F5B000BDEC028B31BD000038B52DED028B9FED07
:10F5C000588ADFED578A10EE100A00F02DFC5FF02C
:10F5D0006632DFF8BC36FDF729FF04000D0038EE77
:10F5E000280A10EE100A00F01FFC22002B00FDF785
:10F5F0001DFF04000D0018EE100A00F015FC00229B
:10F60000DFF89036FDF712FF02000B002000290002
:10F61000FEF7A4F800F084FB00EE100ABDEC028BAC
:10F6200031BD00000AD7233D38B52DED028B00EE29
:10F63000100A9FEDA78ADFEDA78AB8EEC00A10EE88
:10F64000100A00F0F1FB5FF06632DFF84436FDF798
:10F65000EDFE04000D0038EE280A10EE100A00F04E
:10F66000E3FB22002B00FDF7E1FEDFF83426DFF894
:10F670003436FDF7DBFE04000D0018EE100A00F032
:10F68000D3FB0022DFF80C36FDF7D0FE02000B00A2
:10F6900020002900FEF762F800F042FB00EE100A9D
:10F6A000BDEC028B31BD000038B52DED028B9FED16
:10F6B000888ADFED888A10EE100A00F0B5FB5FF053
:10F6C0006632DFF8CC35FDF7B1FE04000D0038EEF0
:10F6D000280A10EE100A00F0A7FB22002B00FDF70D
:10F6E000A5FEDFF8BC25DFF8BC35FDF79FFE040062
:10F6F0000D0018EE100A00F097FB0022DFF8943599
:10F70000FDF794FE02000B0020002900FEF726F80A
:10F7100000F006FB00EE100ABDEC028B31BD0000CC
:10F7200000E0924500E8004738B52DED028B00EE71
:10F73000100A9FED678ADFED678AB8EEC00A10EE07
:10F74000100A00F071FB5FF06632DFF84435FDF718
:10F750006DFE04000D0038EE280A10EE100A00F0CD
:10F7600063FB22002B00FDF761FE04000D0018EE84
:10F77000100A00F059FB0022DFF81835FDF756FE9D
:10F7800002000B0020002900FDF7E8FF00F0C8FA96
:10F7900000EE100ABDEC028B31BD000038B52DED36
:10F7A000028B9FED4B8ADFED4B8A10EE100A00F0C2
:10F7B0003BFB5FF06632DFF8D834FDF737FE04001C
:10F7C0000D0038EE280A10EE100A00F02DFB220082
:10F7D0002B00FDF72BFE04000D0018EE100A00F0C0
:10F7E00023FB0022DFF8AC34FDF720FE02000B0003
:10F7F00020002900FDF7B2FF00F092FA00EE100A97
:10F80000BDEC028B31BD80B500EE100AB8EEC00A27
:10F8100010EE100A00F008FB5FF06632DFF870347B
:10F82000FDF704FE0022DFF86C34FDF797FF00F0CF
:10F8300077FA00EE100A10EE100A00F0F5FADFF881
:10F840006824DFF8683401F06FFADFF86424DFF829
:10F850006434FDF783FF02000B000020DFF858142A
:10F8600000F0B4FB00F05CFA00EE100A01BD80B5B8
:10F8700010EE100A00F0D8FA5FF06632DFF81034AC
:10F88000FDF7D4FD0022DFF80C34FDF767FF00F030
:10F8900047FA00EE100A10EE100A00F0C5FADFF881
:10F8A0000824DFF8083401F03FFADFF80424DFF819
:10F8B0000434FDF753FF02000B000020DFF8F813BB
:10F8C00000F084FB00F02CFA00EE100A01BD0000ED
:10F8D00000800945007C924800EE100AB8EEC00A8C
:10F8E0007047704780B5DFF89C0300F0CDFC01BD88
:10F8F00080B5E44800F082FD01BDF8B52DED028B26
:10F9000092B0DFF8B80300210160DFF8B4030021F2
:10F9100001602AE0DFF8AC0390ED030ADFF8A403EE
:10F92000D0ED070A30EE200ADFF89803D0ED0B0A7D
:10F9300030EE200AF0EE080A80EE208AFAF760FE28
:10F94000DE4890ED000A30EE080ADC4880ED000A3F
:10F95000DB480068401CDA490860FAF760FE4FF4A3
:10F960000070FEF783FFFFF7C3FFFFF7BBFF4FF405
:10F97000C072022106A8FEF75FFF0028F5D107A894
:10F98000FEF7A7FA00240698B0F5807F01D14FF466
:10F99000487400258EE00098A11807AB53F8253075
:10F9A00033F91110884206DAA01807A951F825107A
:10F9B00031F910000090A01807A951F8251031F96D
:10F9C00010000199884206DAA01807A951F82510FD
:10F9D00031F9100001900298A11807AB53F82530B7
:10F9E00033F9111040180290DDE90467A01807A947
:10F9F00051F8251031F91000A11807AB53F8253044
:10FA000033F9111010FB01F0C11730187941CDE91D
:10FA10000401521CB2F5487FBDD302984FF44871DF
:10FA200090FBF1F00290DDE904014FF448720023ED
:10FA3000FDF734FACDE9040100980C21A24A01FB3C
:10FA40000521496888479F4810EB051080ED020AA0
:10FA500001980C219C4A01FB052149688847994877
:10FA600010EB051080ED010A02980C21964A01FB6B
:10FA7000052149688847934810EB051080ED000A7E
:10FA8000DDE9040101F0C4F941EC100B01F0ECF9DF
:10FA900051EC100B00F044F900EE100A0C208A49DA
:10FAA00000FB051080688047864810EB051080ED4C
:10FAB000030A6D1C0B2DBFF42DAF07A850F82500CD
:10FAC00030F91400009007A850F8250030F9140010
:10FAD00001900020029000200021CDE904010022C5
:10FAE00098E780B52DED028BFAF78AFD744890ED0A
:10FAF000000AB8EE400A7148D0ED000A80EE808A14
:10FB0000FAF78DFDB0EE480ABDEC028B01BD80B561
:10FB1000FAF776FD6948002101606948002101601B
:10FB2000FAF77DFD01BD10B50400FAF734F9B022F3
:10FB30006449200000F0D6F8FAF73AF910BD000049
:10FB400030B5B7B0FFF7B7F8040001F0B0FA17E02E
:10FB50005E4A402105A801F0F2FA0022002105A822
:10FB600001F07EFA5A4A402105A801F0E8FA012284
:10FB7000002105A801F074FA4FF4FA70FAF7AEFF0D
:10FB800016A8FFF7D0FF002504A800F0C6FC002847
:10FB900000D00125002D17D19DED040ADFED370AB5
:10FBA000B4EE600AF1EE10FA02DB0120FEF70DFA66
:10FBB0009DED040ADFED320AB4EE600AF1EE10FAB0
:10FBC00002D50020FEF701FA206A0028C0D10020EB
:10FBD00001F05EFA012001F05BFA002D0AD02598B1
:10FBE00000F022F9CDE900013A4A402105A801F0D0
:10FBF000A6FA0EE0259800F017F9CDE90201049865
:10FC000000F012F9CDE90001334A402105A801F0C6
:10FC100096FA0022002105A801F022FA9DED190AAA
:10FC2000DDED1D0A30EE200ADDED210A30EE200A5E
:10FC3000F0EE080A80EE200A606A00280DD0606AA3
:10FC4000029010EE100A00F0EFF8CDE90001234A0F
:10FC5000402105A801F073FA0AE010EE100A00F046
:10FC6000E3F8CDE900011E4A402105A801F067FA3A
:10FC70000122002105A801F0F3F97DE701004842C7
:10FC800000002042C898FF1FA086010000400240EB
:10FC900066660A400000B0406891ED7C3F35F03F59
:10FCA0000C022B8716D9EE3F355EBA490C02E7BF2E
:10FCB0009AB1683A3B195C3F00003940C098FF1F79
:10FCC000C498FF1F1098FF1FB46401008C630100EB
:10FCD000A06301004C6301005C6301006C630100E0
:10FCE0008063010010B50446F9F772FC204610BD90
:10FCF000010040F10980F446404200F005F851F05F
:10FD000000416047010000BF09D0B0FA80F188408F
:10FD1000C91CC1F58461090501EBD021400570477C
:10FD20004FEAF17CBCF1E04C2CBFBCF5001F11E0A8
:10FD30005FEA4C0C34BFBCF17F5F2EE05FEA9C0CA5
:10FD40004FEA0C1C4FEA3C0CC10071F100414CEB36
:10FD500050707047C90241EA5051C00218BF41F0CB
:10FD6000010141F000414FEA6C50C0F10900212827
:10FD700010D240EACC7CCCF1200C11FA0CF070F1DE
:10FD80000040CCF1200C21FA0CF00CF0004C40EBC0
:10FD90000C0070474FEACC707047490011F5001F06
:10FDA00004D84FEACC10FF30C0057047C817704721
:10FDB000C0F3C7517F392CD420290DDAC1F11F0CB3
:10FDC00041004FEAC11141F0004121FA0CF0894194
:10FDD00028BF4042C9437047D1F13F0C1CD44100B9
:10FDE0004FEAC11141F0004161FA0CF021FA0CF127
:10FDF00080EA0100094244BF4FF00041002004D3D3
:10FE00004942404271F10001704701D5401E491E30
:10FE1000704700200021704709424FF0004158BF51
:10FE2000C9430020704700005FF0FF0C1CEAD0516E
:10FE300014BF614506E0C110400721F0E04101F127
:10FE40006051704779B900F0004100020AD0B0FA61
:10FE500080FC00FA0CF001F16051A1EB0C5101EBB8
:10FE6000D0214005704741020CBF40F4E0016FF023
:10FE7000000100207047000070B50400514805687B
:10FE8000002C06D0082C04D00C20F9F7D4FF002059
:10FE90002EE0288B002804D00D20F9F7CCFF00209D
:10FEA00026E01C20F9F7BFFD0600002E01D100203E
:10FEB0001EE011213000F9F704FEF460002116F174
:10FEC0001000FAF725FC4048B060FAF799FBD5F826
:10FED0003401002804D1002115F59A70FAF718FCB6
:10FEE000310015F59A70FAF719FCFAF798FB300013
:10FEF00070BD38B5040033480068002C01D10C20D7
:10FF00002CE0018B002901D00D2027E0C569FAF70C
:10FF100077FBA0682C49884203D0FAF780FB1E20AB
:10FF20001CE040F22920A8606868296801604860E8
:10FF300014F11000A863207B000705D5290014F1F7
:10FF4000100001F040F904E0290014F11000FAF764
:10FF5000E5FB04F077FDFAF762FB002032BD38B50F
:10FF600004000D0017480068002C01D11E2027E076
:10FF7000FAF746FBA0681449884203D0FAF74FFB12
:10FF80001E201DE0208B002803D1FAF748FB0F202C
:10FF900016E0002D09D0208B00280CD014F11000A1
:10FFA000FAF7DBFBFAF78BF8F5E714F11000FAF734
:10FFB000D4FBFAF784F8FAF732FB04F035FD0020A1
:10FFC00032BD00000004FF1F716B737470B44FF0FA
:10FFD000004591EA030F44BF6B4000F0AFBE00BF85
:10FFE000841A71EB030604D26E40001BB141121952
:10FFF00073414FF4001C1CEB410F34BF7CEB4306F4
:020000040001F9
:1000000084E00C0DA4EB1356362E7DDC012E43DC70
:1000100045EAC32343EA525312BFD20292025B085D
:10002000240545EAC12141EA5051D2EBC020994153
:1000300025D407D1B0FA80F610FA06F164D000207A
:10004000203608E0B1FA81F6B140C6F1200220FA6C
:1000500002F21143B0404FEAF474B4EB465434F06A
:1000600001064FEA74040AD8D6F50016760D04F09E
:100070000044F04061FA06F25040F1404840C00AA6
:1000800040EA415021F0004128BF5FEA500550F19D
:10009000000044EBD12137E045EAC323DB0A45EAFF
:1000A000C121C90AB6F120050EDD42EA0242120C56
:1000B000C5F1200603FA06F6EB4042EA06056D425A
:1000C000984161F100010DE062FA06F5F2405540F9
:1000D00063FA06FC82EA0C02F3405A406D429041FA
:1000E00061EB030111F4801F05D1641E620502D08B
:1000F0006D004041494121F48011430875F10043EE
:1001000050F1000041EB045170BC70471CEB410FF3
:1001100015D223F0004352EA43060BD04FEA4C0CB1
:10012000BCEB410F04D80C0D661E342EB7DDEBE797
:10013000801A994150EA410608BF0021E4E708BF50
:100140001CEB430F28BF6FF00001DDE7002802D150
:100150004FF482600BE00021016000218160DFF834
:10016000541341600021C1600421016100207047E7
:1001700038B5DFF844030468D4F80002002801D041
:10018000002028E01020F9F7A8FC0500002D01D17F
:10019000042020E018212800F9F793FC0021280012
:1001A000FAF7B6FADFF80C03E860FAF729FAD4F8A0
:1001B0000002002806D0FAF732FA2800F9F7A8FB67
:1001C000002008E0C4F800520FF2ED10C4F840021D
:1001D000FAF725FA002032BDF0B585B004000D0015
:1001E000DFF8D4020768002D03D100AD2800FFF727
:1001F000ADFF002C02D14FF4826043E06868DFF865
:10020000B412884202D04FF482603BE0D7F800621B
:10021000002E05D1FFF7ACFFD7F80062002E31D0D9
:10022000F068DFF89012884201D01A202AE0FAF72D
:10023000E7F9306800E00068B04206D0A042FAD189
:10024000FAF7EDF94FF482601CE028682969084349
:10025000A060DFF86002E060E8686061A868206183
:100260000020A0760020E0620020A062002114F1AE
:100270001C00FAF74DFA21003000FAF74FFAFAF7AE
:10028000CEF9002005B0F0BDF8B50400DFF8280273
:100290000068C569008B002801D00D208AE0002C81
:1002A00002D14FF4826085E0E068DFF808128842EE
:1002B00002D04FF482607DE0A06AA84202D140F2F1
:1002C000094077E0E869C68904F21A07FAF798F955
:1002D0003878002837D0A068C00510D5A06A006A19
:1002E000C08986420BD2A06AC069C089864203D207
:1002F0003100A06A00F03EFFE06A401CE0626868DE
:1003000029680160486014F11C00A863207A000786
:1003100005D5290014F11C0000F055FF04E0290068
:1003200014F11C00FAF7FAF940F22320A86004F057
:1003300089FBE068DFF87C11884207D0FAF76FF993
:100340004FF4826036E08020A076A562A06810F4A9
:100350008470B0F5807F12D114F11C0000F049FFC9
:10036000296AC98988420AD2E969C989884203D2BF
:100370000100280000F0FEFEE06A401CE062FAF78F
:100380004EF9A068800514D5FAF73AF92069296A70
:10039000C98988420BD22069E969C989884203D298
:1003A0002169280000F0E6FEE06A401CE062FAF7EE
:1003B00036F90020F2BD000070B504003E48056823
:1003C000D5F80062002E18D0F0683A49884214D15E
:1003D000FAF716F9306804E0E969816200F00EF876
:1003E0003068B04207D0817E002902D0816AA142E4
:1003F000F2D00068F5E7FAF712F970BDF8B504001D
:100400002D480568EF69002C02D14FF4826050E05E
:10041000E0682849884202D04FF4826049E0A07E1B
:10042000802802D04FF4826043E0A06AB84202D034
:100430004FF482603DE0FAF7E3F8E66A0020E062FC
:10044000207A10F0030F04D00020A0620020A076D4
:1004500026E0A08C00281FD014F11C00FAF77DF9CB
:100460000700A7623800F9F72AFEA068800510D5BA
:100470002069396AC98988420BD22069F969C9891A
:10048000884203D22169380000F074FEE06A401C03
:10049000E06204F0C9FA03E00020A0760020A06228
:1004A000002E03D03100E86900F073FEFAF7B7F8C8
:1004B0000020F2BD7874756D0004FF1F80B5002127
:1004C0005E48FCF79BFC5E4908605D4800680028B8
:1004D00001D1FF2020E05B48009000AA40F20141DA
:1004E0005748006800F0CAFE002805D0544800684C
:1004F00000F0E3FEFF200FE0002240F203415048ED
:10050000006800F0BBFE002805D04D48006800F0F0
:10051000D4FEFF2000E0002002BD7CB5060048208C
:10052000019001AA4FF481614548006800F0A6FEE1
:10053000002801D0FF207FE0002200A94048006889
:1005400000F0D5FE012190FBF1F001AA03213C4807
:10055000006800F093FE002824D10198002808D0FC
:10056000002240F20C413648006800F087FEFF2070
:1005700062E000208DF80000012200A930480068E8
:1005800000F0B5FE012190FBF1F001280CD1002212
:1005900040F20B412A48006800F070FE002805D0A8
:1005A000FF2049E0FF2047E0FF2045E002240194BE
:1005B00001AA40F20A412248006800F05FFE0028CC
:1005C00001D0FF2038E0220000A91D48006800F09B
:1005D000A0FE012190FBF1F0A04201D0FF202BE012
:1005E000002240F20C411648006800F047FE9DF8DA
:1005F000000000EE100AB8EE400A10EE100AFFF7F5
:1006000013FC04000D009DF8010000EE100AB8EE86
:10061000400A10EE100AFFF707FC00220A4BFDF714
:100620009DF822002B0000F07FFBFFF779FB00EE26
:10063000100A86ED000A002076BD0000B4AE01006D
:10064000B09BFF1F801A06000000704010B582B0FA
:1006500000900098046B002C06D02100DFF884067F
:10066000FEF7E3FC0098046313BD81B0009000988E
:10067000006ADFF874160840002801D0009908626B
:1006800001B07047F0B4B0FBF1F300241460002413
:100690005460002494600024D46000241461072B6B
:1006A00001D2FF2057E00E000024192505E0CF1BE2
:1006B000B74201D23E002C006D1E082D0CD3B3FBB7
:1006C000F5F717611769B7F5807FF5D8176907FB4C
:1006D00005F7BB4214D12C00082C3BD31069B0F5B0
:1006E000807F37D8B4F10800400850605068022875
:1006F00001D202205060082C0BD1012010600AE0CA
:100700001769B0FBF7F7B7FBF5F7B942CFD27F1AFD
:10071000CEE7506810601068201A5168401A401ED9
:1007200090601068042802D21068D06001E00420B4
:10073000D0609068401E9060D068401ED060106805
:10074000401E10605068401E50601069401E1061CD
:10075000002000E0FF20F0BC7047F0B587B0060035
:100760000C000096DFF88475DFF884550021DFF86F
:100770007405FEF739FC0121DFF87805F9F7BBFDB8
:10078000DFF87405864240F0898041F23C00C05990
:1007900050F0100041F23C01C8510098416851F4FA
:1007A000005141603200DFF854152D20F9F750FF59
:1007B000012203212D20FBF74FFF3200DFF8401507
:1007C0002E20F9F745FF012203212E20FBF744FFDD
:1007D0003200DFF82C152F20F9F73AFF0122032110
:1007E0002F20FBF739FF3200DFF814153020F9F71E
:1007F0002FFF012203213020FBF72EFF3200DFF80C
:1008000000153120F9F724FF012203213120FBF7E5
:1008100023FF3200DFF8E8143220F9F719FF012234
:1008200003213220FBF718FF00980068C00208D5AA
:100830000098016849004908016000980068C002FA
:10084000FBD400985FF0007101600098006880019F
:10085000FBD40098016851F0A04101600098006845
:10086000C001FBD501AA21002800FFF70BFF059866
:100870000499890511EB0060019910EBC1400299C0
:1008800010EB01400399081810F56C40009948607E
:100890000098DFF870144163002074E0DFF868040A
:1008A00086424FD141F23000C05950F0100041F261
:1008B0003001C8510098416851F400514160320044
:1008C000DFF838143520F9F7C3FE01220321352063
:1008D000FBF7C2FE3200DFF828143620F9F7B8FE25
:1008E000012203213620FBF7B7FE3200DFF8101497
:1008F0003720F9F7ADFE012203213720FBF7ACFECC
:100900003200DFF8FC133820F9F7A2FE01220321A0
:100910003820FBF7A1FE3200DFF8E4133920F9F7A5
:1009200097FE012203213920FBF796FE3200DFF803
:10093000D0133A20F9F78CFE012203213A20FBF76D
:100940008BFE71E7FF2025E0009911EB800100226A
:10095000C1F88028009911EB00110022C1F8802015
:10096000009911EB00110022C1F88420009911EBCD
:1009700000110022C1F88820009911EB001100221B
:10098000C1F88C20401C1028DED30098DFF87C13BF
:100990000160002007B0F0BD31B40098046854F045
:1009A000A044046000980068C001FBD50098046B67
:1009B00001258D402C430463039C0498000510EB33
:1009C000445010F58000C9B2009C14EB0114C4F827
:1009D0008000C9B2009810EB0110C0F88420C9B2A1
:1009E000009810EB01100022C0F88820C9B20098CE
:1009F00010EB01100022C0F88C20C9B2009810EB57
:100A00008100C0F880380098826A01238B401A4325
:100A100082620098C9B210EB0112D2F8802052F025
:100A20008062C9B210EB0110C0F880200098016804
:100A300031F0A041016000980068C001FBD431BCD6
:100A4000704701B481B0C9B2019810EB0110D0F821
:100A50008000030C13F00F031373430D13F0010315
:100A60005373030D13F001039373000E10F00F0086
:100A7000D073C9B2019810EB0110D0F88400106057
:100A8000C9B2019810EB0110D0F88800030E137161
:100A9000030C5371030A9371D071C9B2019810EB22
:100AA0000110D0F88C00010E1172010C5172010A74
:100AB0009172D07201988068009002B07047E0B5E2
:100AC000009001A892490CC90CC0083908384FF4AD
:100AD0007A70FAF703F8FAE780B5030000225FF0B6
:100AE00000418048FEF777FB002806D15FF0004107
:100AF0007C48FEF77EFA002000E0FF2002BD10B522
:100B000004007C48F9F736FC82480068824909688D
:100B1000884219D0200080490968804A12EB0111EF
:100B20001022F8F765FD7C480068401C7A4908608F
:100B300079480068802802D37748002101606D4819
:100B4000F9F7DFFB002003E06A48F9F7DAFBFF2042
:100B500010BD10B504006748F9F70CFC6D4800683B
:100B60006E4911EB001021001022F8F741FD694891
:100B70000068401C6749086066480068802802D306
:100B8000644800210160634800686349096888423D
:100B90000BD161480068401C5F4908605E480068EE
:100BA000802802D35C48002101605248F9F7A9FB74
:100BB0005FF000414B48FEF738FA002010BDF0B559
:100BC00087B002900024FEF776F805005148002116
:100BD000016051480021016000261FE000200190C3
:100BE000012000900C204E4900FB061083680C2069
:100BF0004B4900FB061042680C20494900FB0610D7
:100C000001780298FFF7C8FE01200C21444A01FB3D
:100C1000062191F9001088400443761C082EDDD38C
:100C20000023002221002F48FEF7D5FA0028F7D133
:100C3000FEF7F5F9070039002A48FEF7DAF9002631
:100C400002E0FDF744FE761C082EE9D20C20344960
:100C500000FB0610007837FA00F0C007F3D503AAAE
:100C60000C202F4900FB061001780298FFF7E9FEDF
:100C700003A8FFF76EFF03982A498842E3D19DF845
:100C80001000012804D0DED30328DAD01CD3DAE721
:100C90009DF81100002809D19DF8120068639DF8A5
:100CA0001300A8632020FDF7E1FD0CE09DF8110082
:100CB000012808D19DF81200E8649DF8130028650A
:100CC0001020FDF7D3FDBEE76868012803D19DF829
:100CD0001100686502E09DF81100E8634020FDF70F
:100CE000C5FDB0E7B08FFF1F070003000070044090
:100CF00000879303DC97FF1F004002404D06010070
:100D00006B0601000000101100400A401000230093
:100D1000CC4C0100D48FFF1FD88FFF1FDC8FFF1F2B
:100D2000D44C0100FFFFF11B70B44FF0004591EA75
:100D3000030C44BF6B40FFF753B900BF841A71EB3B
:100D4000030603D2001BB141121973414FF4001C7A
:100D50001CEB410F34BF7CEB430443E00C0DA4EBD0
:100D60001356352E50DC45EAC323DB0A45EAC12180
:100D7000C912B6F120050DDD63FA05F6EB4086EAEF
:100D80000305124218BF45F00105C01851F10001DA
:100D90000CD213E062FA06F5F2405540F3415A4096
:100DA000B340F3405A408018594107D349085FEADD
:100DB00030005FEA350528BF45F0010501F58011D7
:100DC000420875F1004250F1000041EB045170BC43
:100DD0004FF4001C1CEB410F38BF70470020090D79
:100DE000090570471CEB410F10D252EA43060BD0A5
:100DF000BCEB410F05D80C0DAB43661E342EB5DDA0
:100E000002E0AB438018594170BC704770BC70471A
:100E1000094240F10B80F4464942404271F1000121
:100E200000F004F851F000416047000008BFFEF7F1
:100E300069BF02460846B0FA80F150408A40C1F1CD
:100E40002001C8415040C91E01F58461090501EB2C
:100E5000D021400540EAD220520572F1004250F103
:100E6000000041F10001704751EC100B00B500F09B
:100E700003F841EC100B00BD40F2FF7C0B0D4DD090
:100E8000634566D230B421EA035141F4801103F284
:100E9000FD3C5FEA5C0C01D300184941890041EA3E
:100EA000907180004FF440140023E202D50AB1F59E
:100EB000100107D46D081DD2091B6419001849419F
:100EC000491BF7D56D080AD20919641B001849415E
:100ED000491BEFD56D08F7D301E0520817D0C018B1
:100EE00061419B1AAC4100184941801AA941F4D4D0
:100EF00052080AD0C01AA1419B186C410018494100
:100F0000801AA941E9D45208F4D15B1C6C416108F4
:100F10004FEA330001EB0C5130BC704750EA01033B
:100F2000FBD030B4B1FA81F311B9B0FA80F41B19D7
:100F30000B3BB3F120042FBF00FA04F19940C3F139
:100F4000200420FA04F438BF21439840D3F1010370
:100F50009DE76345E1D011F5801FDED850EA4101DD
:100F6000DBD0D94300F00ABA38B504000020FDF701
:100F70007EF80E20FCF72CF90020FDF76CF80E200F
:100F8000FCF726F9002519E00020FDF758F8640069
:100F90000E20FCF71DF90020FDF745F80E20FCF7A8
:100FA00017F90120FDF73FF80E20FCF711F900209A
:100FB000FDF739F80E20FCF70BF96D1C082D05DA4A
:100FC0002006E1D50120FDF73AF8E0E70120FDF722
:100FD0004EF80020FDF733F840F2C110FCF7F8F8A6
:100FE00031BD38B504000020FDF741F80E20FCF7B4
:100FF000EFF80120FDF72FF80E20FCF7E9F80025A7
:1010000019E00020FDF71BF864000E20FCF7E0F863
:101010000020FDF708F80E20FCF7DAF80120FDF7B4
:1010200002F80E20FCF7D4F80020FCF7FCFF0E209D
:10103000FCF7CEF86D1C082D05DA2006E1D501205D
:10104000FCF7FDFFE0E70120FDF711F80020FDF7B8
:1010500002F80020FCF7F3FF0E20FCF7B9F831BDD1
:1010600010B504000800110000F009F803E0207832
:10107000FFF7B7FF641C20780028F8D110BD80B5B9
:10108000402202FB0100C0B28030FFF76DFF01BDBE
:1010900010B510F001010020FFF7F1FF002403E07C
:1010A0002020FFF79EFF641C102CF9DB10BD80B5DB
:1010B0000020FCF7ACFF0120F9F789FD0120FCF7C7
:1010C000A6FF0820F9F783FD3020FFF74DFF012030
:1010D000F9F77DFD3020FFF747FF3020FFF744FF91
:1010E0003920FFF741FF1420FFF73EFF5620FFF79E
:1010F0003BFF6D20FFF738FF7020FFF735FF0C2016
:10110000FFF732FF0620FFF72FFF0120FFF72CFF2C
:101110000220F9F75CFD01BD0DB400B582B004A852
:1011200000900B005FF0FF320FF23D0103A800F0CA
:1011300078F9039900220A7006BC5DF810FB09B427
:1011400010B582B00C0005A80090130022000FF229
:10115000190104A800F065F9002C02D004990022BE
:101160000A7016BC5DF80CFB0A68531C0B6010700B
:101170007047000010B5404A1468826A52F4004279
:101180008262026D521C026500F044F803F04CFCD0
:1011900010BD80B5384A1268836A1B0412D5026DEF
:1011A000914203D2026D511A01650BE000210165E5
:1011B000816A31F400418162016AC98900F02AF82C
:1011C00003F032FC01BD70B5030002680489651CA0
:1011D000CC69E48901E0130012686D1E002D03D074
:1011E000D669F689B442F6D20A001900F9F7CCFAAA
:1011F00070BD01680089421C5FF0FF3006E0CB69DA
:10120000DB89834201D2C869C0890968521E002A5D
:10121000F5D17047F8B504000D0017480668306A2C
:10122000E169CF897FF00F0101FB05008189A1846D
:10123000E061A068022817D16068216801604860F9
:101240002000F8F73CFFF069A04206D1A08C708323
:10125000AF420FD203F0F6FB0CE0606D002809D11D
:101260002000F8F747FF05E0606D002802D120005C
:10127000F8F740FFF1BD00000004FF1F10B50300A8
:101280000020002B02D15FF0FF3015E00C00012C94
:1012900002D0022C03D005E0996811600CE01168BF
:1012A000996009E01C68E069002803D01800E36930
:1012B000984701E040F6092010BD38B50400002C25
:1012C00002D15FF0FF3011E021680869002805D1E4
:1012D0002000F8F71DFB5FF0FF3007E020000969F0
:1012E000884705002000F8F713FB280032BD10B531
:1012F000002802D15FF0FF300AE003689C69002CEF
:1013000004D12C21C1605FF0FF3001E09B69984758
:1013100010BD70B504000E0015000020002C02D195
:101320005FF0FF3029E0A169002901D0022D18DB10
:1013300023685869002804D12C20E0605FF0FF305A
:101340001BE0A069002805D06A1E711C20005B69A3
:10135000984704E02A00310020005B699847002884
:101360000BD4A169002908D0012D01DA002004E086
:10137000E16931700021A161401C70BD1FB5FCF70F
:1013800011FB212101601FBD2DE9F84304000D0070
:1013900016001F005FF00009DDF82080B8F1000F93
:1013A00004D55FF0000801E019F10109C1450ADA2E
:1013B00019F10100B042F7DAFFB22100FFB23800A4
:1013C000A8478742F0D04846BDE8F2832DE9F843AC
:1013D00004000D00160098460027012003E00120BC
:1013E0007F1C18F1010898F80010002911D000287E
:1013F0000FD0781CB042F2DA98F80090210098F8EB
:101400000000A847814501D1012000E00020C0B2C2
:10141000E6E798F80000002800D07F1E3800BDE8FD
:10142000F2832DE9F74FE4B01D000020079000245F
:10143000669810F1010F02D17FF000406690709F16
:1014400008E0641C66998C4204DA6499C0B2659A1B
:101450009047079028786D1C0100C9B225290DD04E
:10146000C0B20028EDD1079810F1010F04D15FF050
:10147000FF3067B0BDE8F08F2000FAE72878252814
:101480000AD1641C6698844205DA64992878659AC2
:10149000904707906D1CDDE720208DF8100000209C
:1014A0008DF80C00042000210A915FF0000E00214D
:1014B00000228DF80E205FF0000C00238DF8113013
:1014C00000238DF80F3000238DF80D3000238DF8A8
:1014D00012300023002604E05FF0010ECDF828E072
:1014E0006D1C2A78002A22D0F6B2002E1FD12A784D
:1014F000202A11D0232A12D02B2A09D02D2AEBD052
:10150000302A12D15FF0300E8DF810E06D1CE8E744
:101510005FF0010C6D1CE4E701216D1CE1E75FF059
:10152000010E8DF80EE06D1CDBE70126D9E70026E1
:1015300006962A782A2A0ED13E6806963F1D6D1C13
:101540000DE0069A0A2695F800E006FB02E2B2F1E9
:10155000300606966D1C2A78303A0A2AF1D35FF0DD
:10156000FF362A782E2A15D100266D1C2A782A2AC1
:101570000CD13E683F1D01236D1C0BE00A222B7825
:1015800002FB0632B2F130066D1C01232A78303A94
:101590000A2AF3D30DF12C0895F800E06D1CCDF864
:1015A00014E0BEF1000F11D1641C6698844204DA85
:1015B00064992520659A90470790079810F1010FCC
:1015C00002D15FF0FF3054E7200052E7059A4C2A21
:1015D00024D0682A02D06C2A10D026E0002095F88A
:1015E00000E0CDF814E06D1C059A682A05D10120B1
:1015F00095F800E0CDF814E06D1C16E0022095F897
:1016000000E0CDF814E06D1C059A6C2A05D103208A
:1016100095F800E0CDF814E06D1C06E0042095F884
:1016200000E0CDF814E06D1CFFE75FF0000E5FF006
:10163000000A5FF0000B059A432A3CD0442A5CD094
:10164000452A00F0AC82462A00F06582472A00F065
:101650002482492A51D04E2A00F019824F2A00F0E4
:101660006581502A00F0B081532A3CD0552A46D0DB
:10167000582A00F0B781632A1DD0642A3DD0652A1C
:1016800000F08D82662A00F04682672A00F005820B
:10169000692A32D06E2A00F0FA816F2A00F0468162
:1016A000702A00F09381732A1DD0752A27D0782ADA
:1016B00000F09D81B0E238688DF82C003F1D9DF848
:1016C0002C00002804D11BF1010B01208DF8120021
:1016D00000208DF82D00002620208DF8100000201D
:1016E0008DF80E00ACE2D7F800803F1D20208DF869
:1016F000100000208DF80E00A2E25FF0010A012E1A
:1017000002DB01238DF811305FFA8AFABAF1000F7B
:101710006DD0032835D1FF1D37F00707D7E9002327
:10172000CDE908230837DDE90823002B03D1002A7F
:1017300001D1012300E000238DF80D30DDE90823FD
:10174000002B0DDC01DB002A0AD22D218DF80C10B4
:10175000DDE90823524273EB4303CDE9082391E00E
:101760005FFA8CFCBCF1000F03D02B218DF80C101C
:1017700088E0C9B2002900F0858020218DF80C1086
:1017800080E0002803D1B7F900903F1D0EE001284A
:1017900003D197F900903F1D08E0022803D1D7F844
:1017A00000903F1D02E0D7F800903F1DB9F1000FF7
:1017B00001D1012300E000238DF80D30B9F1000FB5
:1017C00005D52D218DF80C10D9F100095AE05FFAEA
:1017D0008CFCBCF1000F03D02B218DF80C1051E0D4
:1017E000C9B200294ED020218DF80C104AE0002803
:1017F0000BD1B7F800903F1DB9F1000F01D10121C5
:1018000000E000218DF80D103CE001280BD197F885
:1018100000903F1DB9F1000F01D1012100E000212E
:101820008DF80D102EE002280BD1D7F800903F1D47
:10183000B9F1000F01D1012100E000218DF80D1058
:1018400020E0032813D1FF1D37F00707D7E9002355
:10185000CDE908230837DDE90823002B03D1002A4E
:1018600001D1012100E000218DF80D100AE0D7F828
:1018700000903F1DB9F1000F01D1012100E00021CE
:101880008DF80D105FF0000A03283AD10BE0DDE976
:101890000823DFF84809DFF8481910185941CDE945
:1018A00008011AF1010ADDE908010029EFDB01DC7A
:1018B0000028ECD35FFA8EFECDF800E0142318F177
:1018C0000102DDE9080100F00DFC98F801001AEBB7
:1018D000000088F8010098F801003A2808DB98F821
:1018E00001000A3888F80100312088F8000019E06A
:1018F00018F1010816E0DFF8EC0810EB09091AF1FD
:10190000010AB9F1000FF6D45FFA8EFE73460A227F
:101910004146484600F092FB98F800001AEB0000A0
:1019200088F8000000208DF80E0089E1012E02DB0E
:1019300001218DF8111003281DD1FF1D37F0070775
:10194000D7E90001CDE908010837DDE908010029E0
:1019500003D1002801D1012000E000208DF80D0006
:101960005FFA8EFECDF800E016234246DDE908015D
:1019700000F0B8FB24E0002803D1B7F800903F1D29
:101980000EE0012803D197F800903F1D08E00228DF
:1019900003D1D7F800903F1D02E0D7F800903F1D1B
:1019A000B9F1000F01D1012000E000208DF80D00F9
:1019B0005FFA8EFE73460B224146484600F03EFB1E
:1019C00003208DF80F003BE15FF0010E5FF0000A8D
:1019D00038683F1D5FFA8EFE73460822414600F0CC
:1019E0002DFB2DE15FF0010E01218DF80F10012E6E
:1019F00002DB01218DF811109DF80F10491C8DF8A4
:101A00000F1003281DD1FF1D37F00707D7E900018C
:101A1000CDE908010837DDE90801002903D10028D4
:101A200001D1012000E000208DF80D005FFA8EFE4C
:101A3000CDF800E010234246DDE9080100F052FB3A
:101A400024E0002803D1B7F800903F1D0EE00128E4
:101A500003D197F800903F1D08E0022803D1D7F882
:101A600000903F1D02E0D7F800903F1DB9F1000F34
:101A700001D1012000E000208DF80D005FFA8EFEFC
:101A8000734608224146484600F0D8FAD8E0D7F815
:101A900000803F1DC8F80040DCE4DBB2002B00D121
:101AA0000626042806D1FF1D37F0070797ED000B27
:101AB000083705E0FF1D37F0070797ED000B0837E3
:101AC0000598C0B20290701E01909DF80E00009023
:101AD0000B00DBB26246D2B204A913A800F04BFEA1
:101AE00081460DF14C0898F800002B2805D12B20D9
:101AF0008DF80C0018F1010808E098F800002D2876
:101B000004D12D208DF80C0018F1010800208DF86B
:101B10000E00002694E0DBB2002B00D10626002E3A
:101B200000D10126042806D1FF1D37F0070797EDE5
:101B3000000B083705E0FF1D37F0070797ED000B96
:101B40000837DFF8A40680ED000B0598C0B20290BC
:101B500001969DF80E0000900B00DBB26246D2B2F7
:101B600004A913A800F080FD81460DF14C0898F8F7
:101B700000002B2805D12B208DF80C0018F101084E
:101B800008E098F800002D2804D12D208DF80C00D5
:101B900018F1010800208DF80E00002650E0DBB29D
:101BA000002B00D10626042806D1FF1D37F00707B9
:101BB00097ED000B083705E0FF1D37F0070797ED9D
:101BC000000B08370598C0B2029001969DF80E00F0
:101BD00000900B00DBB26246D2B204A913A800F059
:101BE000BFFC81460DF14C0898F800002B2805D168
:101BF0002B208DF80C0018F1010808E098F800007F
:101C00002D2804D12D208DF80C0018F1010800209A
:101C10008DF80E00002613E0641C6698844204DAF6
:101C200064990598659A90470790079810F1010FFD
:101C300002D15FF0FF301CE420001AE41BF1010B1D
:101C40001BF808000028F9D10698002801D50020CB
:101C50000690002E01D5002608E00598732802D0D2
:101C60000598532802D15E4500DAB3465FF0000ABA
:101C70000698304300284FD09DF8110000280BD162
:101C8000002E09D05E4507DA0BA8804503D1BBEBD7
:101C9000060010EB0808B3469DF8110000281FD07D
:101CA0000698864219DAB34503DA0698B0EB060ABD
:101CB00002E00698B0EB0B0A9DF80D00002815D144
:101CC0009DF80E00002811D09DF80F0003280DD1BB
:101CD000B3450BDA1AF1010A08E05FF0000A05E0EB
:101CE0000698002802D00698B0EB0B0A9DF80C006D
:101CF000002801D0BAF1010A9DF80E0000280BD08F
:101D00009DF80D00002807D1BAF1010A9DF80F00D7
:101D1000032801DABAF1010ABAF1000F01D55FF028
:101D2000000A0A98002840F001819DF8110000285F
:101D30005BD0CDF800A020236698021B65996498BB
:101D4000FFF722FB04199DF80C002B2807D09DF803
:101D50000C002D2803D09DF80C0020280AD101206A
:101D600000909DF80C306698021B65996498FFF707
:101D70000BFB04199DF80E0000282AD09DF80D00D9
:101D8000002826D19DF80F00012802D0022809D092
:101D900011E0D2A36698021B65996498FFF716FBC1
:101DA000041916E0CEA36698021B65996498FFF7A4
:101DB0000DFB04190DE0B6EB0B00012809DA012038
:101DC000009030236698021B65996498FFF7DCFA4F
:101DD0000419B6EB0B00009030236698021B65993E
:101DE0006498FFF7D1FA0419F9E09DF81000302843
:101DF0004DD19DF80C002B2807D09DF80C002D2804
:101E000003D09DF80C0020280AD1012000909DF8F5
:101E10000C306698021B65996498FFF7B5FA0419AF
:101E20009DF80E00002826D09DF80D00002822D134
:101E30009DF80F00012802D0022809D011E0A7A3C5
:101E40006698021B65996498FFF7C0FA041912E0BE
:101E5000A3A36698021B65996498FFF7B7FA041963
:101E600009E00120009030236698021B6599649870
:101E7000FFF78AFA0419CDF800A09DF81030669893
:101E8000021B65996498FFF77FFA0419A7E0CDF863
:101E900000A09DF810306698021B65996498FFF7C2
:101EA00073FA04199DF80C002B2807D09DF80C003C
:101EB0002D2803D09DF80C0020280AD10120009085
:101EC0009DF80C306698021B65996498FFF75CFAE0
:101ED00004199DF80E00002800F081809DF80D0087
:101EE00000287CD19DF80F00012802D0022809D0DB
:101EF00011E07AA36698021B65996498FFF766FA69
:101F000004196CE076A36698021B65996498FFF744
:101F10005DFA041963E00120009030236698021BEB
:101F200065996498FFF730FA041958E09DF80C00A1
:101F30002B2807D09DF80C002D2803D09DF80C000D
:101F400020280AD1012000909DF80C306698021BD1
:101F500065996498FFF718FA04199DF80E00002897
:101F60002ED09DF80D0000282AD19DF80F000128E1
:101F700002D0022809D011E058A36698021B659987
:101F80006498FFF723FA04191AE055A36698021B18
:101F900065996498FFF71AFA041911E09DF8110089
:101FA000002803D0B6EB0B00002809D501200090D3
:101FB00030236698021B65996498FFF7E5F90419C8
:101FC0009DF8110000280AD0B6EB0B0000903023DA
:101FD0006698021B65996498FFF7D6F904191BF1FE
:101FE000010B6698001B584502DA6698B0EB040BAB
:101FF0009DF8120000280AD00120009098F80030C7
:102000005A4665996498FFF7BFF9041906E04346FC
:102010005A4665996498FFF7D9F904190A98002877
:102020003FF418AACDF800A020236698021B6599FA
:102030006498FFF7A9F90419FFF70CBA7FB40024DC
:102040008DF800400B2A12D1012406E010F007039E
:10205000303300AD6355C010641CA242F6DA9DF81F
:102060000B0010F033008DF80B00140025E00A2A55
:102070000FD10124A242F8DB0A2390FBF3F503FB06
:102080001503303300AD63550A2390FBF3F0641C55
:10209000F0E7012407E010F00F05544EAD5D00AEEF
:1020A000A5550011641CA242DFDB002BF3D010F019
:1020B0000F054F4EAD5DF2E7641E00A8205C30288E
:1020C000FAD0002C06D1641C04E000A8205C087043
:1020D000641E491C002CF8D57FBC70473078000086
:1020E000305800002DE9F04788B004000D001600BC
:1020F0001F0000208DF80000162F18D15FF0010A94
:102100000BE014F00700303000A90AF80100E408E1
:1021100044EA4574ED101AF1010A5745F1DA9DF8C9
:10212000160010F031008DF81600BA463DE0142F6D
:102130001FD15FF0010A5745F7DB200029005FF04F
:102140000A085FF00009040042464B46FAF7A6FE73
:1021500008FB1040303000A90AF8010020002900D7
:102160000A220023FAF79AFE04000D001AF1010A70
:10217000E1E75FF0010A10980CE014F00F011B4A30
:10218000895C00AA0AF80210240944EA05742D119A
:102190001AF1010A5745C8DB0028EED014F00F01F0
:1021A000134A895CEDE7BAF1010A00A81AF80000A9
:1021B0003028F8D0BAF1000F09D11AF1010A06E06F
:1021C00000A81AF800003070BAF1010A761CBAF1C2
:1021D000000FF5D508B0BDE8F087000000009C585E
:1021E0004C491FF2003665C40805FF1F9C620100C0
:1021F000886201002DE9F84F2DED028B2DED020BC9
:1022000082B081468A469B460026B9F1000F01D56F
:102210005FF00009B9F1990F01DB5FF09809002424
:10222000DDF8408045460398002808D5012010704D
:10223000DDE9020191F00041CDE9020101E0002059
:1022400010700398C0F30A5040F2FF7188420BD11E
:1022500003980003000B02990843002804D1692069
:1022600088F8000040460AE10398C0F30A5040F2A3
:10227000FF7188420DD103980003000B02990843B7
:10228000002806D0002010706E2088F8000040461C
:10229000F5E00398400040080299084300281AD14D
:1022A0001198C0B2652802D0C0B2452803D10120E0
:1022B000CAF8000002E00020CAF80000002003E095
:1022C000302100F80810401C4845F9D3002009F8D7
:1022D00008004046D3E06C489DED020B80ED000BFA
:1022E00000A89DED020B00F075FB8DED020BDDE902
:1022F000002300200021FBF7F5F931D008F29A07FE
:102300001EE0DDE900010022604BFBF727FA604A7E
:10231000604BFEF709FD41EC100B00A800F05AFBE2
:1023200053EC102B00205949FBF780F841EC100BBF
:102330007F1E51EC100B00F0ADFB30303870641C88
:10234000DDE9002300200021FBF7CCF9D9D118F1F9
:102350009A0087421ED2387828707F1C6D1CF6E7E1
:10236000DDE902010022002300F0BAFB12D202E0F4
:102370008DED028B641EDDE9022300204349FBF74B
:1023800055F841EC180B51EC180B0022424B00F0B1
:10239000BFFBEDD319EB08075FFA8BFBBBF1000F16
:1023A00023D12600012E0ADB002E1ED018F1990041
:1023B00087421AD27F1C761EF6E77F1E761C002EFF
:1023C00001D0B845F9D3002E0FD5002003E030210D
:1023D00000F80810401C4845F9D30020CAF8000056
:1023E000002009F80800404649E0CAF8004013E020
:1023F000DDE9022300202549FBF718F841EC100B1A
:1024000000A800F0E7FA8DED020BDDE9000100F015
:1024100041FB303028706D1CAF42E9D25FFA8BFB74
:10242000BBF1000F06D1002E04D0302088F89900AF
:10243000404624E03D003878401D387003E07F1EA0
:102440003878401C387038783A2815DB30203870DE
:10245000B845F4D331203870DAF80000401CCAF8CF
:1024600000005FFA8BFBBBF1000FECD1A84501D255
:10247000302028706D1CE6E700202870404604B02C
:10248000BDEC028BBDE8F28F1005FF1F0000244059
:10249000B81E85EB51B89E3F0000F03F30B42025B8
:1024A000029C002C03D02D220270401C0CE0D2B202
:1024B000002A03D02B220270401C05E0DBB2002B67
:1024C00002D020220270401C039AD2B2472A05D0C3
:1024D000D2B2452A02D0D2B2462A00D100250A78CB
:1024E000692A0CD115F149010170401C15F14E010A
:1024F0000170401C15F146010170401C0EE0097886
:102500006E290BD115F14E010170401C15F14101EE
:102510000170401C15F14E010170401C002101703A
:1025200030BC704730B4002800D54042642801DB3D
:10253000032200E0022201240CE00A2390FBF3F5C1
:1025400003FB15030A2590FBF5F0E4B2151B3033AD
:102550006B54641CE4B2A242EFDA100030BC704746
:102560002DE9F043ABB005000E0017009846349CEF
:10257000E4B2019404A80090012302AA03A93398AD
:10258000401CFFF737FEA9460178692902D001787F
:102590006E290FD1E4B201949DF8081000914346D2
:1025A000DBB23A00D2B201004846FFF777FF2020A5
:1025B000307054E09DF80810002905D02D2189F8CD
:1025C000001019F1010912E0FFB2002F05D02B21F4
:1025D00089F8001019F1010909E05FFA88F8B8F1EB
:1025E000000F04D0202189F8001019F101090178A9
:1025F00089F80010401C19F101090178002902D165
:10260000329900290BD02E2189F8001019F1010907
:1026100005E0017889F80010401C19F101090178E2
:102620000029F6D189F8004019F101090398401EEC
:10263000002805D42B2089F8000019F1010904E0D5
:102640002D2089F8000019F1010949460398401E20
:10265000FFF768FF10EB0909002089F80000B9EBCB
:1026600005002BB0BDE8F0832DE9F043ABB00500C9
:102670000F00904699462E0033989B2800DB9A2045
:10268000349CE4B2019404A90091002302AA03A996
:10269000FFF7B0FD01000878692802D008786E289D
:1026A0000ED1E4B201949DF8080000904B46DBB2D5
:1026B0004246D2B23000FFF7F1FE2020387056E0DB
:1026C0009DF80800002803D02D203070761C10E003
:1026D0005FFA88F8B8F1000F03D02B203070761C19
:1026E00007E05FFA89F9B9F1000F02D020203070BD
:1026F000761C039801281BDA30203070761C2E20BF
:102700003070761C02E030203070761C0398421C3A
:1027100003920028F7D40878491C3070761CC0B2A8
:102720000028F8D1761E22E008783070491C761C0B
:102730000878002804D00398421E03920028F3D1A1
:102740000878002802D13298002802D02E2030705C
:10275000761C0878002808D00878491C3070761C50
:10276000C0B20028F8D1761E01E000203070701B46
:102770002BB0BDE8F0832DE9F0472DED028BACB016
:102780000500B0EE408AF0EE608A89461700984650
:10279000389CA41EDDF8DCA0E4B2019404A80090EB
:1027A000012302AA03A91AF10100B0EE480AF0EED3
:1027B000680AFFF71FFD2E000178692902D0017811
:1027C0006E2910D1E4B201949DF80810009143469F
:1027D000DBB23A00D2B201003000FFF75FFE2020EA
:1027E00089F80000EFE00399491E11F1040F18DB8E
:1027F0000399491E514514DABAF19B0F01DB5FF0D2
:102800009A0AA01EC0B2019004A80090002302AA58
:1028100003A95046B0EE480AF0EE680AFFF7EAFC5A
:10282000641C3699C9B200292DD1002200E0521C47
:10283000135C002BFBD1521E00E0521E002A05D46F
:10284000135C302B02D1039B9A42F6D1002A03D4A9
:10285000135C302B00D1521E12F1010F09D1E4B2EA
:10286000652C02D0E4B2452C0AD13022027000223D
:1028700006E0135C303B0A2B02D3521C3023135466
:10288000121800235370E4B2652C02D0E4B2452C38
:1028900041D19DF80820002A03D02D223270761CE9
:1028A0000EE0FFB2002F03D02B223270761C07E01F
:1028B0005FFA88F8B8F1000F02D020223270761C3F
:1028C00002783270401C761C0278002A02D1C9B20C
:1028D000002907D02E213170761C03E00178317079
:1028E000401C761C01780029F8D13470761C0398BE
:1028F000401E002803D42B203070761C02E02D20CF
:102900003070761C31000398401EFFF70BFE8619CD
:102910000020307057E09DF80820002A03D02D22B7
:102920003270761C0EE0FFB2002F03D02B223270E3
:10293000761C07E05FFA88F8B8F1000F02D0202279
:102940003270761C039A012A1EDA30213170761C0F
:102950000178002906D02E213170761C02E030214A
:102960003170761C03994A1C03920029F7D4017830
:10297000401C3170761CC9B20029F8D1761E22E0C5
:1029800002783270401C761C0278002A04D0039A28
:10299000531E0393002AF3D10278002A02D1C9B250
:1029A000002902D02E213170761C0178002908D030
:1029B0000178401C3170761CC9B20029F8D1761E0E
:1029C00001E000203070701B2CB0BDEC028BBDE824
:1029D000F087000010B5044651EC100B00F006F82B
:1029E0002260636041EC100B10BD0000C1F30A5C73
:1029F00040F2FE32BCEB020CCCBFDCF1350237E01A
:102A0000BCF115031ADA9B415B0543FA0CF30B404A
:102A10000022994319D0B1FA81FCACF10B0C414072
:102A200000FA0CF0CCF1200C61FA0CF14140CCF131
:102A3000210CCCEB135C01EB0C5170476FF00002E2
:102A4000DA4020EA02020B469043F8B1B0FA80FC6B
:102A50000CF1150C0021BCF11F0FE0D9ACF12001E5
:102A60008840CCEB1351491E00EB01510020704708
:102A7000BCF1350F03DA01F00043002270470B462A
:102A800002464FF4001C1CEB430F02D803F0004138
:102A900000207047F446400D40EAC120490006D2AC
:102AA00000F00EF8004248BF6FF00040604700F0B1
:102AB00007F84FF0004188428CBF0846404260470B
:102AC00040F00040490DA1F58061491C05D4D1F1C9
:102AD0001F0154BFC840C01770474FF00000704737
:102AE0004FF4001C1CEB410F94BF1CEB430F09E09B
:102AF00041EA030C50EA4C0C52EA0C0C03D28B4214
:102B000008BF8242704714BF99429042704700004C
:102B10004FF4001C1CEB410F94BF1CEB430F09E06A
:102B200041EA030C50EA4C0C52EA0C0C03D29942D5
:102B300008BF9042704714BF8B428242704700002A
:102B400081B01148006800900098D0F8C812491C64
:102B5000C0F8C8120029F7D10098D0F8CC12491C4F
:102B6000C0F8CC120029EFD10098D0F8D012491C3F
:102B7000C0F8D0120029E7D10098D0F8D412491C2F
:102B8000C0F8D412E0E700BF0004FF1F1049096835
:102B900080B2002811D0022815D011D3042806D005
:102BA00002D3052806D011E0D1F89C020FE0D1F83D
:102BB000A0020CE0D1F8A40209E0C869406F06E069
:102BC000C869806F03E0C869C06F00E000207047EB
:102BD0000004FF1F0EB430B582B0040005AD012023
:102BE000FFF7D4FF009523005FF0FF320249FEF7A4
:102BF00018FC36BC5DF810FB014901002DE9F34FCC
:102C000081B02DED028B84B0140000260025002732
:102C100001E00098C719089800780899491C0891A4
:102C2000002800F0D6825FF0000A202801D0092891
:102C300010D100A908A800F001FB002801D128004C
:102C4000C8E2002200A907A800F0CEFA0028E0D1CF
:102C50002800BFE225280FD08046002200A907A83F
:102C600000F0C2FA804501D02800B3E20798401C6A
:102C700007900098C719CEE75FF000085FF0000AE0
:102C800003200290012003905FF0000900A908A82A
:102C900000F0D4FA002801D128009BE208980078BF
:102CA0002A2805D118F101080898401C08900078DE
:102CB00000A908A800F0C2FA002801D1280089E282
:102CC000089800785FF0000A08E00A2101FB0A007A
:102CD000B0F1300A0898401C08900078B0F130013B
:102CE0000A29F2D300A908A800F0A8FA002801D107
:102CF00028006FE2089800780899491C0891B0F103
:102D000061011A2900D2203848280FD101200290F1
:102D100000A908A800F092FA002801D1280059E281
:102D2000089800780899491C089134E04C280FD184
:102D30000020029000A908A800F080FA002801D124
:102D4000280047E2089800780899491C089122E079
:102D50005A280FD10220029000A908A800F06EFAAC
:102D6000002801D1280035E2089800780899491C0C
:102D7000089110E04D280ED10320029000A908A868
:102D800000F05CFA002801D1280023E208980078BE
:102D90000899491C0891B0F161011A2900D2203824
:102DA000422800F0E380432800F0B481442869D031
:102DB000452800F0E081462800F0DD81472800F03A
:102DC000DA81492810D04E2800F0CA814F2800F03F
:102DD000AF80502877D0532800F05B81552800F051
:102DE000FA8058286FD0F2E1002200A907A800F06D
:102DF000FBF907990978302944D17F1C0798401CBA
:102E00000790BAF1000F05D0BAF1010ABAF1010F2B
:102E1000C0F2198107980078782803D007980078C5
:102E200058280ED15FF0100B0798401C07907F1CAC
:102E3000BAF1000F25D0BAF1010ABAF1010F20DA78
:102E400001E107980078622803D0079800784228AB
:102E50000ED15FF0020B0798401C07907F1CBAF15F
:102E6000000F0ED0BAF1010ABAF1010F09DAEAE057
:102E70005FF0080B0798007800F014FA002800F0C3
:102E8000E280AFE05FF00A0B00200090002200A972
:102E900007A800F0A9F92D2840F09B800098C719D9
:102EA0005FF0FF3003900798401C07907F1CBAF139
:102EB000000F00F090800098BAEB000ABAF1010F01
:102EC00080F28980BFE05FF0100B002200A907A804
:102ED00000F08AF907990978302928D10798401C11
:102EE00007907F1CBAF1000F05D0BAF1010ABAF1C0
:102EF000010FC0F2A88007980078782803D00798BF
:102F0000007858280CD10798401C07907F1CBAF114
:102F1000000F0CD0BAF1010ABAF1010F07DA92E002
:102F20000798007800F0C6F9002800F08C8059E07E
:102F30005FF0080B002200A907A800F055F90799D7
:102F40000978302911D17F1C0798401C0790BAF1ED
:102F5000000F04D0BAF1010ABAF1010F73DB079830
:102F6000007800F09FF900286DD03BE05FF0020B85
:102F7000002200A907A800F037F90799097830293D
:102F800026D10798401C07907F1CBAF1000F04D08F
:102F9000BAF1010ABAF1010F55DB079800786228EF
:102FA00003D00798007842280CD10798401C07905E
:102FB0007F1CBAF1000F0BD0BAF1010ABAF1010F70
:102FC00006DA40E00798007800F074F900283AD05B
:102FD00008E00098C7195FF00A0B002200A907A8B3
:102FE00000F002F95FF00009079800780099CF1906
:102FF000BAF1000F06D00099BAEB010ABAF1010F3D
:10300000FFF609AE5946C0B200F02DF910F1010FDC
:1030100001D12800DEE059460798007800F023F936
:1030200010F1010F0FD00799491C07917F1C10F078
:103030007F000BFB0909BAF1000FECD0BAF1010ACD
:10304000BAF1010FE7DA5FFA88F8B8F1000F1FD183
:10305000039800FB09F920680190241D02980028BC
:1030600005D002280BD006D303280CD00FE001981E
:10307000C0F800900BE00198A0F8009007E00198DC
:1030800080F8009003E00198C0F80090FFE76D1C05
:10309000C1E500200090002200A907A800F0A4F8D4
:1030A0000098C7195FFA88F8B8F1000F01D12668B7
:1030B000241DBAF1000F05D00098BAEB000ABAF14E
:1030C000010F1EDB0798007800281AD00799491CC9
:1030D00007917F1C08990978884203D10898401C01
:1030E00008900EE05FFA88F8B8F1000F01D1307057
:1030F000761CBAF1000FE5D0BAF1010ABAF1010F5E
:10310000E0DA5FFA88F8B8F1000F02D16D1C0020F8
:10311000307080E5BAF1000F01D15FF0010A5FFA6B
:1031200088F8B8F1000F0FD12668241D0CE05FFA73
:1031300088F8B8F1000F03D1079800783070761C3A
:103140000798401C07907F1C5046B0F1010A0128E7
:10315000EDDA5FFA88F8B8F1000F00D16D1C5AE57E
:103160005FFA88F8B8F1000F04D120680190241D9F
:10317000019807604FE501A9079800F0ADF8B0EE9F
:10318000408AF0EE608A53EC182B00201449FAF7BD
:10319000A9FA06D053EC182B00201249FAF7A2FA2C
:1031A00001D1280016E00198079020680190241DA5
:1031B0000298002803D1019880ED008B05E051ECC6
:1031C000180BFCF7ADFD019908606D1C23E5280084
:1031D00000E0280004B0BDEC028BBDE8FE8F0000CB
:1031E0000000F07F0000F0FF10B403681B7800249B
:1031F0000C60DBB2202B0ED0DBB2092B0BD0DBB284
:103200000A2B08D0DBB20D2B05D0DBB20B2B02D082
:10321000DBB20C2B0ED103685B1C03601B780C68BF
:10322000641C0C60002AE4D0521E002AE1D1180070
:10323000C0B201E01800C0B210BC704700220A60A2
:103240000268127806E00268521C026012780B686D
:103250005B1C0B60D2B2202AF5D0D2B2092AF2D080
:103260001000C0B27047C0B2B0F161021A2A00D299
:103270002038C0B2B0F141021A2A07D23738491EAD
:10328000C0B281420CD25FF0FF300AE0C0B2B0F1B0
:1032900030020A2A01D23038F1E75FF0FF3000E057
:1032A000C0B27047C0B23038082801D2012000E017
:1032B00000207047C0B2B0F130010A2908D3C0B273
:1032C000B0F16101062903D3C0B24138062801D20A
:1032D000012000E00020704780B5002200F0B6F821
:1032E00041EC100B01BD00002DE9F14D81B0064607
:1032F0002DED028B88B0884617461D460BA800F0BE
:10330000A7F804460DB10021296020F0080001282B
:1033100035D10220009004AB0B994246304600F0B4
:1033200031F9060003D10020CDE902001FE0059825
:10333000FCF7DEFCCDE90201022E18DB0DF11808C6
:10334000761E9FED3D8BDDE9022351EC180BFAF759
:103350006DF8824658F8040B8B46FCF7C9FC5246C0
:103360005B46FDF7E1FCCDE90201761EEBD1049846
:10337000C219DDE902012B46F9F764FF44E0022897
:1033800037D1009004AB0B994246304600F0D6F995
:10339000060003D10020CDE902001FE00598FCF7EC
:1033A000A7FCCDE90201022E18DB0DF11808761EEC
:1033B0009FED238BDDE9022351EC180BFAF736F869
:1033C000824658F8040B8B46FCF792FC52465B464B
:1033D000FDF7AAFCCDE90201761EEBD1049902A803
:1033E000FAF7F6F8DDE902012B463A46F9F72AFF2B
:1033F0000AE0032802D10020134905E0042806D181
:103400004FF0FF306FF00041CDE9020102E00020F3
:10341000CDE90200200743BFDDE9020181F0004150
:1034200041EC100B9DED020B08B051EC100BBDEC04
:10343000028BBDE8FC8D00000000000065CDCD4191
:10344000000000000000B0410000F07F00234BE7C7
:103450002DE9F84304460D462668002700E0761C57
:10346000307800F079FA0028F9D130782D280CBF97
:1034700008272B2800D1761C307840F020016E29D7
:1034800029D1761C16F8010B40F02000612802BFFC
:1034900016F8010B40F020006E2802D026680027A5
:1034A0004CE0B046042798F80000282846D118F8C8
:1034B000019F484600F046FA0028F8D1A9F13000F3
:1034C0000A28F4D398F800005F28F0D0292835D1D5
:1034D00008F1010632E0692933D1761C16F8010B98
:1034E00040F020006E2802BF16F8010B40F02000CB
:1034F000662802D02668002720E0304647F0030700
:10350000017841F02001692902BF10F8011F41F044
:1035100020016E2912D110F8011F41F02001692904
:1035200002BF10F8011F41F02001742906D110F8E4
:10353000011F41F02001792908BF461CF5B12E601A
:103540001CE0302802BF707840F02000782813D1AA
:10355000B01C01782E2908BF401C0078A0F1610141
:10356000062921BFA0F14101062930380A2803D2DB
:10357000B61C47F0020701E047F001072660384615
:10358000BDE8F2832DE9F04F8DB08046169800EB30
:10359000C00A0D4691461C464FF0000BBAF12E0FA3
:1035A000A8BF4FF02D0AC4F800B0C4F804B000263C
:1035B00001E06D1C012628783028FAD0002700A8E9
:1035C00004E02168491C21606D1C01262978A1F1C5
:1035D00030020A2A09D300F0E6F9406A2978007817
:1035E000814208BF6D1C77B90AE0BA45E9DB303982
:1035F00039547F1CE8E72068401E20606D1C0126BE
:1036000028783028F7D02878A0F130010A2912D381
:10361000BA4525DA00A81AF80000052806DB00A83C
:10362000504410F8011C491C00F8011C5746206842
:10363000401C206014E0BA4506DB00A930387854FD
:103640007F1C2068401E20606D1C0126DBE700A85F
:10365000381810F8010C48B92068401C20607F1E03
:10366000012FF4DA17B98DF800B00127002E58D0D9
:10367000092297FBF2F2C7F1090002EBC20212180D
:10368000092092FBF0F0002100EBC000101A0DD0D1
:103690004FF0010B0AE054F82B30085C03EB830376
:1036A00000EB430044F82B00521C491CB9420BDAD2
:1036B000092392FBF3F303EBC30300A8D31AEAD167
:1036C000085C0BF1010BEDE7287840F0200065283D
:1036D00027D1284615F8011F2B2916BF2D2915F8CB
:1036E000011B2B214FF0000C0023134A09E09342E9
:1036F00004DA03EB83070EEB4703303B6D1C4FF0FE
:10370000010C95F800E0AEF130070A2FEFD32D2918
:1037100008BF5B42216859182160BCF1000F08BF47
:103720000546B9F1000F03D006B1A846C9F80080DC
:1037300058460DB0BDE8F08F00E1F5052DE9F14FD9
:103740008AB00E461498C0EBC00B90461D464FF051
:10375000000ABBF1240FA8BF4FF0230BC5F800A04F
:10376000C5F804A0002701E0761C01273078302836
:10377000FAD00FF2A010002400900DF1040904E02B
:103780002868401C2860761C0127317816220FF229
:10379000841000F021F950B1A345F1DB0099401AE3
:1037A0000FF28811405C04F80900641CEBE700F09C
:1037B000FAF8406A31780078814208BF761C44B933
:1037C00004E02868401E2860761C012730783028E5
:1037D000F7D0317816220FF23C1000F0FDF880B1DE
:1037E000A3450BDB0FF22C11401A0FF24011405C85
:1037F00001A96054641C2868401E2860761C0127BB
:10380000E7E7A34519DA01A81BF80000082806DB42
:1038100001A8584410F8011C491C00F8011C5C4622
:103820002868401C286008E001A8201810F8010C46
:1038300048B92868401C2860641E012CF4DA14B9C9
:103840008DF804A00124286880002860002F53D040
:10385000072294FBF2F2C4F10701C2EBC202511835
:10386000072291FBF2F20020C2EBC2028A1A06D0B4
:103870004FF0010A03E045F82A20491C401CA042F1
:103880000FDA072391FBF3F310F80920C3EBC3030E
:10389000CB1A0EBF0AF1010A55F82A3002EB0312C7
:1038A000E9E7307840F02000702825D1304616F83E
:1038B000011F2B2916BF2D2916F8011B2B210022D1
:1038C0000023134C09E0A34205DA03EB83020CEB5F
:1038D0004202A2F13003761C012296F800C0ACF13E
:1038E000300EBEF10A0FEED32D2908BF5B422968C6
:1038F0005918296002B90646B8F1000F03D007B97C
:103900000A9EC8F8006050460BB0BDE8F08F00007A
:1039100000E1F505303132333435363738396162FC
:10392000636465664142434445460000000102036A
:103930000405060708090A0B0C0D0E0F0A0B0C0DE7
:103940000E0F000010B50446012000F071F820466B
:10395000BDE8104000F078B810B50446012000F032
:1039600067F82046BDE8104000F079B880B51348EC
:10397000FAF71EF80FF24801016041608160C160F2
:103980000161416181610FF23C0242628162C16268
:10399000016341630FF2300282630FF23402C263AB
:1039A0000164416401BD10B50448FAF701F804460A
:1039B000206808B9FFF7DAFF204610BD7804FF1F22
:1039C000000000002E00000066616C7365000000BE
:1039D0007472756500000000C9B2830706D0521EDC
:1039E00022D310F8013B9942F7D11FE0083A13D3D4
:1039F00002F1040241EA012141EA014150F8043B8D
:103A0000121F21BF4B40A3F1013C2CEA030C1CF018
:103A1000803FF3D0C9B2001F083210F8013B521E9C
:103A200028BF91EA030FF8D818BF0120401E704745
:103A300010B50446DFF80C00F9F7BAFF50F824007F
:103A400010BD00000C04FF1FA0F161011A2904D36E
:103A500041381A288041C00F704701207047A0F1FB
:103A60000901052901D3202801D101207047002038
:103A70007047000080B5DFF8F40BFFF7ABF800F0FB
:103A800045F9642100A800F013FA00280ED19DF832
:103A9000000000280AD0DFF8D80BC06D002805D040
:103AA0009DF80000DFF8C81BC96D8847DFF8C00B20
:103AB000406DDFF8BC1B11EB80004068DFF8641C30
:103AC000884203D10021142000F052F9D9E780B5D3
:103AD000DFF8980BFFF77EF8DFF8940B406DDFF806
:103AE000901B11EB80004068002832D0DFF8800B7B
:103AF000406DDFF87C1B11EB80004068006800F02F
:103B000053F90200D2B20121DFF8640B406DDFF8F7
:103B1000603B13EB80004068006800F033F900223E
:103B20000221DFF8040C00F02DF900220321DFF858
:103B3000400B406DDFF8383B13EB80004068406875
:103B400000F020F997A0FFF745F8DFF8DC0BFFF74E
:103B500041F801BD38B504000D00EDB22800FFF7B3
:103B6000F1FE002804D0EDB2280000F03FFE050071
:103B7000002000E0401CDFF8F81A496DDFF8F02A59
:103B800012EB81014968B1F90C1000B2884213DAD6
:103B90000C21DFF8DC2A526DDFF8D43A13EB8202F5
:103BA0005268926810FB0121216021680978EDB20A
:103BB000A942DFD1012000E0002032BD70B582B003
:103BC00004000D0000264FF6FF7100A800F070F908
:103BD0009DF80000082809D0112806D0132804D029
:103BE0001B280BD07F2801D00CE013E0002E11D051
:103BF000761E641EADA0FEF7EDFF0BE000202070E6
:103C0000FF2011E0BAA0FEF7E5FF9DF8000020704C
:103C1000641C761C681E864203DA9DF800000D289D
:103C2000D1D100202070002076BD00B589B0DFF82A
:103C3000040B0068002801D0002017E0DFF8F80A24
:103C4000FEF7C8FF1F2100A8FFF7B8FF00280CD11E
:103C5000DFF8E81A00A800F0D5FD002805D1DFF84C
:103C6000D40A01210160002000E0FF2009B000BD5E
:103C700080B50100C9B200A8FFF76CFF002844D04E
:103C80000098806800282DD000988068DFF8B01A6E
:103C9000884206D1FFF7C9FF002802D0FFF717FFBF
:103CA00033E0DFF8CC09406D401CDFF8C4194865EB
:103CB000DFF8BC09406DDFF8B81911EB80000099FE
:103CC00089684160FFF703FF0098406800281CD016
:103CD000DFF89C0900994968C1650020009949688E
:103CE000884712E000984068002804D100F025F8C9
:103CF000FFF7EDFE09E0DFF87409FEF76BFF002027
:103D0000009949688847FFF7E2FE01BD80B5DFF8FA
:103D1000600900214165DFF85809406DDFF850194E
:103D200011EB8000DFF8FC194160FFF7D0FEDFF8EF
:103D30004009DFF8101AC16501BDDFF83409406D94
:103D400000280FD0DFF82809406DDFF8241911EBA7
:103D5000800000214160DFF81809406D401EDFF847
:103D600010194865DFF80809DFF8D819C1657047F0
:103D700080B5C9B20A00C0B20100DFF8CC09FEF775
:103D800029FF01BD10B50400D2B2C9B2DFF8B809ED
:103D9000FEF720FF200000F057FD0100200000F09A
:103DA00077F810BD0D0A0000002100E0491C09B29F
:103DB0000A5C002AFAD109B2D1F15000022190FB2D
:103DC000F1F0C0B270472DE9FC4104000E0015006F
:103DD000984601A8DFF874190A68026000270021DC
:103DE0002800C0B2FFF7C4FF42A0FEF7F3FE42A0D6
:103DF000FEF7F0FEB8F1000F0AD0404600F024FDB7
:103E00000700B74203DA4046FEF7E4FE00E0002771
:103E10004FF47A7100A800F04BF8002801D0FF267B
:103E200013E09DF8000008281AD1012F04DB7F1E43
:103E3000042101A800F02CF89DF800000D2801D005
:103E4000502FE5DB00260020385500212800C0B2A5
:103E5000FFF78EFF27A0FEF7BDFE3000BDE8F6811C
:103E60009DF800000D28E7D09DF800000A28E3D057
:103E70009DF800000028DFD0012100A800F008F81C
:103E80009DF8000038557F1CB742D5DBFF26DCE7E4
:103E900070B504000D00002604E0315D17A0FEF7A8
:103EA00099FE761CAE42F8D3002070BD08200800B1
:103EB00038B504000D0003E00220F6F788FE6D1E01
:103EC0000020FEF763FE00F0DAFC002803D1002D8D
:103ED000F2D1FF2006E00020FEF758FE00F0E5FCDE
:103EE0002070002032BDDFF86818086070470000BD
:103EF0002A0000001B5B4B003E0000002563000011
:103F000030B5DFB0DFF84C08FEF764FEDFF8480894
:103F1000FEF760FE0AE1DFF84408FEF75BFE20983A
:103F2000002804D0DFF83808FEF754FE03E0DFF87D
:103F30003408FEF74FFE32A8FBF7F5FD3C98FBF77F
:103F400073FFCDE902013898FBF76EFFCDE9000160
:103F50003498FBF769FF02000B00DFF80C08FEF74E
:103F600039FE3B98FBF760FFCDE902013798FBF77C
:103F70005BFFCDE900013398FBF756FF02000B0011
:103F8000DFF8E807FEF726FE3A98FBF74DFFCDE98C
:103F900002013698FBF748FFCDE900013298FBF7A4
:103FA00043FF02000B00DFF8C807FEF713FE3D9841
:103FB000FBF73AFFCDE902013998FBF735FFCDE970
:103FC00000013598FBF730FF02000B00DFF8A40773
:103FD000FEF700FED6A0FEF7FDFD4198FBF724FF9B
:103FE000CDE904013E98FBF71FFFCDE902013F98A0
:103FF000FBF71AFFCDE900014098FBF715FF02001F
:104000000B00DFF87407FEF7E5FD4598FBF70CFFA2
:10401000CDE904014298FBF707FFCDE9020143987F
:10402000FBF702FFCDE900014498FBF7FDFE02001B
:104030000B00DFF84807FEF7CDFD322106A8FFF799
:1040400037FF00286FD19DF8180030283FD0312865
:1040500000F01481322800F03E81332800F06E8198
:10406000342800F08781352800F0A281362800F03E
:10407000BD81372800F0E781382800F01082392808
:1040800000F039823C2800F08E823E2800F08F82BA
:10409000412800F04C82422800F06782462800F058
:1040A0008E82472800F08F82512800F084825228A7
:1040B00000F08D82662800F08282672800F08382FB
:1040C000712800F07882722800F081822BE022981B
:1040D000FBF7AAFE02000B00DFF8A41607A8FDF705
:1040E0001BF807AB18221E2107A8FFF76CFE00285B
:1040F00019D122AA8FA107A800F0FAFB012812D13A
:104100009DED220ADFED8C0AB4EE600AF1EE10FAA2
:1041100009D59DED220AB5EE400AF1EE10FA02DB58
:1041200018A8FAF703FC641C55F1000500210320D0
:10413000FFF71EFEDFF84C06FEF74CFD22002B00B9
:10414000DFF84406FEF746FD18A8FAF7E2FB2298CE
:10415000FBF76AFE02000B00DFF83006FEF73AFDBF
:104160002498FBF761FE02000B00DFF82406FEF73F
:1041700031FD2398FBF758FE02000B00DFF8140610
:10418000FEF728FD2599DFF81006FEF723FD269996
:10419000DFF80806FEF71EFD2799DFF80406FEF794
:1041A00019FD2898FBF740FE02000B00DFF8F4052C
:1041B000FEF710FD2A98FBF737FE02000B00DFF830
:1041C000E805FEF707FD2998FBF72EFE02000B001D
:1041D000DFF8D805FEF7FEFC2B99DFF8D405FEF7D3
:1041E000F9FC2C99DFF8CC05FEF7F4FC2D99DFF8EB
:1041F000C805FEF7EFFCDFF8C405FEF7EBFC1B99E2
:10420000DFF8BC05FEF7E6FC1999DFF8B805FEF704
:10421000E1FCDDE91C01CDE90001DDE91E231A996D
:10422000DFF8A405FEF7D6FC2E98FBF7FDFD020093
:104230000B00DFF89805FEF7CDFC17A8FCF76DF929
:1042400000287FF468AE1798FBF7EEFDCDE900017A
:10425000DFF87C253F2107A8FCF771FF07A800F0D5
:10426000F3FA072804D307A800F0EEFAFFF73BFEA5
:1042700007A9DFF86005FEF7ADFC50E62498FBF7D0
:10428000D3FD02000B00DFF8F81407A8FCF744FF89
:1042900007AB18221E2107A8FFF795FD002819D1AA
:1042A00024AA24A107A800F023FB012812D19DED28
:1042B000240ADFED210AB4EE600AF1EE10FA09D506
:1042C0009DED240AB5EE400AF1EE10FA02DB18A8C3
:1042D000FAF72CFB27E72398FBF7A6FD02000B005B
:1042E000DFF89C1407A8FCF717FF07AB18221E2164
:1042F00007A8FFF768FD002819D123AA0DA107A878
:1043000000F0F6FA012812D19DED230ADFED0A0A2A
:10431000B4EE600AF1EE10FA09D59DED230AB5EE70
:10432000400AF1EE10FA02DB18A8FAF7FFFAFAE6F3
:104330000D0A0000256600000100803F259AC8A1F3
:1043400007A8FCF7E9FE07AB18221E2107A8FFF714
:104350003AFD00280DD125AAC1A107A800F0C8FA8E
:10436000012806D12598401E642802D218A8FAF721
:10437000DDFAD8E6269ABAA107A8FCF7CDFE07AB6E
:1043800018221E2107A8FFF71EFD00280FD126AA1C
:10439000B3A107A800F0ACFA012808D12698001EA6
:1043A00042F21071884202D218A8FAF7BFFABAE6B0
:1043B000279AABA107A8FCF7AFFE07AB18221E2176
:1043C00007A8FFF700FD00280FD127AAA4A107A87E
:1043D00000F08EFA012808D12798001E42F21071D1
:1043E000884202D218A8FAF7A1FA9CE62898FBF7AF
:1043F0001BFD02000B00DFF8881307A8FCF78CFEFA
:1044000007AB18221E2107A8FFF7DDFC002819D1F1
:1044100028AA94A107A800F06BFA012812D19DEDFB
:10442000280ADFED910AB4EE600AF1EE10FA09D520
:104430009DED280AB5EE400AF1EE10FA02DB18A84D
:10444000FAF774FA6FE62A98FBF7EEFC02000B000D
:10445000CB4907A8FCF760FE07AB18221E2107A86E
:10446000FFF7B1FC002819D12AAA7EA107A800F005
:104470003FFA012812D19DED2A0ADFED7B0AB4EE46
:10448000600AF1EE10FA09D59DED2A0AB5EE400A50
:10449000F1EE10FA02DB18A8FAF748FA43E6299879
:1044A000FBF7C2FC02000B00B54907A8FCF734FE7D
:1044B00007AB18221E2107A8FFF785FC002819D199
:1044C00029AA68A107A800F013FA012812D19DEDCE
:1044D000290ADFED650AB4EE600AF1EE10FA09D59B
:1044E0009DED290AB5EE400AF1EE10FA02DB18A89C
:1044F000FAF71CFA17E62B9A59A107A8FCF70CFE4D
:1045000007AB18221E2107A8FFF75DFC00280DD17C
:104510002BAA53A107A800F0EBF9012806D12B988C
:10452000401E642802D218A8FAF700FAFBE52C9A7C
:104530004BA107A8FCF7F0FD07AB18221E2107A826
:10454000FFF741FC00280FD12CAA45A107A800F0D5
:10455000CFF9012808D12C98001E42F21071884230
:1045600002D218A8FAF7E2F9DDE52D9A3CA107A8D6
:10457000FCF7D2FD07AB18221E2107A8FFF723FC8A
:1045800000280FD12DAA36A107A800F0B1F9012803
:1045900008D12D98001E42F21071884202D218A84C
:1045A000FAF7C4F9BFE51020FAF760F9BBE520205F
:1045B000FAF75CF9B7E54020FAF758F9B3E50120BE
:1045C000F9F703FDAFE50020F9F7FFFCABE55FB0BD
:1045D00030BD10B588B08048FEF7FCFA7F48FEF782
:1045E000F9FAFFE70A20FCF777FA002810D000213B
:1045F00002A8FFF75DFC0028F4D19DF808005228BE
:1046000001D07228EED108B010BD48A0FEF7E2FA42
:1046100003A8FCF774FA0028E9D19DF8180001906E
:104620009DF81A0000909DF81930039A9DF81B1010
:104630006B48FEF7CFFA002406E003A820180179A2
:104640006848FEF7C7FA641C9DF818008442F4D34A
:10465000082CDAD236A0FEF7BDFA641CF8E7000099
:1046600025640000256600000100803F5C660100B3
:10467000F898FF1F80B52DED028BB0B0FFE76421E5
:1046800002A8FFF715FC0028F9D19DF80800302892
:1046900004D0522801D07228F1D13FE04FF40072CB
:1046A000022103A8FAF7C8F84FF40072022103A808
:1046B000FAF7C2F8002823D1FBF713FAB0EE408ACC
:1046C00004A8FBF730FA18EE100AFBF7ADFBCDE9B2
:1046D00000019DED070ADDED0B0A30EE200ADDED4D
:1046E0000F0A30EE200AF0EE080A80EE200A10EEE3
:1046F000100AFBF799FB02000B003B48FEF76AFA31
:10470000002102A8FFF7D4FB0028CDD19DF80800B6
:10471000522803D09DF808007228C5D130B0BDECF6
:10472000028B01BD746D0100706601000D0A00006E
:1047300020202000689BFF1FC4660100E86601007E
:10474000B86D0100713C0100F066010000670100D6
:104750006C9BFF1F046701001C670100F86A0100E1
:10476000206B01004C6B0100646B01009C6B01002D
:10477000D46B01000C6C0100446C0100886C0100DA
:10478000CC6C010068670100BC670100C8670100CC
:10479000FC6701003068010064680100986801004E
:1047A000CC680100006901003469010068690100FA
:1047B0009C690100D0690100046A0100386A0100A7
:1047C000406A0100606A0100806A0100BC6A010061
:1047D000D46A0100DC6A0100D46C0100E06C0100C5
:1047E000F86C0100146D01001C6D010010B5044649
:1047F0000120FFF71DF9A4F161001A2838BF203C01
:10480000204610BD820707D010F8012B11F8013B9C
:10481000BAB19A42F6D014E002680B689A42A2F14B
:10482000013301BF934313F0803F50F8042F51F838
:10483000043FF3D010F8012B11F8013B0AB19A4262
:10484000F8D0D01A7047000000F10103810704D0AE
:1048500010F8011B89B18107FAD10268B2F1013168
:10486000914311F0803F04BF50F8042FF6E710F891
:10487000011B11B110F8011BFBE7C01A704780B58E
:10488000002801D100200FE08169002901D001201A
:104890000AE00368D969002905D000AA0621DB696E
:1048A0009847009800E0002002BD80B5002802D1A2
:1048B0005FF0FF301BE08169002904D0C16900224C
:1048C0008261080013E003685969002904D12C2192
:1048D000C1605FF0FF300AE0012200A95B699847E0
:1048E000012802D19DF8000001E05FF0FF3002BD19
:1048F0000CB480B502AAFEF781F902BC5DF80CFB8E
:1049000010B582B004000800002802D15FF0FF302B
:1049100015E003689969002904D12C21C1605FF07A
:10492000FF300CE021008DF80010012200A99B69E6
:104930009847012802D05FF0FF3000E0200016BD4C
:10494000816807E002681168536889185B18C360C2
:1049500008320260C2689142F4D04A1C8260087832
:1049600070472DE9FF4D00F1080100910027016813
:10497000009A490802EBC1010191B8460021029159
:1049800003910168490800EBC101406800F001058E
:1049900001F10804400804EBC00631E000A8FFF76D
:1049A000CFFF4FFA80FA0AE00098016808180099D2
:1049B0000290496808180390009808300090029807
:1049C00003998842F0D0401C029010F801BD474581
:1049D0000CD1B44208BF00F01DF8276805B14F4460
:1049E000606800EB070808344745F2D007F801BBC0
:1049F000BAF1000F0AD51AF1010AE8D14745CDD125
:104A0000B442CBD1304604B0BDE8F08DBAF1010A12
:104A1000D5D5F3E70120F5F7D7BE00000000000070
:104A200001DF704701DFFEE7A148006872B6018B25
:104A300031B9416AC269D369994201D062B603DFD4
:104A400062B6704703DF7047FEE702DF704772B659
:104A50001EF0040F0CBFEFF30881EFF309818969A1
:104A600011F8021C032905D100B500F01CF85DF80F
:104A700004EB16E0012902D18D48006849E00229C3
:104A80000FD18B480068C1698A6842F001028A60D0
:104A900000B54A680B6813605A6000F004F85DF8CE
:104AA00004EB62B6704707B58248416811F0805F39
:104AB00007D1EFF31182A2F1100280F822207E4983
:104AC000416007BD72B6EFF3098C7C498A78EFF339
:104AD00011832CE9FC4F76480068C369C3F814C001
:104AE000996A11F0020F14D0D3F834C0744A52F806
:104AF000041B4CF8041B52F8041B4CF8041B52F81E
:104B0000041B4CF8041BF1EE101A4CF8081B8CEC3B
:104B1000200A72B6416A0A688A420CD18968090083
:104B2000F9D181F311886549FF228A7062B630BFDE
:104B300072B6016AEFE74162C261938C4383916A66
:104B400011F0020F18D0836C9A4215D08264D2F80B
:104B500034C05B4C5CF8043B44F8043B5CF8043B19
:104B600044F8043B5CF8043B44F8043B5CF8083B25
:104B7000E1EE103ABCEC200AD2F814C0BCE8FC4FBD
:104B800083F311888CF309884A484E49416062B624
:104B9000704772B600B5464B1B68198B01F10101D5
:104BA0001983002001B4EFF31182EFF30581586BF4
:104BB00007B4EFF30880586308461A6B02B925E082
:104BC000904223D8DA6A811A20DB4FF00C0202FBF4
:104BD00001F19A6B11440A68886862B608B490477C
:104BE00008BC72B607BC586301BC198B491E1983F7
:104BF000DA69906A10F4805F06D129B9596A0968A8
:104C0000914218BFFFF74FFF62B600BD9A6AE4E712
:104C100072B6F1B4264B1B68D3F834C00CF1100CFB
:104C20005CF804EB284820F00100CCF818009CE860
:104C3000FF005DF804CBACF1040C2CE9FF00F0BCE4
:104C40008CF3088862B6704719480068C369996A8E
:104C5000D3F834C01A4A52F8041B4CF8041B52F81B
:104C6000041B4CF8041B52F8041B4CF8041BF1EE17
:104C7000101A4CF8081B8CEC200A70474FF0800289
:104C8000D0E84F1F00290CBFC0E8432F01E0002BE4
:104C9000F6D108467047EFF309807047EFF30880BC
:104CA000704780F308887047EFF303807047000077
:104CB0000004FF1F00ED00E00000001020ED00E008
:104CC00034EF00E000000008E14B010001000200A9
:104CD0000000000000000000FFFFF11B0000F0FFDB
:104CE00001000000FFFFF11B0000F0FF02000000C8
:104CF000FFFFF11B0000F0FF03000000FFFFF11BAE
:104D00000000F0FF04000000FFFFF11B0000F0FFB7
:104D100005000000FFFFF11B0000F0FF060000008F
:104D2000FFFFF11B0000F0FF07000000FFFFF11B79
:104D30000000F0FF0001020202000100000000007C
:104D4000020303020202030403030303040000003E
:104D50000100000002000000040000001400000038
:104D600016000000180000001A0000001C000000DF
:104D70001E00000022000000280000001C000000AF
:104D80002000000024000000280000002C0000008B
:104D90003000000038000000440000003000000037
:104DA00038000000400000004800000050000000F3
:104DB0005800000068000000800000005000000063
:104DC0006000000070000000800000009000000003
:104DD000A0000000C0000000F0000000A0000000E3
:104DE000C0000000E0000000000100002001000001
:104DF0004001000080010000E001000040010000CF
:104E000080010000C001000000020000400200001C
:104E10008002000000030000C003000080020000C8
:104E20000003000080030000000400008004000074
:104E300000050000000600008007000000050000DB
:104E40000006000000070000000800000009000044
:104E5000000A0000000C0000180B00007474796157
:104E60003A000000693263303A00000000F00F4061
:104E7000009004400000000000000000010000005D
:104E8000070000000100000000000000000000001A
:104E90000000000000000000000000000000000012
:104EA00000F00F40009004400100000000000000EE
:104EB00001000000070000000100000000000000E9
:104EC00000000000000000000000000000000000E2
:104ED0000000000000F00F400090044002000000BD
:104EE00000000000010000000700000001000000B9
:104EF00000000000000000000000000000000000B2
:104F0000000000000000000000F00F40009004408E
:104F10000300000000000000010000000700000086
:104F20000100000000000000000000000000000080
:104F300000000000000000000000000000F00F4032
:104F40000090044004000000000000000000000089
:104F5000010000000100000000000000000000004F
:104F6000000000000300000000000000000000003E
:104F700000F00F4000900440050000000000000019
:104F80000100000007000000010000000000000018
:104F90000000000000000000000000000000000011
:104FA0000000000000F00F400090044006000000E8
:104FB00000000000000000000500000001000000EB
:104FC00000000000000000000000000003000000DE
:104FD000000000000000000000F00F4000900440BE
:104FE00007000000000000000000000001000000B9
:104FF00001000000000000000000000000000000B0
:1050000003000000000000000000000000F00F405E
:1050100000900440080000000000000000000000B4
:10502000010000000100000000000000000000007E
:10503000000000000300000000000000000000006D
:1050400000F00F4000900440090000000000000044
:10505000000000000100000001000000000000004E
:10506000000000000000000003000000000000003D
:105070000000000000F00F40009004400A00000013
:10508000000000000000000001000000010000001E
:105090000000000000000000000000000000000010
:1050A000000000000000000000F00F4000900440ED
:1050B0000B000000000000000000000001000000E4
:1050C00001000000000000000000000000000000DF
:1050D00000000000000000000000000000F00F4091
:1050E000009004400C0000000000000000000000E0
:1050F00001000000010000000000000000000000AE
:10510000000000000000000000000000000000009F
:1051100000F00F40009004400D000000000000006F
:10512000000000000100000001000000000000007D
:10513000000000000000000000000000010000006E
:105140000100000000F00F40009004400E0000003D
:10515000000000000000000001000000010000004D
:10516000000000000000000000000000000000003F
:10517000000000000000000000F00F40009004401C
:105180000F0000000000000000000000010000000F
:10519000010000000000000000000000000000000E
:1051A00000000000000000000000000000F00F40C0
:1051B000009004401000000000000000000000000B
:1051C00001000000010000000000000000000000DD
:1051D00000000000000000000000000000000000CF
:1051E00000F00F400090044011000000000000009B
:1051F00000000000010000000100000000000000AD
:10520000000000000000000000000000000000009E
:105210000000000000F00F40009004401800000063
:10522000000000000000000001000000010000007C
:10523000000000000100000000000000030000006A
:10524000010000000000000000F00F40009004404A
:105250001900000000000000000000000100000034
:10526000010000000000000001000000000000003C
:1052700003000000010000000000000000F00F40EB
:10528000009004401A000000000000000000000030
:10529000010000000100000000000000010000000B
:1052A00000000000030000000100000000000000FA
:1052B00000F00F40009004401B00000000000000C0
:1052C00000000000010000000100000000000000DC
:1052D00000000000000000000300000000000000CB
:1052E0000000000000F00F40009004401C0000008F
:1052F00000000000000000000100000001000000AC
:10530000000000000000000000000000030000009A
:10531000000000000000000000F00F40009004407A
:105320001D00000000000000000000000000000060
:10533000010000000000000000000000000000006C
:1053400003000000000000000000000040F00F40DB
:1053500000A0044000000000000000000000000069
:10536000010000000100000000000000000000003B
:10537000000000000300000000000000000000002A
:1053800040F00F4000A004400100000000000000B9
:10539000000000000100000001000000000000000B
:1053A00000000000000000000300000000000000FA
:1053B0000000000040F00F4000A004400200000088
:1053C00000000000000000000000000001000000DC
:1053D00000000000000000000000000003000000CA
:1053E000000000000000000040F00F4000A004405A
:1053F00003000000000000000000000001000000A9
:10540000010000000000000000000000000000009B
:1054100003000000000000000000000040F00F400A
:1054200000A0044004000000000000000000000094
:10543000010000000100000000000000000000006A
:105440000000000003000000000000000000000059
:1054500040F00F4000A004400500000000000000E4
:10546000000000000100000001000000000000003A
:105470000000000000000000030000000000000029
:105480000000000040F00F4000A0044006000000B3
:10549000000000000000000000000000010000000B
:1054A00000000000000000000000000003000000F9
:1054B000000000000000000040F00F4000A0044089
:1054C00007000000000000000000000001000000D4
:1054D00001000000000000000000000000000000CB
:1054E00003000000000000000000000040F00F403A
:1054F00000A00440080000000000000000000000C0
:105500000100000001000000000000000000000099
:105510000000000003000000000000000000000088
:1055200040F00F4000A0044009000000000000000F
:105530000000000001000000010000000000000069
:105540000000000000000000030000000000000058
:105550000000000040F00F4000A004400A000000DE
:105560000000000000000000010000000100000039
:105570000000000000000000000000000300000028
:10558000000000000000000040F00F4000A00440B8
:105590000B000000000000000000000001000000FF
:1055A00001000000000000000000000000000000FA
:1055B00003000000000000000000000040F00F4069
:1055C00000A00440100000000000000000000000E7
:1055D00003000000010000000000000000000000C7
:1055E00000000000030000000000000000000000B8
:1055F00040F00F4000A00440110000000000000037
:105600000000000003000000010000000000000096
:105610000000000000000000030000000000000087
:105620000000000040F00F4000A004401200000005
:105630000000000000000000020000000100000067
:105640000000000000000000000000000300000057
:10565000000000000000000040F00F4000A00440E7
:105660001300000000000000000000000200000025
:105670000100000000000000000000000000000029
:1056800003000000000000000000000040F00F4098
:1056900000A0044014000000000000000000000012
:1056A00002000000010000000000000000000000F7
:1056B00000000000030000000000000000000000E7
:1056C00040F00F4000A00440150000000000000062
:1056D00000000000020000000100000000000000C7
:1056E00000000000000000000300000000000000B7
:1056F0000000000040F00F4000A004401600000031
:105700000000000000000000020000000100000096
:105710000000000000000000000000000300000086
:10572000000000000000000040F00F4000A0044016
:105730001700000000000000000000000200000050
:105740000100000000000000000000000000000058
:1057500003000000000000000000000080F00F4087
:1057600000B0044000000000000000000000000045
:105770000100000001000000000000000000000027
:105780000000000003000000010000000000000015
:1057900080F00F4000B00440010000000000000055
:1057A00000000000040000000100000000000000F4
:1057B00000000000000000000200000000000000E7
:1057C0000000000080F00F4000B004400200000024
:1057D00000000000000000000400000001000000C4
:1057E00000000000000000000000000002000000B7
:1057F000000000000000000080F00F4000B00440F6
:105800000300000000000000000000000400000091
:105810000100000000000000000000000000000087
:1058200002000000000000000000000080F00F40B7
:1058300000B0044004000000000000000000000070
:105840000400000001000000000000000000000053
:105850000000000002000000000000000000000046
:1058600080F00F4000B00440050000000000000080
:105870000000000001000000010000000000000026
:105880000000000000000000030000000000000015
:105890000000000080F00F4000B00440060000004F
:1058A00000000000000000000100000001000000F6
:1058B00000000000000000000000000003000000E5
:1058C000000000000000000080F00F4000B0044025
:1058D00007000000000000000000000001000000C0
:1058E00001000000000000000000000000000000B7
:1058F00003000000000000000000000080F00F40E6
:1059000000B004400800000000000000000000009B
:105910000100000001000000000000000000000085
:105920000000000003000000000000000000000074
:1059300080F00F4000B004400900000000000000AB
:105940000000000001000000010000000000000055
:105950000000000000000000030000000000000044
:105960000000000080F00F4000B004400A0000007A
:105970000000000000000000010000000100000025
:105980000000000000000000000000000300000014
:10599000000000000000000080F00F4000B0044054
:1059A0000B000000000000000000000001000000EB
:1059B00001000000000000000000000000000000E6
:1059C00003000000000000000000000080F00F4015
:1059D00000B004400C0000000000000000000000C7
:1059E00001000000010000000000000000000000B5
:1059F00000000000030000000000000000000000A4
:105A000080F00F4000B004400D00000000000000D6
:105A10000000000001000000010000000000000084
:105A20000000000000000000030000000100000072
:105A30000000000080F00F4000B004400E000000A5
:105A40000000000000000000010000000100000054
:105A50000000000000000000000000000300000043
:105A6000010000000000000080F00F4000B0044082
:105A70000F00000000000000000000000100000016
:105A80000100000000000000000000000000000015
:105A900003000000000000000000000080F00F4044
:105AA00000B00440100000000000000000000000F2
:105AB00001000000010000000000000000000000E4
:105AC00000000000030000000000000000000000D3
:105AD00080F00F4000B00440110000000000000002
:105AE00000000000010000000100000000000000B4
:105AF00000000000000000000300000000000000A3
:105B00000000000080F00F4000B0044012000000D0
:105B10000000000000000000010000000100000083
:105B20000000000000000000000000000300000072
:105B3000000000000000000080F00F4000B00440B2
:105B40001300000000000000000000000100000041
:105B50000100000000000000000000000000000044
:105B6000030000000000000000000000C0F00F4033
:105B700000C0044000000000000000000000000021
:105B80000100000001000000000000000000000013
:105B90000000000003000000010000000000000001
:105BA000C0F00F4000C004400100000000000000F1
:105BB00000000000010000000100000000000000E3
:105BC00000000000000000000300000001000000D1
:105BD00000000000C0F00F4000C0044002000000C0
:105BE00000000000000000000100000001000000B3
:105BF00000000000000000000000000003000000A2
:105C00000000000000000000C0F00F4000C0044091
:105C10000300000000000000000000000100000080
:105C20000100000000000000000000000000000073
:105C3000030000000100000000000000C0F00F4061
:105C400000C004400400000000000000000000004C
:105C5000040000000100000000000000000000003F
:105C60000000000002000000000000000000000032
:105C7000C0F00F4000C0044005000000000000001C
:105C8000000000000400000001000000000000000F
:105C90000000000000000000020000000000000002
:105CA00000000000C0F00F4000C0044006000000EB
:105CB00000000000000000000100000001000000E2
:105CC00000000000000000000000000003000000D1
:105CD0000100000000000000C0F00F4000C00440C0
:105CE00007000000000000000000000001000000AC
:105CF00001000000000000000000000000000000A3
:105D0000030000000000000000000000C0F00F4091
:105D100000C0044008000000000000000000000077
:105D20000200000001000000000000000000000070
:105D3000010000000300000000000000000000005F
:105D4000C0F00F4000C00440090000000000000047
:105D50000000000002000000010000000000000040
:105D6000000000000100000003000000000000002F
:105D700000000000C0F00F4000C004400A00000016
:105D80000000000000000000010000000100000011
:105D90000000000000000000000000000300000000
:105DA0000000000000000000C0F00F4000C00440F0
:105DB0000B000000000000000000000001000000D7
:105DC00001000000000000000000000000000000D2
:105DD000030000000100000000000000C0F00F40C0
:105DE00000C004400C0000000000000000000000A3
:105DF00001000000010000000000000000000000A1
:105E0000000000000300000001000000000000008E
:105E1000C0F00F4000C004400D0000000000000072
:105E20000000000001000000010000000000000070
:105E3000000000000000000003000000010000005E
:105E400000000000C0F00F4000C004400E00000041
:105E50000000000000000000010000000100000040
:105E6000000000000000000000000000030000002F
:105E70000100000000000000C0F00F4000C004401E
:105E80000F00000000000000000000000100000002
:105E90000100000000000000000000000000000001
:105EA00003000000010000000000000000F10F40AE
:105EB00000D00440000000000000000001000000CD
:105EC00004000000010000000000000000000000CD
:105ED00000000000030000000000000000000000BF
:105EE00000F10F4000D0044001000000000000005D
:105EF000010000000400000001000000000000009C
:105F0000000000000000000003000000000000008E
:105F10000000000000F10F4000D00440020000002B
:105F2000000000000100000004000000010000006B
:105F3000000000000000000000000000030000005E
:105F4000000000000000000000F10F4000D00440FD
:105F50000300000000000000010000000400000039
:105F60000100000000000000000000000000000030
:105F700003000000000000000000000000F10F40DE
:105F800000D00440040000000000000001000000F8
:105F900004000000010000000000000000000000FC
:105FA00000000000030000000000000000000000EE
:105FB00000F10F4000D00440050000000000000088
:105FC00001000000040000000100000000000000CB
:105FD00000000000000000000300000000000000BE
:105FE0000000000000F10F4000D004400600000057
:105FF000000000000000000006000000010000009A
:10600000000000000000000000000000030000008D
:10601000000000000000000000F10F4000D004402C
:106020000700000000000000000000000100000068
:10603000010000000000000000000000000000005F
:1060400003000000010000000000000000F10F400C
:1060500000D0044008000000000000000000000024
:10606000000000000100000000000000000000002F
:10607000000000000300000000000000000000001D
:1060800000F10F4000D004400900000000000000B3
:1060900000000000010000000100000000000000FE
:1060A00000000000000000000300000000000000ED
:1060B0000000000000F10F4000D004400A00000082
:1060C00000000000000000000100000001000000CE
:1060D00000000000000000000000000003000000BD
:1060E000000000000000000000F10F4000D004405C
:1060F0000B00000000000000000000000100000094
:10610000010000000000000000000000000000008E
:1061100003000000000000000000000000F10F403C
:1061200000D004400C00000000000000000000004F
:10613000010000000100000000000000000000005D
:10614000000000000300000000000000000000004C
:1061500000F10F4000D004401800000000000000D3
:10616000000000000000000001000000000000002E
:10617000000000000000000003000000000000001C
:106180000000000000F10F4000D0044019000000A2
:1061900000000000000000000100000001000000FD
:1061A00000000000000000000000000003000000EC
:1061B000000000000000000000F10F4000D004408B
:1061C0001A000000000000000000000000000000B5
:1061D00001000000000000000000000000000000BE
:1061E00003000000000000000000000000F10F406C
:1061F00000D004401B000000000000000000000070
:10620000010000000100000000000000000000008C
:10621000000000000300000000000000000000007B
:1062200000F10F4000D004401C00000000000000FE
:10623000000000000000000001000000000000005D
:10624000000000000000000003000000000000004B
:106250000000000000006E00A086010005000000A4
:10626000400000004000000040000000000000006E
:10627000000E270700100E003D0000003E00000049
:10628000030000000400000030313233343536376B
:106290003839414243444546000000003031323332
:1062A0003435363738396162636465660000000052
:1062B0001F001C001F001E001F001E001F001F00EB
:1062C0001E001F001E001F004D6F744973720000F6
:1062D0004374726C000000004D65617300000000A3
:1062E00056543130300000004C43440043414E5F6F
:1062F0005458000043414E5F5258000069695F776F
:106300002020000069695F762020000069695F75C0
:1063100020200000765F62757320000074656D7048
:10632000657200003135762020200000357620206F
:106330002020000076765F772020000076765F765A
:106340002020000076765F7520200000543A2D2D25
:106350002D2D2D2044433A252E306600543A253009
:106360002E31662044433A252E306600493A2534C2
:106370002E3166204572722E4E3A256400000000D0
:10638000493A25342E316620000000002A2A2A2AA4
:106390004F5645524C4F41442A2A2A2A00000000F9
:1063A0002A2A2A2A2A4552524F522A2A2A2A2A2A95
:1063B000000000000100000029EB0000E8030000DD
:1063C00007000000C8620100020000000000000099
:1063D000000000000200000041F20000DC050000A7
:1063E00008000000D062010003000000000000006F
:1063F0000000000003000000FBF80000DC050000C6
:1064000009000000D8620100020000000000000046
:106410000000000004000000753A0100B80B000005
:106420000A000000E0620100060000000000000019
:10643000020000000500000041FB0000D007000042
:106440000B000000E86201000200000000000000F4
:106450000000000006000000BF0A0100DC0500008B
:1064600009000000EC6201000000000000000000D4
:106470000000000007000000BF0B0100DC05000069
:1064800009000000F46201000200000000000000AA
:1064900000000000000000000000000000000000FC
:1064A00000000000000000000000000000000000EC
:1064B00000000000FC62010075F30000E5F300003D
:1064C0000463010075F30000E5F300000C630100B4
:1064D00075F30000E5F300001463010029F60000E5
:1064E000A9F600001C63010007F800006FF8000027
:1064F000246301004DF40000CDF400002C63010082
:1065000045F50000B9F500000C63010029F7000013
:106510009DF7000034630100D9F80000E3F80000A3
:106520003C630100D9F80000E3F800004463010077
:10653000D9F80000E3F80000496E76657274657260
:1065400020312E30204D4F4E49544F522056657207
:106550002E313330393034001B5B3543204D4149F7
:106560004E204D454E55200D0A1B5B3543203C31D6
:106570003E202D2041646A75737461626C652070E1
:106580006172616D657465727320616E64207365FC
:106590007474696E67730D0A1B5B3543203C323E91
:1065A000202D204D6F746F7220746573740D0A1B5B
:1065B0005B3543203C333E202D2043414E20746503
:1065C00073740D0A1B5B3543203C383E202D204D53
:1065D000656173757265642076616C75657320768C
:1065E0006965770D0A0000001B5B35432053504559
:1065F0004349414C204D454E55200D0A1B5B354308
:10660000203C313E202D205369676E616C732064FD
:106610006961676E6F737469630D0A1B5B35432094
:106620003C523E202D20446973706C617920707259
:106630006576696F7573206D656E750D0A1B5B3528
:1066400043203C4D3E202D20446973706C617920BD
:106650006D61696E206D656E750D0A001B5B324AB7
:106660001B5B481B5B6D1B5B3F32356C0000000001
:106670002D2D2D2D2D2D2D2D2D2D2D2D2D2D2D2D4A
:106680002D2D2D2D2D2D2D2D2D2D2D2D2D2D2D2D3A
:106690002D2D2D2D2D2D2D2D2D2D2D2D2D2D2D2D2A
:1066A0002D2D2D2D2D2D2D2D2D2D2D2D2D2D2D2D1A
:1066B0002D2D2D2D2D2D2D2D2D2D2D2D2D2D2D2D0A
:1066C000000000001B5B324A1B5B481B5B6D1B5BC1
:1066D0003F32356C456E7465722061636365737318
:1066E00020636F64653E0000343332310D000000DA
:1066F0001B5B252E32643B252E32644800000000CF
:10670000082008004D6F746F7220616C676F7269AA
:1067100074686D20746573742E0A0D005072657371
:10672000732027522720746F20657869742E2027E4
:106730003C272D646F776E2C20273E272D75702CFB
:10674000202746272D46756E206F6E2C2747272D54
:1067500046756E206F66662C202751272D73746F47
:1067600070200A0D000000002D2D2D2D2D2D2D2D1A
:106770002D2D2D2D2D2D2D2D2D2D2D2D2D2D2D2D49
:106780002D2D2D2D2D2D2D2D2D2D2D2D2D2D2D2D39
:106790002D2D2D2D2D2D2D2D2D2D2D2D2D2D2D2D29
:1067A0002D2D2D2D2D2D2D2D2D2D2D2D2D2D2D2D19
:1067B0002D2D2D2D2D2D2D2D0D0A00001B5B324B67
:1067C000256C6C640D0A00001B5B324B28302920BD
:1067D0004D6F76696E6720757020616363656C2EFE
:1067E00050574D207363616C6520666163746F72EE
:1067F00020203D2025302E33660D0A001B5B324BD6
:10680000283129204D6F76696E67207570205057AA
:106810004D207363616C6520666163746F72202024
:106820002020202020203D2025302E33660D0A0018
:106830001B5B324B283229204D6F76696E672075BD
:106840007020646563656C2E50574D207363616CD6
:106850006520666163746F7220203D2025302E33E1
:10686000660D0A001B5B324B283329204D6F766979
:106870006E6720757020726F742E7370656564206A
:1068800020202020202020202020202020203D20EB
:1068900025640D0A000000001B5B324B28342920C0
:1068A0004D6F76696E6720757020616363656C65F6
:1068B000722E74696D652020202020202020202049
:1068C00020203D2025640D0A000000001B5B324B98
:1068D000283529204D6F76696E67207570206465B4
:1068E00063656C65722E74696D6520202020202000
:1068F0002020202020203D2025640D0A00000000DB
:106900001B5B324B283629204D6F76696E672064F9
:106910006F776E20616363656C2E50574D207363F3
:10692000616C6520666163746F723D2025302E3383
:10693000660D0A001B5B324B283729204D6F7669A4
:106940006E6720646F776E2050574D207363616CC3
:106950006520666163746F722020202020203D2016
:1069600025302E33660D0A001B5B324B2838292058
:106970004D6F76696E6720646F776E20646563651E
:106980006C2E50574D207363616C65206661637493
:106990006F723D2025302E33660D0A001B5B324B93
:1069A000283929204D6F76696E6720646F776E20D5
:1069B000726F742E73706565642020202020202063
:1069C0002020202020203D2025640D0A000000000A
:1069D0001B5B324B284129204D6F76696E6720641E
:1069E0006F776E20616363656C65722E74696D6587
:1069F000202020202020202020203D2025640D0A5A
:106A0000000000001B5B324B284229204D6F766945
:106A10006E6720646F776E20646563656C65722EA7
:106A200074696D65202020202020202020203D201A
:106A300025640D0A000000001B5B324B0D0A0000AC
:106A40001B5B324B4D6F746F72206375722E726FC9
:106A5000742E7370656564203D2025640D0A000066
:106A60001B5B324B526F746174696F6E2064697284
:106A700020202020202020203D2025640D0A000019
:106A80001B5B324B736B65775F636E74203D202513
:106A90003036642C2073746570203D2025303136EB
:106AA0006C6C582C206C6C5F66726571203D2025E3
:106AB0003031366C6C580D0A000000001B5B324B05
:106AC00050574D207363616C653D2025302E336631
:106AD0000D0A000025302E336C6600001B5B324B24
:106AE000494742542074656D7065726174757265B2
:106AF000203D2025730D0A001B5B324B4947425451
:106B00002074656D7065726174757265207265615F
:106B100064696E67206572726F72210D0A00000051
:106B20001B5B324B44657465637465642056464F45
:106B3000203D20302E204D6F746F72206472697674
:106B40006572206661696C210D0A00001B5B324B87
:106B50004D6F746F7220647269766572204F6B217D
:106B60000D0A00001B5B324B43757272656E7473C5
:106B700028772C762C75292E204D617820203A20FC
:106B80002530352E3266202C202530352E326620D9
:106B90002C202530352E32660D0A00001B5B324B4F
:106BA00043757272656E747328772C762C75292E56
:106BB000204D696E20203A202530352E3266202C5B
:106BC000202530352E3266202C202530352E326699
:106BD0000D0A00001B5B324B43757272656E747355
:106BE00028772C762C75292E2041766572203A2044
:106BF0002530352E3266202C202530352E32662069
:106C00002C202530352E32660D0A00001B5B324BDE
:106C100043757272656E747328772C762C75292EE5
:106C200020524D5320203A202530352E3266202C1C
:106C3000202530352E3266202C202530352E326628
:106C40000D0A00001B5B324B4443204255532E205B
:106C50003A206D61783D2530362E3266202C206D2D
:106C6000696E3D2530362E3266202C206176723DCD
:106C70002530362E32662C20524D533D2530362E8F
:106C800032660D0A000000001B5B324B54656D70CC
:106C900065722E203A206D61783D2530362E3266A1
:106CA000202C206D696E3D2530362E3266202C203A
:106CB0006176723D2530362E32662C20524D533D82
:106CC0002530362E32660D0A0000000025302E33A6
:106CD0006600000043414E206C6F672E0A0D0000D5
:106CE00050726573732027522720746F206578696E
:106CF000742E200A0D00000025303258202530382F
:106D00005820253031582025303158202530315831
:106D1000202D2000253032582000000025302E3153
:106D2000662C2025302E31660D0A0000310000004F
:106D300000000000846D010032000000013F0100EE
:106D40000000000033000000D345010000000000F7
:106D500038000000754601000000000052000000ED
:106D600000000000000000004D00000000000000D6
:106D7000746D010038650100586501002C6D01003B
:106D800006000000B0B10100B0B101000000000039
:106D900000000000310000000000000000000000C2
:106DA0005200000000000000000000004D00000044
:106DB00000000000746D010038650100E865010005
:106DC000946D010003000000467265657363616C99
:106DD000652F467265657363616C65204D5158007F
:106DE0005F6D71785F69646C655F7461736B0000DF
:106DF000000000000000000000000000010000048E
:106E0000C86D0100747479613A0000000000000050
:106E1000C09BFF1FF0FF002000040000B4630100CE
:106E2000020000000200000010000000046E0100DB
:106E3000010000000000000000000000000E270715
:106E400000879303005A6202002D31010000000008
:106E5000000E270780841E0000127A0000800000C8
:106E6000093D0000001BB700001BB700001BB70066
:106E7000001BB70000000000000E270780841E00E2
:106E800000127A0000800000093D000080841E008E
:106E900080841E0080841E0020A1070000000000E6
:106EA00080841E0080841E0000127A000000000012
:106EB0000040000000000000E3876400880FC90064
:106EC000B1962D01201D920197A2F601D7265B02F3
:106ED000A4A9BF02BF2A2403EAA98803E626ED037A
:106EE00077A151045D19B6045C8E1A0535007F0543
:106EF000A96EE3057CD947066F40AC0645A3100791
:106F0000BE0175079E5BD907A7B03D089A00A2088D
:106F10003A4B060949906A0989CFCE09BD08330A60
:106F2000A53B970A0568FB0A9F8D5F0B35ACC30B29
:106F300089C3270C5ED38B0C76DBEF0C92DB530DF1
:106F400076D3B70DE4C21B0E9EA97F0E6687E30EB3
:106F5000FF5B470F2B27AB0FADE80E1048A0721058
:106F6000BD4DD610CFF0391141899D11D5160112B2
:106F70004E9964126F10C812F97B2B13B1DB8E137C
:106F8000582FF213B17655147FB1B81486DF1B1554
:106F900086007F154514E215831A45160513A816B9
:106FA0008DFD0A17DED96D17BCA7D017E966331817
:106FB000281796183CB8F818EA495B19F3CBBD19A5
:106FC0001B3E201A26A0821AD6F1E41AEF32471B84
:106FD0003563A91B6A820B1C53906D1CB38CCF1CAC
:106FE0004D77311DE54F931D3F16F51D1ECA561EE8
:106FF000466BB81E7BF9191F81747B1F1BDCDC1FDD
:107000000D303E201C709F200C9C0021A0B36121FC
:107010009CB6C221C5A42322E07D8422AF41E52293
:10702000F8EF45237F88A623080B072458776724A9
:1070300033CDC7245E0C28259D348825B645E82528
:107040006C3F48268621A826C7EB0727F49D6727B3
:10705000D337C72728B92628B92186284B71E528B8
:10706000A2A7442985C4A329B8C7022A01B1612A6D
:107070002680C02AEB341F2B17CF7D2B6F4EDC2BC5
:10708000B9B23A2CBAFB982C3929F72CFC3A552D79
:10709000C730B32D620A112E92C76E2E1E68CC2EF9
:1070A000CCEB292F6252872FA79BE42F61C7413079
:1070B00056D59E304DC5FB300E9758315E4AB531DE
:1070C00004DF1132C7546E326FABCA32C3E22633CB
:1070D00088FA823387F2DE3387CA3A345082963494
:1070E000A819F23457904D3525E6A835D91A04363B
:1070F0003B2E5F361420BA362AF01437469E6F377F
:10710000302ACA37B09324388EDA7E3893FED838C6
:1071100087FF323932DD8C395E97E639D22D403A1D
:1071200057A0993AB7EEF23ABA184C3B291EA53B44
:10713000CDFEFD3B70BA563CDA50AF3CD6C1073DA0
:107140002C0D603DA632B83D0D32103E2C0B683E32
:10715000CDBDBF3EB849173FB8AE6E3F98ECC53FB6
:1071600021031D401DF2734058B9CA409B5821416C
:10717000B1CF7741651ECE4181442442D0417A424D
:107180001E16D04235C12543E1427B43ED9AD043E0
:1071900023C9254450CD7A4440A7CF44BD56244549
:1071A00093DB78458F35CD457D642146286875464B
:1071B0005C40C946E7EC1C47936D70472FC2C3473C
:1071C00086EA164865E6694899B5BC48EE570F4906
:1071D00033CD61493315B449BD2F064A9E1C584A28
:1071E000A2DBA94A986CFB4A4DCF4C4B90039E4BB7
:1071F0002D09EF4BF4DF3F4CB187904C3400E14C4C
:107200004B49314DC462814D6E4CD14D1706214E14
:107210008F8F704EA5E8BF4E26110F4FE3085E4FCB
:10722000ABCFAC4F4D65FB4F99C949505EFC9750B1
:107230006DFDE55094CC3351A56981516ED4CE518A
:10724000C20C1C526E12695246E5B55218850253A3
:10725000B5F14E53F02A9B539730E7537D023354D8
:1072600073A07E544B0ACA54D43F1555E240605572
:10727000460DAB55D2A4F55558074056A9348A5649
:10728000992CD456FAEE1D579D7B675756D2B057AE
:10729000F8F2F95754DD425840918B588C0ED4586F
:1072A0000E551C5998646459FD3CAC5912DEF359D3
:1072B000AB473B5A9A79825AB573C95ACF35105B9E
:1072C000BDBF565B54119D5B672AE35BCC0A295C0A
:1072D00058B26E5CE020B45C3856F95C37523E5DC3
:1072E000B114835D7C9DC75D6EEC0B5E5D01505EED
:1072F0001FDC935E8A7CD75E74E21A5FB30D5E5F1B
:107300001FFEA05F8DB3E35FD62D2660CF6C686053
:107310005070AA603038EC6047C42D616C146F6106
:107320007628B0613F00F1619D9B316269FA71621C
:107330007B1CB262AC01F262D4A93163CC147163DC
:107340006D42B0639032EF630DE52D64BF596C64FC
:107350007F90AA642689E8648F43266592BF63659F
:107360000BFDA065D3FBDD65C5BB1A66BB3C57664C
:10737000917E93662081CF6644440B67D8C74667E9
:10738000B70B8267BD0FBD67C5D3F767AB573268D0
:107390004B9B6C68819EA6682961E06820E31969AF
:1073A000422453696C248C697AE3C4694A61FD699B
:1073B000B99D356AA4986D6AE951A56A64C9DC6A09
:1073C000F5FE136B79F24A6BCDA3816BD112B86BCA
:1073D000623FEE6B6029246CA9D0596C1C358F6C10
:1073E0009856C46CFC34F96C27D02D6DFA27626D69
:1073F000543C966D140DCA6D1C9AFD6D4AE3306EB7
:107400007FE8636E9DA9966E8326C96E125FFB6E40
:107410002C532D6FB2025F6F846D906F8593C16F97
:107420009774F26F9A10237071675370FF788370AE
:107430002545B370C6CBE270C50C127105084171C9
:1074400068BD6F71D22C9E712656CC714939FA7184
:107450001CD62772852C5572673C8272A705AF72C5
:107460002888DB72D0C3077383B8337326665F73D3
:107470009ECC8A73D1EBB573A3C3E073FB530B743B
:10748000BD9C3574D19D5F741C57897484C8B274D7
:10749000EFF1DB7445D304756C6C2D754CBD5575DF
:1074A000CAC57D75CF85A57542FDCC750B2CF475CD
:1074B00011121B763DAF417676036876A60E8E7666
:1074C000B4D0B3768949D9760E79FE762D5F2377CD
:1074D000CEFB4777DB4E6C773E589077DF17B4775B
:1074E000AA8DD77789B9FA77659B1D7829334078BB
:1074F000BF80627814848478113DA678A2ABC778E7
:10750000B2CFE8782DA90979FE372A79127C4A7919
:1075100054756A79B1238A791587A9796E9FC879DC
:10752000A76CE779ADEE057A6F25247AD810427AF8
:10753000D8B05F7A5B057D7A500E9A7AA4CBB67A82
:10754000453DD37A2363EF7A2C3D0B7B4FCB267BD3
:107550007A0D427B9E035D7BA8AD777B890B927B86
:10756000311DAC7B90E2C57B945BDF7B3088F87B80
:107570005368117CEEFB297CF242427C503D5A7CE0
:10758000F9EA717CDE4B897CF15FA07C2427B77C13
:1075900069A1CD7CB2CEE37CF0AEF97C18420F7DC0
:1075A0001B88247DEC80397D7F2C4E7DC68A627DD0
:1075B000B59B767D405F8A7D5AD59D7DF8FDB07D77
:1075C0000DD9C37D8F66D67D70A6E87DA898FA7D1B
:1075D000293D0C7EEA931D7EDF9C2E7EFF573F7E69
:1075E0003EC54F7E93E45F7EF4B56F7E57397F7E54
:1075F000B26E8E7EFC559D7E2CEFAB7E393ABA7E04
:107600001A37C87EC6E5D57E3646E37E6058F07EE2
:107610003C1CFD7EC491097FEEB8157FB491217F9B
:107620000E1C2D7FF657387F6345437F51E44D7F15
:10763000B734587F8F36627FD4E96B7F804E757F79
:107640008C647E7FF32B877FB0A48F7FBDCE977F26
:1076500015AA9F7FB436A77F9574AE7FB363B57FBD
:107660000A04BC7F9655C27F5458C87F3E0CCE7F1B
:107670005371D37F8E87D87FEC4EDD7F6BC7E17F60
:1076800008F1E57FC0CBE97F9157ED7F7894F07FDB
:107690007482F37F8221F67FA271F87FD172FA7F24
:1076A0000F25FC7F5A88FD7FB29CFE7F1662FF7F0C
:1076B00086D8FF7FFFFFFF7F86D8FF7F1662FF7FA0
:1076C000B29CFE7F5A88FD7F0F25FC7FD172FA7F26
:1076D000A271F87F8221F67F7482F37F7894F07F25
:1076E0009157ED7FC0CBE97F08F1E57F6BC7E17F64
:1076F000EC4EDD7F8E87D87F5371D37F3E0CCE7FDB
:107700005458C87F9655C27F0A04BC7FB363B57FC7
:107710009574AE7FB436A77F15AA9F7FBDCE977FA5
:10772000B0A48F7FF32B877F8C647E7F804E757F24
:10773000D4E96B7F8F36627FB734587F51E44D7F39
:107740006345437FF657387F0E1C2D7FB491217F10
:10775000EEB8157FC491097F3C1CFD7E6058F07E19
:107760003646E37EC6E5D57E1A37C87E393ABA7EFC
:107770002CEFAB7EFC559D7EB26E8E7E57397F7EA0
:10778000F4B56F7E93E45F7E3EC54F7EFF573F7E2C
:10779000DF9C2E7EEA931D7E293D0C7EA898FA7D03
:1077A00070A6E87D8F66D67D0DD9C37DF8FDB07DCE
:1077B0005AD59D7D405F8A7DB59B767DC68A627D68
:1077C0007F2C4E7DEC80397D1B88247D18420F7DF7
:1077D000F0AEF97CB2CEE37C69A1CD7C2427B77CE6
:1077E000F15FA07CDE4B897CF9EA717C503D5A7CCC
:1077F000F242427CEEFB297C5368117C3088F87B96
:10780000945BDF7B90E2C57B311DAC7B890B927B67
:10781000A8AD777B9E035D7B7A0D427B4FCB267BA9
:107820002C3D0B7B2363EF7A453DD37AA4CBB67A0C
:10783000500E9A7A5B057D7AD8B05F7AD810427A7A
:107840006F25247AADEE057AA76CE7796E9FC8792B
:107850001587A979B1238A7954756A79127C4A7996
:10786000FE372A792DA90979B2CFE878A2ABC7787B
:10787000113DA67814848478BF80627829334078DB
:10788000659B1D7889B9FA77AA8DD777DF17B4770A
:107890003E589077DB4E6C77CEFB47772D5F237792
:1078A0000E79FE768949D976B4D0B376A60E8E7657
:1078B000760368763DAF417611121B760B2CF4757A
:1078C00042FDCC75CF85A575CAC57D754CBD557576
:1078D0006C6C2D7545D30475EFF1DB7484C8B274FC
:1078E0001C578974D19D5F74BD9C3574FB530B7418
:1078F000A3C3E073D1EBB5739ECC8A7326665F7326
:1079000083B83373D0C307732888DB72A705AF72BF
:10791000673C8272852C55721CD627724939FA71E0
:107920002656CC71D22C9E7168BD6F7105084171CD
:10793000C50C1271C6CBE2702545B370FF78837019
:10794000716753709A1023709774F26F8593C16FAB
:10795000846D906FB2025F6F2C532D6F125FFB6EC0
:107960008326C96E9DA9966E7FE8636E4AE3306EEA
:107970001C9AFD6D140DCA6D543C966DFA27626D0C
:1079800027D02D6DFC34F96C9856C46C1C358F6C67
:10799000A9D0596C6029246C623FEE6BD112B86B90
:1079A000CDA3816B79F24A6BF5FE136B64C9DC6A77
:1079B000E951A56AA4986D6AB99D356A4A61FD6965
:1079C0007AE3C4696C248C694224536920E3196901
:1079D0002961E068819EA6684B9B6C68AB57326852
:1079E000C5D3F767BD0FBD67B70B8267D8C74667BA
:1079F00044440B672081CF66917E9366BB3C5766FB
:107A0000C5BB1A66D3FBDD650BFDA06592BF636540
:107A10008F4326652689E8647F90AA64BF596C6409
:107A20000DE52D649032EF636D42B063CC14716349
:107A3000D4A93163AC01F2627B1CB26269FA716253
:107A40009D9B31623F00F1617628B0616C146F61DB
:107A500047C42D613038EC605070AA60CF6C68600C
:107A6000D62D26608DB3E35F1FFEA05FB30D5E5F72
:107A700074E21A5F8A7CD75E1FDC935E5D01505E04
:107A80006EEC0B5E7C9DC75DB114835D37523E5D2D
:107A90003856F95CE020B45C58B26E5CCC0A295CC4
:107AA000672AE35B54119D5BBDBF565BCF35105B0E
:107AB000B573C95A9A79825AAB473B5A12DEF359C9
:107AC000FD3CAC59986464590E551C598C0ED45821
:107AD00040918B5854DD4258F8F2F95756D2B057BE
:107AE0009D7B6757FAEE1D57992CD456A9348A56B8
:107AF00058074056D2A4F555460DAB55E2406055A7
:107B0000D43F15554B0ACA5473A07E547D0233549A
:107B10009730E753F02A9B53B5F14E531885025323
:107B200046E5B5526E126952C20C1C526ED4CE514B
:107B3000A569815194CC33516DFDE5505EFC9750A1
:107B400099C949504D65FB4FABCFAC4FE3085E4F31
:107B500026110F4FA5E8BF4E8F8F704E1706214E8E
:107B60006E4CD14DC462814D4B49314D3400E14CD6
:107B7000B187904CF4DF3F4C2D09EF4B90039E4BA7
:107B80004DCF4C4B986CFB4AA2DBA94A9E1C584A2D
:107B9000BD2F064A3315B44933CD6149EE570F491D
:107BA00099B5BC4865E6694886EA16482FC2C347BE
:107BB000936D7047E7EC1C475C40C94628687546E2
:107BC0007D6421468F35CD4593DB7845BD562445F0
:107BD00040A7CF4450CD7A4423C92544ED9AD043E1
:107BE000E1427B4335C125431E16D042D0417A4243
:107BF00081442442651ECE41B1CF77419B5821413B
:107C000058B9CA401DF2734021031D4098ECC53F8E
:107C1000B8AE6E3FB849173FCDBDBF3E2C0B683E96
:107C20000D32103EA632B83D2C0D603DD6C1073D49
:107C3000DA50AF3C70BA563CCDFEFD3B291EA53B49
:107C4000BA184C3BB7EEF23A57A0993AD22D403AC7
:107C50005E97E63932DD8C3987FF323993FED838AA
:107C60008EDA7E38B0932438302ACA37469E6F3772
:107C70002AF014371420BA363B2E5F36D91A043650
:107C800025E6A83557904D35A819F2345082963420
:107C900087CA3A3487F2DE3388FA8233C3E2263366
:107CA0006FABCA32C7546E3204DF11325E4AB5314F
:107CB0000E9758314DC5FB3056D59E3061C74130C7
:107CC000A79BE42F6252872FCCEB292F1E68CC2E66
:107CD00092C76E2E620A112EC730B32DFC3A552D75
:107CE0003929F72CBAFB982CB9B23A2C6F4EDC2B01
:107CF00017CF7D2BEB341F2B2680C02A01B1612AC0
:107D0000B8C7022A85C4A329A2A744294B71E52834
:107D1000B921862828B92628D337C727F49D672795
:107D2000C7EB07278621A8266C3F4826B645E825DD
:107D30009D3488255E0C282533CDC72458776724C9
:107D4000080B07247F88A623F8EF4523AF41E522DF
:107D5000E07D8422C5A423229CB6C221A0B3612168
:107D60000C9C00211C709F200D303E201BDCDC1F72
:107D700081747B1F7BF9191F466BB81E1ECA561EE5
:107D80003F16F51DE54F931D4D77311DB38CCF1C6C
:107D900053906D1C6A820B1C3563A91BEF32471B85
:107DA000D6F1E41A26A0821A1B3E201AF3CBBD1985
:107DB000EA495B193CB8F81828179618E966331891
:107DC000BCA7D017DED96D178DFD0A170513A816AD
:107DD000831A45164514E21586007F1586DF1B15AC
:107DE0007FB1B814B1765514582FF213B1DB8E134E
:107DF000F97B2B136F10C8124E996412D51601121D
:107E000041899D11CFF03911BD4DD61048A0721097
:107E1000ADE80E102B27AB0FFF5B470F6687E30E15
:107E20009EA97F0EE4C21B0E76D3B70D92DB530DD5
:107E300076DBEF0C5ED38B0C89C3270C35ACC30B00
:107E40009F8D5F0B0568FB0AA53B970ABD08330AA7
:107E500089CFCE0949906A093A4B06099A00A208CF
:107E6000A7B03D089E5BD907BE01750745A3100763
:107E70006F40AC067CD94706A96EE30535007F0547
:107E80005C8E1A055D19B60477A15104E626ED0350
:107E9000EAA98803BF2A2403A4A9BF02D7265B024C
:107EA00097A2F601201D9201B1962D01880FC900FD
:107EB000E3876400000000001D789BFF78F036FF28
:107EC0004F69D2FEE0E26DFE695D09FE29D9A4FD8D
:107ED0005C5640FD41D5DBFC165677FC1AD912FCE6
:107EE000895EAEFBA3E649FBA471E5FACBFF80FAFD
:107EF00057911CFA8426B8F991BF53F9BB5CEFF88F
:107F000042FE8AF862A426F8594FC2F766FF5DF771
:107F1000C6B4F9F6B76F95F6773031F643F7CCF57E
:107F20005BC468F5FB9704F56172A0F4CB533CF495
:107F3000773CD8F3A22C74F38A2410F36E24ACF2AD
:107F40008A2C48F21C3DE4F1625680F19A781CF1CB
:107F500001A4B8F0D5D854F05317F1EFB85F8DEF06
:107F600043B229EF310FC6EEBF7662EE2BE9FEED8C
:107F7000B2669BED91EF37ED0784D4EC4F2471ECA2
:107F8000A8D00DEC4F89AAEB814E47EB7A20E4EAAA
:107F90007AFF80EABBEB1DEA7DE5BAE9FBEC57E925
:107FA0007302F5E8222692E844582FE81799CCE7A7
:107FB000D8E869E7C44707E716B6A4E60D3442E6F9
:107FC000E5C1DFE5DA5F7DE52A0E1BE511CDB8E4FA
:107FD000CB9C56E4967DF4E3AD6F92E34D7330E3B2
:107FE000B388CEE21BB06CE2C1E90AE2E235A9E156
:107FF000BA9447E18506E6E07F8B84E0E52323E041
:10800000F3CFC1DFE48F60DFF463FFDE604C9EDE00
:1080100064493DDE3B5BDCDD20827BDD51BE1ADD49
:108020000810BADC817759DCF8F4F8DBA88898DB13
:10803000CD3238DBA2F3D7DA63CB77DA4ABA17DA74
:1080400094C0B7D97ADE57D93914F8D80C6298D8C9
:108050002DC838D8D846D9D747DE79D7B58E1AD7A4
:108060005E58BBD67B3B5CD64838FDD5FF4E9ED5CF
:10807000DA7F3FD515CBE0D4E93082D491B123D457
:10808000474DC5D3460467D3C7D608D304C5AAD283
:1080900039CF4CD29EF5EED16E3891D1E29733D1E3
:1080A0003414D6D09EAD78D059641BD09F38BECF43
:1080B000AA2A61CFB33A04CFF268A7CEA2B54ACEBE
:1080C000FC20EECD39AB91CD915435CD3D1DD9CCB1
:1080D00078057DCC790D21CC7935C5CBB07D69CBC8
:1080E00058E60DCBA96FB2CADB1957CA27E5FBC901
:1080F000C5D1A0C9ECDF45C9D60FEBC8BA6190C89D
:10810000D0D535C8506CDBC7722581C76D0127C734
:108110007900CDC6CE2273C6A26819C62ED2BFC5BD
:10812000A95F66C549110DC546E7B3C4D7E15AC476
:10813000330102C49045A9C326AF50C32A3EF8C2FA
:10814000D4F29FC25ACD47C2F3CDEFC1D4F497C148
:10815000334240C148B6E8C0485191C068133AC0A4
:10816000DFFCE2BFE30D8CBFA84635BF65A7DEBECE
:108170004F3088BE9BE131BE7FBBDBBD30BE85BDCD
:10818000E2E92FBDCB3EDABC1FBD84BC13652FBC1A
:10819000DD36DABBB03285BBC05830BB43A9DBBA91
:1081A0006D2487BA71CA32BA839BDEB9D8978AB96F
:1081B000A4BF36B91913E3B86D928FB8D13D3CB85E
:1081C0007A15E9B79B1996B7674A43B712A8F0B674
:1081D000CD329EB6CDEA4BB643D0F9B562E3A7B532
:1081E0005E2456B5689304B5B330B3B470FC61B483
:1081F000D3F610B40C20C0B34F786FB3CCFF1EB3CE
:10820000B5B6CEB23C9D7EB292B32EB2E9F9DEB1E4
:1082100071708FB15B1740B1DAEEF0B01DF7A1B00D
:10822000553053B0B39A04B06736B6AFA20368AF07
:1082300093021AAF6C33CCAE5B967EAE922B31AE0E
:108240003EF3E3AD92ED96ADBA1A4AADE87AFDACD5
:108250004B0EB1AC10D564AC69CF18AC83FDCCAB80
:108260008D5F81ABB5F535AB2CC0EAAA1EBF9FAAC6
:10827000BAF254AA2E5B0AAAA8F8BFA957CB75A9CF
:1082800067D32BA90611E2A8638498A8AA2D4FA84A
:10829000080D06A8AC22BDA7C06E74A774F12BA769
:1082A000F2AAE3A6689B9BA603C353A6EE210CA6E5
:1082B00055B8C4A566867DA54B8C36A531CAEFA4FA
:1082C0004340A9A4ACEE62A499D51CA434F5D6A36E
:1082D000A84D91A320DF4BA3C8A906A3C9ADC1A295
:1082E0004FEB7CA2846238A29213F4A1A3FEAFA14B
:1082F000E1236CA1768328A18C1DE5A04DF2A1A0FD
:10830000E1015FA0734C1CA02AD2D99F3193979FA3
:10831000B08F559FD0C7139FB93BD29E94EB909ED0
:108320008AD74F9EC1FF0E9E6364CE9D97058E9D9A
:1083300085E34D9D54FE0D9D2C56CE9C34EB8E9CBA
:1083400093BD4F9C70CD109CF31AD29B41A6939B7A
:10835000816F559BDA76179B71BCD99A6E409C9AB7
:10836000F5025F9A2D04229A3B44E59945C3A899EA
:108370006F816C99E07E3099BCBBF4982838B9982D
:1083800049F47D9843F042983B2C089855A8CD9726
:10839000B56493977F615997D79E1F97E01CE69627
:1083A000BEDBAC9694DB7396861C3B96B69E02961B
:1083B0004762CA955C67929517AE5A959C3623958D
:1083C0000B01EC94870DB594335C7E942FED4794AC
:1083D0009EC01194A0D6DB93572FA693E4CA709346
:1083E00068A93B9304CB0693D92FD29206D89D92CD
:1083F000ACC36992ECF23592E4650292B61CCF915F
:1084000081179C91635669917DD93691EEA00491B4
:10841000D4ACD2904EFDA0907C926F907B6C3E903D
:10842000698B0D9066EFDC8F8F98AC8F01877C8F06
:10843000DBBA4C8F3A341D8F3BF3ED8EFBF7BE8ECB
:108440009842908E2ED3618EDAA9338EB7C6058EF0
:10845000E429D88D7BD3AA8D99C37D8D59FA508D8F
:10846000D877248D303CF88C7D47CC8CDA99A08C61
:108470006233758C2F144A8C5D3C1F8C05ACF48BD9
:108480004363CA8B2F62A08BE4A8768B7C374D8B1D
:10849000110E248BBB2CFB8A9493D28AB442AA8AF5
:1084A000363A828A317A5A8ABE02338AF5D30B8AE7
:1084B000EFEDE489C350BE898AFC97895AF171892E
:1084C0004C2F4C8977B62689F2860189D3A0DC88A7
:1084D0003204B88825B19388C2A76F8821E84B88F9
:1084E00056722888774605889B64E287D7CCBF8779
:1084F000417F9D87EC7B7B87EFC259875E5438872D
:108500004E301787D356F68602C8D586EE83B586D9
:10851000AC8A95864FDC7586EB78568692603786F6
:10852000599318865311FA8591DADB8528EFBD85BA
:10853000284FA085A5FA8285B0F165855C34498510
:10854000BBC22C85DD9C1085D4C2F484B134D9849F
:1085500086F2BD8462FCA2845852888477F46D84CC
:10856000CFE25384701D3A846CA42084D0770784B2
:10857000AD97EE831204D6830EBDBD83B0C2A58332
:1085800007158E8322B476830FA05F83DCD84883DF
:10859000975E32834E311C8310510683E8BDF08212
:1085A000E577DB82147FC68281D3B1823A759D82E2
:1085B0004B648982C0A07582A62A628208024F821B
:1085C000F3263C8271992982905917825867058257
:1085D000D7C2F381166CE2812163D18101A8C081E9
:1085E000C23AB0816D1BA0810C4A9081A9C68081DE
:1085F0004E91718104AA6281D4105481C7C545810E
:10860000E6C837813A1A2A81CAB91C81A0A70F810E
:10861000C4E302813C6EF6801247EA804C6EDE8035
:10862000F2E3D2800AA8C7809DBABC80AF1BB2809B
:1086300049CBA78071C99D802C16948080B18A8017
:10864000749B81800DD47880505B7080433168804A
:10865000EB5560804CC958806B8B51804D9C4A8093
:10866000F6FB43806AAA3D80ACA73780C2F3318015
:10867000AD8E2C807278278014B1228095381E80B0
:10868000F80E1A80403416806FA81280886B0F8015
:108690008C7D0C807EDE09805E8E07802F8D0580AC
:1086A000F1DA0380A67702804E630180EA9D0080A4
:1086B0007A270080000000807A270080EA9D0080F1
:1086C0004E630180A6770280F1DA03802F8D05804A
:1086D0005E8E07807EDE09808C7D0C80886B0F802B
:1086E0006FA8128040341680F80E1A8095381E80CC
:1086F00014B1228072782780AD8E2C80C2F3318035
:10870000ACA737806AAA3D80F6FB43804D9C4A8027
:108710006B8B51804CC95880EB5560804331688029
:10872000505B70800DD47880749B818080B18A808A
:108730002C16948071C99D8049CBA780AF1BB28055
:108740009DBABC800AA8C780F2E3D2804C6EDE805E
:108750001247EA803C6EF680C4E30281A0A70F8135
:10876000CAB91C813A1A2A81E6C83781C7C5458132
:10877000D410548104AA62814E917181A9C680816E
:108780000C4A90816D1BA081C23AB08101A8C081C2
:108790002163D181166CE281D7C2F38158670582CB
:1087A0009059178271992982F3263C8208024F82E0
:1087B000A62A6282C0A075824B6489823A759D8226
:1087C00081D3B182147FC682E577DB82E8BDF08277
:1087D000105106834E311C83975E3283DCD8488368
:1087E0000FA05F8322B4768307158E83B0C2A58362
:1087F0000EBDBD831204D683AD97EE83D077078478
:108800006CA42084701D3A84CFE2538477F46D8485
:108810005852888462FCA28486F2BD84B134D98423
:10882000D4C2F484DD9C1085BBC22C855C344985A0
:10883000B0F16585A5FA8285284FA08528EFBD8512
:1088400091DADB855311FA85599318869260378641
:10885000EB7856864FDC7586AC8A9586EE83B586B6
:1088600002C8D586D356F6864E3017875E543887B1
:10887000EFC25987EC7B7B87417F9D87D7CCBF8731
:108880009B64E287774605885672288821E84B88E2
:10889000C2A76F8825B193883204B888D3A0DC883A
:1088A000F286018977B626894C2F4C895AF1718955
:1088B0008AFC9789C350BE89EFEDE489F5D30B8A12
:1088C000BE02338A317A5A8A363A828AB442AA8AF6
:1088D0009493D28ABB2CFB8A110E248B7C374D8B50
:1088E000E4A8768B2F62A08B4363CA8B05ACF48B14
:1088F0005D3C1F8C2F144A8C6233758CDA99A08CE6
:108900007D47CC8C303CF88CD877248D59FA508D2B
:1089100099C37D8D7BD3AA8DE429D88DB7C6058EEA
:10892000DAA9338E2ED3618E9842908EFBF7BE8EDD
:108930003BF3ED8E3A341D8FDBBA4C8F01877C8F71
:108940008F98AC8F66EFDC8F698B0D907B6C3E90BF
:108950007C926F904EFDA090D4ACD290EEA004918A
:108960007DD936916356699181179C91B61CCF9140
:10897000E4650292ECF23592ACC3699206D89D92FE
:10898000D92FD29204CB069368A93B93E4CA709383
:10899000572FA693A0D6DB939EC011942FED47943A
:1089A000335C7E94870DB5940B01EC949C36239533
:1089B00017AE5A955C6792954762CA95B69E029625
:1089C000861C3B9694DB7396BEDBAC96E01CE69669
:1089D000D79E1F977F615997B564939755A8CD97F8
:1089E0003B2C089843F0429849F47D982838B99870
:1089F000BCBBF498E07E30996F816C9945C3A8990F
:108A00003B44E5992D04229AF5025F9A6E409C9AA8
:108A100071BCD99ADA76179B816F559B41A6939BBF
:108A2000F31AD29B70CD109C93BD4F9C34EB8E9C5F
:108A30002C56CE9C54FE0D9D85E34D9D97058E9D35
:108A40006364CE9DC1FF0E9E8AD74F9E94EB909E8D
:108A5000B93BD29ED0C7139FB08F559F3193979F3C
:108A60002AD2D99F734C1CA0E1015FA04DF2A1A0B6
:108A70008C1DE5A0768328A1E1236CA1A3FEAFA104
:108A80009213F4A1846238A24FEB7CA2C9ADC1A2BB
:108A9000C8A906A320DF4BA3A84D91A334F5D6A304
:108AA00099D51CA4ACEE62A44340A9A431CAEFA49A
:108AB0004B8C36A566867DA555B8C4A5EE210CA6BF
:108AC00003C353A6689B9BA6F2AAE3A674F12BA747
:108AD000C06E74A7AC22BDA7080D06A8AA2D4FA88A
:108AE000638498A80611E2A867D32BA957CB75A970
:108AF000A8F8BFA92E5B0AAABAF254AA1EBF9FAA61
:108B00002CC0EAAAB5F535AB8D5F81AB83FDCCAB4C
:108B100069CF18AC10D564AC4B0EB1ACE87AFDACA3
:108B2000BA1A4AAD92ED96AD3EF3E3AD922B31AE5B
:108B30005B967EAE6C33CCAE93021AAFA20368AFE5
:108B40006736B6AFB39A04B0553053B01DF7A1B035
:108B5000DAEEF0B05B1740B171708FB1E9F9DEB1B8
:108B600092B32EB23C9D7EB2B5B6CEB2CCFF1EB350
:108B70004F786FB30C20C0B3D3F610B470FC61B45F
:108B8000B330B3B4689304B55E2456B562E3A7B5B9
:108B900043D0F9B5CDEA4BB6CD329EB612A8F0B6A9
:108BA000674A43B79B1996B77A15E9B7D13D3CB8E8
:108BB0006D928FB81913E3B8A4BF36B9D8978AB9A4
:108BC000839BDEB971CA32BA6D2487BA43A9DBBA76
:108BD000C05830BBB03285BBDD36DABB13652FBC65
:108BE0001FBD84BCCB3EDABCE2E92FBD30BE85BDE3
:108BF0007FBBDBBD9BE131BE4F3088BE65A7DEBECB
:108C0000A84635BFE30D8CBFDFFCE2BF68133AC056
:108C1000485191C048B6E8C0334240C1D4F497C12E
:108C2000F3CDEFC15ACD47C2D4F29FC22A3EF8C25B
:108C300026AF50C39045A9C3330102C4D7E15AC43B
:108C400046E7B3C449110DC5A95F66C52ED2BFC59D
:108C5000A26819C6CE2273C67900CDC66D0127C79A
:108C6000722581C7506CDBC7D0D535C8BA6190C8B2
:108C7000D60FEBC8ECDF45C9C5D1A0C927E5FBC9B4
:108C8000DB1957CAA96FB2CA58E60DCBB07D69CBC4
:108C90007935C5CB790D21CC78057DCC3D1DD9CC5E
:108CA000915435CD39AB91CDFC20EECDA2B54ACE55
:108CB000F268A7CEB33A04CFAA2A61CF9F38BECFBD
:108CC00059641BD09EAD78D03414D6D0E29733D1FE
:108CD0006E3891D19EF5EED139CF4CD204C5AAD2CF
:108CE000C7D608D3460467D3474DC5D391B123D423
:108CF000E93082D415CBE0D4DA7F3FD5FF4E9ED544
:108D00004838FDD57B3B5CD65E58BBD6B58E1AD7AE
:108D100047DE79D7D846D9D72DC838D80C6298D82D
:108D20003914F8D87ADE57D994C0B7D94ABA17DAC5
:108D300063CB77DAA2F3D7DACD3238DBA88898DBB9
:108D4000F8F4F8DB817759DC0810BADC51BE1ADD83
:108D500020827BDD3B5BDCDD64493DDE604C9EDEDA
:108D6000F463FFDEE48F60DFF3CFC1DFE52323E0B0
:108D70007F8B84E08506E6E0BA9447E1E235A9E11D
:108D8000C1E90AE21BB06CE2B388CEE24D7330E376
:108D9000AD6F92E3967DF4E3CB9C56E411CDB8E43D
:108DA0002A0E1BE5DA5F7DE5E5C1DFE50D3442E61D
:108DB00016B6A4E6C44707E7D8E869E71799CCE7F1
:108DC00044582FE8222692E87302F5E8FBEC57E9B5
:108DD0007DE5BAE9BBEB1DEA7AFF80EA7A20E4EA96
:108DE000814E47EB4F89AAEBA8D00DEC4F2471ECD4
:108DF0000784D4EC91EF37EDB2669BED2BE9FEEDE5
:108E0000BF7662EE310FC6EE43B229EFB85F8DEF49
:108E10005317F1EFD5D854F001A4B8F09A781CF1AB
:108E2000625680F11C3DE4F18A2C48F26E24ACF2CB
:108E30008A2410F3A22C74F3773CD8F3CB533CF480
:108E40006172A0F4FB9704F55BC468F543F7CCF5B9
:108E5000773031F6B76F95F6C6B4F9F666FF5DF771
:108E6000594FC2F762A426F842FE8AF8BB5CEFF8BD
:108E700091BF53F98426B8F957911CFACBFF80FAB9
:108E8000A471E5FAA3E649FB895EAEFB1AD912FC90
:108E9000165677FC41D5DBFC5C5640FD29D9A4FD74
:108EA000695D09FEE0E26DFE4F69D2FE78F036FFA3
:108EB0001D789BFFFFFFFF7F86D8FF7F1662FF7F35
:108EC000B29CFE7F5A88FD7F0F25FC7FD172FA7F0E
:108ED000A271F87F8221F67F7482F37F7894F07F0D
:108EE0009157ED7FC0CBE97F08F1E57F6BC7E17F4C
:108EF000EC4EDD7F8E87D87F5371D37F3E0CCE7FC3
:108F00005458C87F9655C27F0A04BC7FB363B57FAF
:108F10009574AE7FB436A77F15AA9F7FBDCE977F8D
:108F2000B0A48F7FF32B877F8C647E7F804E757F0C
:108F3000D4E96B7F8F36627FB734587F51E44D7F21
:108F40006345437FF657387F0E1C2D7FB491217FF8
:108F5000EEB8157FC491097F3C1CFD7E6058F07E01
:108F60003646E37EC6E5D57E1A37C87E393ABA7EE4
:108F70002CEFAB7EFC559D7EB26E8E7E57397F7E88
:108F8000F4B56F7E93E45F7E3EC54F7EFF573F7E14
:108F9000DF9C2E7EEA931D7E293D0C7EA898FA7DEB
:108FA00070A6E87D8F66D67D0DD9C37DF8FDB07DB6
:108FB0005AD59D7D405F8A7DB59B767DC68A627D50
:108FC0007F2C4E7DEC80397D1B88247D18420F7DDF
:108FD000F0AEF97CB2CEE37C69A1CD7C2427B77CCE
:108FE000F15FA07CDE4B897CF9EA717C503D5A7CB4
:108FF000F242427CEEFB297C5368117C3088F87B7E
:10900000945BDF7B90E2C57B311DAC7B890B927B4F
:10901000A8AD777B9E035D7B7A0D427B4FCB267B91
:109020002C3D0B7B2363EF7A453DD37AA4CBB67AF4
:10903000500E9A7A5B057D7AD8B05F7AD810427A62
:109040006F25247AADEE057AA76CE7796E9FC87913
:109050001587A979B1238A7954756A79127C4A797E
:10906000FE372A792DA90979B2CFE878A2ABC77863
:10907000113DA67814848478BF80627829334078C3
:10908000659B1D7889B9FA77AA8DD777DF17B477F2
:109090003E589077DB4E6C77CEFB47772D5F23777A
:1090A0000E79FE768949D976B4D0B376A60E8E763F
:1090B000760368763DAF417611121B760B2CF47562
:1090C00042FDCC75CF85A575CAC57D754CBD55755E
:1090D0006C6C2D7545D30475EFF1DB7484C8B274E4
:1090E0001C578974D19D5F74BD9C3574FB530B7400
:1090F000A3C3E073D1EBB5739ECC8A7326665F730E
:1091000083B83373D0C307732888DB72A705AF72A7
:10911000673C8272852C55721CD627724939FA71C8
:109120002656CC71D22C9E7168BD6F7105084171B5
:10913000C50C1271C6CBE2702545B370FF78837001
:10914000716753709A1023709774F26F8593C16F93
:10915000846D906FB2025F6F2C532D6F125FFB6EA8
:109160008326C96E9DA9966E7FE8636E4AE3306ED2
:109170001C9AFD6D140DCA6D543C966DFA27626DF4
:1091800027D02D6DFC34F96C9856C46C1C358F6C4F
:10919000A9D0596C6029246C623FEE6BD112B86B78
:1091A000CDA3816B79F24A6BF5FE136B64C9DC6A5F
:1091B000E951A56AA4986D6AB99D356A4A61FD694D
:1091C0007AE3C4696C248C694224536920E31969E9
:1091D0002961E068819EA6684B9B6C68AB5732683A
:1091E000C5D3F767BD0FBD67B70B8267D8C74667A2
:1091F00044440B672081CF66917E9366BB3C5766E3
:10920000C5BB1A66D3FBDD650BFDA06592BF636528
:109210008F4326652689E8647F90AA64BF596C64F1
:109220000DE52D649032EF636D42B063CC14716331
:10923000D4A93163AC01F2627B1CB26269FA71623B
:109240009D9B31623F00F1617628B0616C146F61C3
:1092500047C42D613038EC605070AA60CF6C6860F4
:10926000D62D26608DB3E35F1FFEA05FB30D5E5F5A
:1092700074E21A5F8A7CD75E1FDC935E5D01505EEC
:109280006EEC0B5E7C9DC75DB114835D37523E5D15
:109290003856F95CE020B45C58B26E5CCC0A295CAC
:1092A000672AE35B54119D5BBDBF565BCF35105BF6
:1092B000B573C95A9A79825AAB473B5A12DEF359B1
:1092C000FD3CAC59986464590E551C598C0ED45809
:1092D00040918B5854DD4258F8F2F95756D2B057A6
:1092E0009D7B6757FAEE1D57992CD456A9348A56A0
:1092F00058074056D2A4F555460DAB55E24060558F
:10930000D43F15554B0ACA5473A07E547D02335482
:109310009730E753F02A9B53B5F14E53188502530B
:1093200046E5B5526E126952C20C1C526ED4CE5133
:10933000A569815194CC33516DFDE5505EFC975089
:1093400099C949504D65FB4FABCFAC4FE3085E4F19
:1093500026110F4FA5E8BF4E8F8F704E1706214E76
:109360006E4CD14DC462814D4B49314D3400E14CBE
:10937000B187904CF4DF3F4C2D09EF4B90039E4B8F
:109380004DCF4C4B986CFB4AA2DBA94A9E1C584A15
:10939000BD2F064A3315B44933CD6149EE570F4905
:1093A00099B5BC4865E6694886EA16482FC2C347A6
:1093B000936D7047E7EC1C475C40C94628687546CA
:1093C0007D6421468F35CD4593DB7845BD562445D8
:1093D00040A7CF4450CD7A4423C92544ED9AD043C9
:1093E000E1427B4335C125431E16D042D0417A422B
:1093F00081442442651ECE41B1CF77419B58214123
:1094000058B9CA401DF2734021031D4098ECC53F76
:10941000B8AE6E3FB849173FCDBDBF3E2C0B683E7E
:109420000D32103EA632B83D2C0D603DD6C1073D31
:10943000DA50AF3C70BA563CCDFEFD3B291EA53B31
:10944000BA184C3BB7EEF23A57A0993AD22D403AAF
:109450005E97E63932DD8C3987FF323993FED83892
:109460008EDA7E38B0932438302ACA37469E6F375A
:109470002AF014371420BA363B2E5F36D91A043638
:1094800025E6A83557904D35A819F2345082963408
:1094900087CA3A3487F2DE3388FA8233C3E226334E
:1094A0006FABCA32C7546E3204DF11325E4AB53137
:1094B0000E9758314DC5FB3056D59E3061C74130AF
:1094C000A79BE42F6252872FCCEB292F1E68CC2E4E
:1094D00092C76E2E620A112EC730B32DFC3A552D5D
:1094E0003929F72CBAFB982CB9B23A2C6F4EDC2BE9
:1094F00017CF7D2BEB341F2B2680C02A01B1612AA8
:10950000B8C7022A85C4A329A2A744294B71E5281C
:10951000B921862828B92628D337C727F49D67277D
:10952000C7EB07278621A8266C3F4826B645E825C5
:109530009D3488255E0C282533CDC72458776724B1
:10954000080B07247F88A623F8EF4523AF41E522C7
:10955000E07D8422C5A423229CB6C221A0B3612150
:109560000C9C00211C709F200D303E201BDCDC1F5A
:1095700081747B1F7BF9191F466BB81E1ECA561ECD
:109580003F16F51DE54F931D4D77311DB38CCF1C54
:1095900053906D1C6A820B1C3563A91BEF32471B6D
:1095A000D6F1E41A26A0821A1B3E201AF3CBBD196D
:1095B000EA495B193CB8F81828179618E966331879
:1095C000BCA7D017DED96D178DFD0A170513A81695
:1095D000831A45164514E21586007F1586DF1B1594
:1095E0007FB1B814B1765514582FF213B1DB8E1336
:1095F000F97B2B136F10C8124E996412D516011205
:1096000041899D11CFF03911BD4DD61048A072107F
:10961000ADE80E102B27AB0FFF5B470F6687E30EFD
:109620009EA97F0EE4C21B0E76D3B70D92DB530DBD
:1096300076DBEF0C5ED38B0C89C3270C35ACC30BE8
:109640009F8D5F0B0568FB0AA53B970ABD08330A8F
:1096500089CFCE0949906A093A4B06099A00A208B7
:10966000A7B03D089E5BD907BE01750745A310074B
:109670006F40AC067CD94706A96EE30535007F052F
:109680005C8E1A055D19B60477A15104E626ED0338
:10969000EAA98803BF2A2403A4A9BF02D7265B0234
:1096A00097A2F601201D9201B1962D01880FC900E5
:1096B000E3876400000000001D789BFF78F036FF10
:1096C0004F69D2FEE0E26DFE695D09FE29D9A4FD75
:1096D0005C5640FD41D5DBFC165677FC1AD912FCCE
:1096E000895EAEFBA3E649FBA471E5FACBFF80FAE5
:1096F00057911CFA8426B8F991BF53F9BB5CEFF877
:1097000042FE8AF862A426F8594FC2F766FF5DF759
:10971000C6B4F9F6B76F95F6773031F643F7CCF566
:109720005BC468F5FB9704F56172A0F4CB533CF47D
:10973000773CD8F3A22C74F38A2410F36E24ACF295
:109740008A2C48F21C3DE4F1625680F19A781CF1B3
:1097500001A4B8F0D5D854F05317F1EFB85F8DEFEE
:1097600043B229EF310FC6EEBF7662EE2BE9FEED74
:10977000B2669BED91EF37ED0784D4EC4F2471EC8A
:10978000A8D00DEC4F89AAEB814E47EB7A20E4EA92
:109790007AFF80EABBEB1DEA7DE5BAE9FBEC57E90D
:1097A0007302F5E8222692E844582FE81799CCE78F
:1097B000D8E869E7C44707E716B6A4E60D3442E6E1
:1097C000E5C1DFE5DA5F7DE52A0E1BE511CDB8E4E2
:1097D000CB9C56E4967DF4E3AD6F92E34D7330E39A
:1097E000B388CEE21BB06CE2C1E90AE2E235A9E13E
:1097F000BA9447E18506E6E07F8B84E0E52323E029
:10980000F3CFC1DFE48F60DFF463FFDE604C9EDEE8
:1098100064493DDE3B5BDCDD20827BDD51BE1ADD31
:109820000810BADC817759DCF8F4F8DBA88898DBFB
:10983000CD3238DBA2F3D7DA63CB77DA4ABA17DA5C
:1098400094C0B7D97ADE57D93914F8D80C6298D8B1
:109850002DC838D8D846D9D747DE79D7B58E1AD78C
:109860005E58BBD67B3B5CD64838FDD5FF4E9ED5B7
:10987000DA7F3FD515CBE0D4E93082D491B123D43F
:10988000474DC5D3460467D3C7D608D304C5AAD26B
:1098900039CF4CD29EF5EED16E3891D1E29733D1CB
:1098A0003414D6D09EAD78D059641BD09F38BECF2B
:1098B000AA2A61CFB33A04CFF268A7CEA2B54ACEA6
:1098C000FC20EECD39AB91CD915435CD3D1DD9CC99
:1098D00078057DCC790D21CC7935C5CBB07D69CBB0
:1098E00058E60DCBA96FB2CADB1957CA27E5FBC9E9
:1098F000C5D1A0C9ECDF45C9D60FEBC8BA6190C885
:10990000D0D535C8506CDBC7722581C76D0127C71C
:109910007900CDC6CE2273C6A26819C62ED2BFC5A5
:10992000A95F66C549110DC546E7B3C4D7E15AC45E
:10993000330102C49045A9C326AF50C32A3EF8C2E2
:10994000D4F29FC25ACD47C2F3CDEFC1D4F497C130
:10995000334240C148B6E8C0485191C068133AC08C
:10996000DFFCE2BFE30D8CBFA84635BF65A7DEBEB6
:109970004F3088BE9BE131BE7FBBDBBD30BE85BDB5
:10998000E2E92FBDCB3EDABC1FBD84BC13652FBC02
:10999000DD36DABBB03285BBC05830BB43A9DBBA79
:1099A0006D2487BA71CA32BA839BDEB9D8978AB957
:1099B000A4BF36B91913E3B86D928FB8D13D3CB846
:1099C0007A15E9B79B1996B7674A43B712A8F0B65C
:1099D000CD329EB6CDEA4BB643D0F9B562E3A7B51A
:1099E0005E2456B5689304B5B330B3B470FC61B46B
:1099F000D3F610B40C20C0B34F786FB3CCFF1EB3B6
:109A0000B5B6CEB23C9D7EB292B32EB2E9F9DEB1CC
:109A100071708FB15B1740B1DAEEF0B01DF7A1B0F5
:109A2000553053B0B39A04B06736B6AFA20368AFEF
:109A300093021AAF6C33CCAE5B967EAE922B31AEF6
:109A40003EF3E3AD92ED96ADBA1A4AADE87AFDACBD
:109A50004B0EB1AC10D564AC69CF18AC83FDCCAB68
:109A60008D5F81ABB5F535AB2CC0EAAA1EBF9FAAAE
:109A7000BAF254AA2E5B0AAAA8F8BFA957CB75A9B7
:109A800067D32BA90611E2A8638498A8AA2D4FA832
:109A9000080D06A8AC22BDA7C06E74A774F12BA751
:109AA000F2AAE3A6689B9BA603C353A6EE210CA6CD
:109AB00055B8C4A566867DA54B8C36A531CAEFA4E2
:109AC0004340A9A4ACEE62A499D51CA434F5D6A356
:109AD000A84D91A320DF4BA3C8A906A3C9ADC1A27D
:109AE0004FEB7CA2846238A29213F4A1A3FEAFA133
:109AF000E1236CA1768328A18C1DE5A04DF2A1A0E5
:109B0000E1015FA0734C1CA02AD2D99F3193979F8B
:109B1000B08F559FD0C7139FB93BD29E94EB909EB8
:109B20008AD74F9EC1FF0E9E6364CE9D97058E9D82
:109B300085E34D9D54FE0D9D2C56CE9C34EB8E9CA2
:109B400093BD4F9C70CD109CF31AD29B41A6939B62
:109B5000816F559BDA76179B71BCD99A6E409C9A9F
:109B6000F5025F9A2D04229A3B44E59945C3A899D2
:109B70006F816C99E07E3099BCBBF4982838B99815
:109B800049F47D9843F042983B2C089855A8CD970E
:109B9000B56493977F615997D79E1F97E01CE6960F
:109BA000BEDBAC9694DB7396861C3B96B69E029603
:109BB0004762CA955C67929517AE5A959C36239575
:109BC0000B01EC94870DB594335C7E942FED479494
:109BD0009EC01194A0D6DB93572FA693E4CA70932E
:109BE00068A93B9304CB0693D92FD29206D89D92B5
:109BF000ACC36992ECF23592E4650292B61CCF9147
:109C000081179C91635669917DD93691EEA004919C
:109C1000D4ACD2904EFDA0907C926F907B6C3E9025
:109C2000698B0D9066EFDC8F8F98AC8F01877C8FEE
:109C3000DBBA4C8F3A341D8F3BF3ED8EFBF7BE8EB3
:109C40009842908E2ED3618EDAA9338EB7C6058ED8
:109C5000E429D88D7BD3AA8D99C37D8D59FA508D77
:109C6000D877248D303CF88C7D47CC8CDA99A08C49
:109C70006233758C2F144A8C5D3C1F8C05ACF48BC1
:109C80004363CA8B2F62A08BE4A8768B7C374D8B05
:109C9000110E248BBB2CFB8A9493D28AB442AA8ADD
:109CA000363A828A317A5A8ABE02338AF5D30B8ACF
:109CB000EFEDE489C350BE898AFC97895AF1718916
:109CC0004C2F4C8977B62689F2860189D3A0DC888F
:109CD0003204B88825B19388C2A76F8821E84B88E1
:109CE00056722888774605889B64E287D7CCBF8761
:109CF000417F9D87EC7B7B87EFC259875E54388715
:109D00004E301787D356F68602C8D586EE83B586C1
:109D1000AC8A95864FDC7586EB78568692603786DE
:109D2000599318865311FA8591DADB8528EFBD85A2
:109D3000284FA085A5FA8285B0F165855C344985F8
:109D4000BBC22C85DD9C1085D4C2F484B134D98487
:109D500086F2BD8462FCA2845852888477F46D84B4
:109D6000CFE25384701D3A846CA42084D07707849A
:109D7000AD97EE831204D6830EBDBD83B0C2A5831A
:109D800007158E8322B476830FA05F83DCD84883C7
:109D9000975E32834E311C8310510683E8BDF082FA
:109DA000E577DB82147FC68281D3B1823A759D82CA
:109DB0004B648982C0A07582A62A628208024F8203
:109DC000F3263C827199298290591782586705823F
:109DD000D7C2F381166CE2812163D18101A8C081D1
:109DE000C23AB0816D1BA0810C4A9081A9C68081C6
:109DF0004E91718104AA6281D4105481C7C54581F6
:109E0000E6C837813A1A2A81CAB91C81A0A70F81F6
:109E1000C4E302813C6EF6801247EA804C6EDE801D
:109E2000F2E3D2800AA8C7809DBABC80AF1BB28083
:109E300049CBA78071C99D802C16948080B18A80FF
:109E4000749B81800DD47880505B70804331688032
:109E5000EB5560804CC958806B8B51804D9C4A807B
:109E6000F6FB43806AAA3D80ACA73780C2F33180FD
:109E7000AD8E2C807278278014B1228095381E8098
:109E8000F80E1A80403416806FA81280886B0F80FD
:109E90008C7D0C807EDE09805E8E07802F8D058094
:109EA000F1DA0380A67702804E630180EA9D00808C
:109EB0007A270080000000807A270080EA9D0080D9
:109EC0004E630180A6770280F1DA03802F8D058032
:109ED0005E8E07807EDE09808C7D0C80886B0F8013
:109EE0006FA8128040341680F80E1A8095381E80B4
:109EF00014B1228072782780AD8E2C80C2F331801D
:109F0000ACA737806AAA3D80F6FB43804D9C4A800F
:109F10006B8B51804CC95880EB5560804331688011
:109F2000505B70800DD47880749B818080B18A8072
:109F30002C16948071C99D8049CBA780AF1BB2803D
:109F40009DBABC800AA8C780F2E3D2804C6EDE8046
:109F50001247EA803C6EF680C4E30281A0A70F811D
:109F6000CAB91C813A1A2A81E6C83781C7C545811A
:109F7000D410548104AA62814E917181A9C6808156
:109F80000C4A90816D1BA081C23AB08101A8C081AA
